:100000000C944D050C9491050C9491050C9491055C
:100010000C9491050C9491050C9491050C94910508
:100020000C9491050C948D140C9491050C949105ED
:100030000C9492270C9491050C9491050C949105C5
:100040000C9491050C9491050C9402130C94910559
:100050000C94BF0A0C9491050C94890A0C94910598
:100060000C94A3190C9491050C940E230C949105F7
:100070000C9494780C9491050C949073CE19D31928
:10008000D819E119F8190F1A1F1A2F1A4C1A381C0F
:100090000F1AFA1A0B1B3A1B581B751BCF1B2A1C75
:1000A00036235D23A0231024282469241C25DC2565
:1000B000DC25DC25DC25DC25DC25DC25DC25DC2538
:1000C000DC25DC25932595259A25B225B4250A0D36
:1000D0004261743A002025642043656C6C732000F3
:1000E000204C6F77207761726E696E67206C657641
:1000F000656C3A2025642E2564000A0D466F756EE6
:100100006420424C2D4374726C3A20002564000A2E
:100110000D0A0D2121204D495353494E4720424C91
:100120002D4354524C3A202564202121000A0D3DD4
:10013000000A0D43616C6962726174696E672070B8
:10014000726573737572652073656E736F722E2E90
:10015000004F4B0A0D000A0D466C696768742D74D8
:10016000696D65202575206D696E2020543A2575CE
:10017000206D696E000A0D436F6E74726F6C3A20C9
:100180000048656164696E67486F6C64004E6F7209
:100190006D616C20284143432D4D6F646529000A31
:1001A0000D3D0A0D00416E676C654E69636B202042
:1001B0002020416E676C65526F6C6C2020202041BE
:1001C00063634E69636B20202020202041636352CB
:1001D0006F6C6C2020202020205961774779726F46
:1001E0002020202020204865696768742056616CB3
:1001F0007565204163635A20202020202020202084
:1002000047617320202020202020202020436F6D74
:10021000706173732056616C7565566F6C7461679D
:10022000655B302E31565D52656365697665724C4B
:100230006576656C4779726F20436F6D706173737B
:10024000204D6F746F7220312020202020204D6FB0
:10025000746F7220322020202020204D6F746F7226
:1002600020332020202020204D6F746F72203420F6
:1002700020202020204D6F746F72203520202020F8
:1002800020204D6F746F72203620202020202031D6
:10029000382020202020202020202020576F757417
:1002A00043616C635374617465536572766F20208B
:1002B000202020202020486F7665726761732020FF
:1002C00020202043757272656E745B302E31415D63
:1002D00043617061636974795B6D41685D4D6F74F2
:1002E0006F7220372020202020204D6F746F7220E5
:1002F000382020202020204D6F746F72203920205C
:10030000202020204D6F746F72203130202020205B
:10031000204932432D4572726F7220202020424CBA
:10032000204C696D697420202020204750535F4E77
:1003300069636B20202020204750535F526F6C6C04
:1003400020202020202E000A0D20444143206F72DF
:1003500020493243204552524F5221204368656361
:100360006B204932432C2033567265662C20444161
:100370004320616E6420424C2D4374726C000A0D60
:1003800047656E65726174696E6720646566617544
:100390006C7420506172616D657465722053657470
:1003A000202564000A0D5573696E672050617261E3
:1003B0006D6574657220536574202564000A0D47CD
:1003C000656E65726174696E672064656661756CDF
:1003D00074204D69786572205461626C65000A0D65
:1003E0004D697865722D436F6E6669673A202725DF
:1003F000732720282575204D6F746F727329000AAA
:100400000D3D000A0D414343206E6F742063616C03
:1004100069627261746564210D0A0000008F001E1C
:1004200001AD013B02CA025803E603740402058FC2
:10043000051B06A7063307BE074808D2085B09E379
:10044000096B0AF20A780BFD0B810C040D860D076F
:100450000E870E060F840F00107B10F5106E11E54D
:10046000115B12CF124213B31323149214FE146AB9
:1004700015D3153B16A11605176717C8172718833C
:1004800018DE1837198E19E319361A871AD61A2367
:100490001B6E1BB61BFD1B411C831CC31C001D3C9B
:1004A0001D751DAB1DE01D121E421E6F1E9A1EC340
:1004B0001EE91E0D1F2E1F4D1F691F841F9B1FB09D
:1004C0001FC31FD31FE11FEC1FF51FFB1FFF1F00E2
:1004D0002016010000305C00020101235D010302CF
:1004E00002B75D02040303555E03050404EF5E04D6
:1004F0000605055A6105070606F760060807071A8C
:1005000062070908088C62080A0909CF62090B0A08
:100510000A49640A0C0B0B55650B0D0C0C35660C67
:100520000E0D0D41670D0F0E0EC26B0E100F0F4D0D
:10053000680F111010DB6910121111B66A11131235
:1005400012DE6C1214131359691315141407641472
:10055000161515EA6D15001616A56E2532692E259D
:1005600031695600253364256320253033646D00DE
:10057000537461747573004552524F523A202532BC
:100580006400253469202532693A25303269002516
:1005900034696D25630025336920253369202533AF
:1005A00069202533690025336920253369202533E7
:1005B00069202533690054656D70657261747572C8
:1005C0006573202020200025634320202020200068
:1005D0002532692E25316956002533692E2531696A
:1005E00041002533692E25316941002534695720A2
:1005F0002536696D4148002532756D2F7320536192
:10060000743A2564200020203344004E6F46780061
:100610004447505300486F6D653A2533646D20257B
:1006200033642563004E6F204E6176694374726CAB
:10063000210025336920253369202533692025339E
:100640006900253369202533692025336920253346
:10065000690043757272656E747320542533692E78
:1006600025316941002533692E2531694120004932
:1006700032432533692533692533692533690025DC
:100680003369202533692025336920253369002506
:1006900033692025336920253369202533690025F6
:1006A0003369202533692025336920253369004DBE
:1006B00020536574506F696E742020202020200024
:1006C0004D53657450253369002533694E20253319
:1006D000695220202B4E0025336947202020202BF3
:1006E00052202D4E202D52002533693D5653706502
:1006F0006564002533693D48472F34202533693D23
:100700004761730025632533693D535031256325C7
:1007100033693D5350330025632533693D535032CF
:1007200025632533693D53503400737769746368DA
:100730006564204869676874207600566172696F45
:10074000207769746862656570205E0025632533D3
:10075000693D48442025632533693D4841002563B0
:100760002533693D48502025632533693D484D00B8
:1007700025632533693D48562025632533693D4867
:100780005A0025632533693D484720256325336991
:100790003D48530025632533693D53745025632537
:1007A00033693D5347500025632533693D537444F5
:1007B00025632533693D4472430025632533693D34
:1007C00047595025632533693D475949002563251D
:1007D00033693D47594425632533693D4D614900DF
:1007E00025632533693D4E474725632533693D4ED3
:1007F00053430025632533693D4E57432563253315
:10080000693D4E414C0020004C6F6F70696E6776F9
:10081000616C756520253269640025632533693D67
:100820004C474C25632533693D4C487900256325A9
:1008300033693D4C546825630025632533693D4683
:10084000475025632533693D4359430025632533CC
:10085000693D464E5225632533693D555037002585
:10086000632533693D47475025632533693D475329
:10087000740025632533693D47474925632533695E
:100880003D4453740025632533693D4E435425632D
:100890002533693D5243540025632533693D4E435A
:1008A0005025632533693D524350004D7465737480
:1008B000203C2B76203C2B5E253369004D6F746FF6
:1008C000723D2532692053703D25326900534554ED
:1008D00054494E473D253169003C202B203E746F22
:1008E00053544F5245746F20253169004F4B2100FE
:1008F0000A0D7777772E4D696B726F4B6F70746549
:10090000722E6465202863292048695379737465C1
:100910006D7320476D6248000A0D74686520757319
:1009200065206F66207468697320736F66747761E1
:100930007265206973206F6E6C79207065726D69C5
:1009400074746564200A0D6F6E206F726967696E3A
:10095000616C204D696B726F4B6F707465722D48BE
:1009600061726477617265004143542044534C00C6
:100970004A65746920736174656C6C6974005370A6
:10098000656B7472756D20736174656C6C6974202D
:10099000284C6F77207265736F6C7574696F6E2960
:1009A000005370656B7472756D20736174656C6C47
:1009B000697420283230343829005370656B7472A2
:1009C000756D20736174656C6C6974004D756C7421
:1009D000697369676E616C2050504D000A0D526555
:1009E0006365697665723A2000756E6B6E6F776E1F
:1009F0002E205573696E672050504D2E2E2E006E9E
:100A00006F7420737570706F7274656420627920E2
:100A1000686172647761726521000A0D3D3D3D3D5C
:100A20003D3D3D3D3D3D3D3D3D3D3D3D3D3D3D3DF6
:100A30003D3D3D3D3D3D3D3D3D3D3D3D3D3D3D0023
:100A40000A0D466C69676874436F6E74726F6C0A46
:100A50000D48617264776172653A25642E25640AD7
:100A60000D536F6674776172653A5625642E25645E
:100A7000256320000A0D3D3D3D3D3D3D3D3D3D3D55
:100A80003D3D3D3D3D3D3D3D3D3D3D3D3D3D3D3D96
:100A90003D3D3D3D3D3D3D3D3D0011241FBECFEF61
:100AA000D0E1DEBFCDBF11E0A0E0B1E0E6E2F5EFBE
:100AB00002C005900D92A43AB107D9F718E0A4EA54
:100AC000B1E001C01D92A036B107E1F76AEAE2E0A9
:100AD000F0E081E2809357007491AE014F5F5F4F69
:100AE00020EF37EFDA019FE0F9012F5F3F4F84914C
:100AF0008D93915097FFF8CF773911F40000FECF16
:100B0000FA019EE0819168276095915097FFFACF96
:100B10008889681721F0773911F40000FECF0C9412
:100B200052060C9400008091BA05E82FFF27EE0FC3
:100B3000FF1FEF51F94F808191818D5E9F4F14F01F
:100B400010920301808191818A5B9F4FCCF4809148
:100B500003018823A9F481E08093030180911104AB
:100B60008F5F80931104853038F088EE93E0909386
:100B7000D4018093D30104C066E970E00E94262B63
:100B800080911104992790938B0580938A0508958D
:100B90001F93CF93DF93182F882389F08EEC90E07A
:100BA0009F938F9389E890E19F938F93E091DA036D
:100BB000F091DB0309950F900F900F900F908091AB
:100BC000DD05823308F044C084EF91E00E940D14EB
:100BD000EC01112329F0CE010E9416148823D9F3C9
:100BE000C2E0D0E026E530E080911D0190911E0129
:100BF0008217930730F02196255D3F4FC730D1050E
:100C000098F38091DD059927C89F9001C99F300D09
:100C1000D89F300D1124209300011123D9F068ECE6
:100C200070E08C2F0E94262BDF93CF9385ED90E010
:100C30009F938F9389E890E19F938F93E091DA03DC
:100C4000F091DB0309958DB79EB706968DBF02C064
:100C500080930001112311F1809100016AE00E944C
:100C6000BE79892F99279F938F93809100010E94CD
:100C7000BE7999279F938F9380EE90E09F938F93F7
:100C800089E890E19F938F93E091DA03F091DB0381
:100C900009952DB73EB7285F3F4F2DBFDF91CF910C
:100CA0001F910895CFEFD0E1DEBFCDBF88249924F6
:100CB00014B815B807EE13E00253104017FFFCCF2D
:100CC000189B06C0199B02C08DE007C08BE005C0D1
:100CD000199B02C084E101C08AE08093020181E88F
:100CE00087B93E9A8FEF88B98BE184B981E085B9E5
:100CF0008EE38AB987E48BB9469A84B7877F84BF2D
:100D0000809160008861809360001092600084ECA4
:100D100099E09093D4018093D3011092C502109270
:100D2000C4021092E6061092E5061092C7021092D5
:100D3000C6021092C9021092C80220910201243109
:100D400028F084EC94E0A0E0B0E004C08BE095E0F3
:100D5000A0E0B0E08093440190934501A093460148
:100D6000B09347012A3011F0243110F0289801C0C7
:100D7000289A0E9476140E9447140E9491100E94A3
:100D80004E270E945B180E94C5220E9488560E942E
:100D9000BB6F0E94C777809102018C3010F4299AB2
:100DA00001C0299878940E94E42180911A028260FF
:100DB00080931A0210921C020E948E3684EF91E0FA
:100DC0000E940D148C0180911A0280FD05C0C8019B
:100DD0000E9416148823B9F38AEF90E09F938F93B3
:100DE000B9E8AB2EB0E1BB2EBF92AF92E091DA032F
:100DF000F091DB03099580EA9FE00E940D148C01BD
:100E0000C0E0D0E00F900F900F900F90A3E8EA2E73
:100E1000A6E0FA2EF7E3CF2EF6E0DF2E0E948E3604
:100E200080911A0280FD05C0C8010E941614882313
:100E3000B9F3F60180811816ACF40BC00E948E360F
:100E400080911A0280FD05C0C8010E9416148823F3
:100E5000B9F3C8010E941614882321F4F701808198
:100E6000882364F7F701808187FF18C02196DF93FC
:100E7000CF9321978CE091E09F938F93BF92AF9295
:100E8000E091DA03F091DB0309958091A4018F5F73
:100E90008093A4018DB79EB706968DBF2196E4E09E
:100EA000F0E0CE0EDF1E88E090E0E80EF91ECC30B8
:100EB000D10508F4B3CFC0E0D0E000E816E0E7E3E6
:100EC000EE2EE6E0FE2EF801838187FD1CC0F701BF
:100ED00080811816C4F42196DF93CF9321978FE079
:100EE00091E09F938F9389E890E19F938F93E09196
:100EF000DA03F091DB03099582E08093D1018DB78D
:100F00009EB706968DBFF8018381807883832196F2
:100F100084E090E0E80EF91E085F1F4FCC30D10549
:100F200090F28DE291E09F938F93C9E8D0E1DF9337
:100F3000CF93E091DA03F091DB0309959091B80526
:100F40008091A4010F900F900F900F90981728F4A4
:100F50008091F70380618093F70381E391E09F9391
:100F60008F93DF93CF93E091DA03F091DB03099540
:100F700088EE93E00E940D148C010E9461180F907E
:100F80000F900F900F90C8010E9416148823D9F378
:100F900081E591E09F938F93DF93CF93E091DA0304
:100FA000F091DB03099580E00E94E82B809102011B
:100FB0000F900F900F900F908A3011F0843110F045
:100FC000289801C0289A80ED97E09093D4018093EF
:100FD000D30185E5809313048EE090E00E94B32056
:100FE0009927182F00278FE090E00E94B320080F68
:100FF000111D1093AA010093A9018AE090E00E94BC
:10100000B3209927182F00278BE090E00E94B3208F
:10101000080F111D1093A8010093A7010F5F1F4F28
:1010200039F08091A9019091AA018F5F9F4F41F4FF
:101030001092AA011092A9011092A8011092A70182
:101040008091A7019091A8019F938F938091A9010E
:101050009091AA019F938F9386E591E09F938F9340
:10106000DF93CF93E091DA03F091DB0309958DB71D
:101070009EB708968DBF85E791E09F938F93DF938E
:10108000CF93E091DA03F091DB0309958091C605D7
:101090000F900F900F900F90E091DA03F091DB0327
:1010A00082FF07C081E891E09F938F93DF93CF93F6
:1010B00008C08DE891E09F938F9389E890E19F931A
:1010C0008F9309950F900F900F900F9088E893E100
:1010D000909341018093400181E0809312040E942B
:1010E000C8058091E0050E942D778FE991E09F93DC
:1010F0008F93DF93CF93E091DA03F091DB030995AF
:1011000080ED97E00E940D148C018AEF90E00E9420
:101110000D14EC0183E0809362050F900F900F9007
:101120000F90CE010E941614882339F084E690E0D7
:101130000E940D14EC010E9483788091D7018823CE
:1011400009F4DFC180910F01882309F4DAC11092FC
:10115000D70180911104882319F00E94930502C0E1
:101160000E9422390E948E36209102012A3011F00D
:10117000243110F0289801C0289A8091CA029091D9
:10118000F703882339F08091CA0281508093CA0204
:10119000977F0AC080916F00806280936F001092E9
:1011A000E2061092E10698609093F7038091400167
:1011B000909141010197909341018093400180916A
:1011C000400190914101892B29F080911B028823D5
:1011D00009F43EC08091400190914101892B01F5B5
:1011E0000E94EB2285E090E09093410180934001C2
:1011F00080919C0590919D05019690939D0580930B
:101200009C05809196028068809396028091F703F6
:1012100081608093F703809163058260809363050A
:1012200080910801909109018F5F9F4F19F580917E
:10123000C1028823F9F080E197E29093D401809372
:10124000D30180E890E0909309018093080112C0D7
:101250002A3011F0243110F0289801C0289A80918A
:10126000D3019091D401892B29F4809196028F7734
:10127000809396028091D701882309F042C10E9491
:10128000D5100E94F50CC8010E941614882309F499
:1012900034C10C5E1F4F80911B029091F70388238D
:1012A00039F092609093F7038091630582600CC0DF
:1012B0009D7F9093F70380914001909141010797A2
:1012C00028F0809163058D7F8093630580914001B4
:1012D00090914101079728F08091F7038E7F8093CA
:1012E000F70380910501882321F081508093050147
:1012F00025C080931D041092A2021092A1021092A8
:10130000A00210929F0210929E0210929D02809164
:101310000801909109018F5F9F4F81F48091CA026B
:10132000882361F488E99AE39093D4018093D301F0
:1013300080E09CE0909309018093080180919B01DB
:10134000893C70F0815080939B01809196028F7B45
:10135000809396028091F7038B7F8093F70335C0CB
:101360008091CD07882309F1809196028064809353
:1013700096028091F70384608093F70380910801BF
:10138000909109018F5F9F4F81F48091C102882362
:1013900061F088E99AE39093D4018093D30180E0CF
:1013A00098EA90930901809308011092AB03109280
:1013B000AA031092A9031092A8038FEF9FEF9093B6
:1013C000FB078093FA0710929B0180910001282F60
:1013D000332780911D0190911E0182179307CCF451
:1013E000809196028062809396028091080190918C
:1013F00009018F5F9F4FC1F480E797E19093D4017B
:101400008093D30180E093E09093090180930801D9
:101410000BC08091D3019091D401892B29F4809144
:1014200096028F7D809396020E94865A84E0809374
:10143000D2018091C102882329F45AEA852E55E011
:10144000952E12C08091AB018F5F8093AB018133E9
:1014500059F41092AB018091A5019091A6010196DB
:101460009093A6018093A5010894811C911CF2E73A
:101470008F16FBE09F0609F040C088249924209134
:10148000A9013091AA012F5F3F4F3093AA01209309
:10149000A9018091A7019091A80101969093A801BC
:1014A0008093A701832F9927682F8EE090E00E94F8
:1014B000B9208091A9019091AA019070682F8FE0C6
:1014C00090E00E94B9208091A7019091A801892FF6
:1014D0009927682F8AE090E00E94B9208091A701A7
:1014E0009091A8019070682F8BE090E00E94B92045
:1014F00084E190E00E940D148C010E94D65A0E9453
:10150000D26F8091D201882309F00BCE0E94A95698
:1015100008CE1F920F920FB60F9211248F939F93B4
:10152000EF93FF93809107018823E1F48091C50137
:101530009091C60101969093C6018093C501FC016C
:10154000EE53FB4FE081ED3019F0803A910539F40C
:101550001092C6011092C50181E080930701E093CB
:10156000C60004C01092C6011092C501FF91EF9110
:101570009F918F910F900FBE0F901F9018951F9203
:101580000F920FB60F9211242F933F934F935F93B7
:101590008F939F93AF93BF93EF93FF9390E08091CE
:1015A000C6008093BD015091CB01503A10F090934A
:1015B000CC018091BD018D3009F063C08091CC01D8
:1015C000823009F05EC09093CC01852F9927805E10
:1015D0009B4FFC01329740812091C7013091C80197
:1015E000241B3109DC0111978C91281B3109C90199
:1015F0009F709093C8018093C70146E096958795A8
:101600004A95E1F7982F935C9093C9012F7330703E
:10161000235C2093CA018081981729F48C912817A4
:1016200011F491E006C090E08091BA018F5F809341
:10163000BA013091BC01332309F072C0992309F437
:101640006FC081E08093BC01580F5093B901515095
:10165000E52FFF27E05EFB4F8DE080838091220421
:10166000823509F05DC088E190E02CE00FB6F89477
:10167000A895809360000FBE209360003093D10145
:101680004FC02091CC01822F992781309105F9F02C
:10169000823091051CF4892B21F040C0029711F192
:1016A0003DC08091BD01833239F48091BC01882313
:1016B00019F481E08093CC018091BD0180932004D6
:1016C00081E08093CB018091BD01992722C02F5FDB
:1016D0002093CC01E52FFF27E05EFB4F8091BD01F9
:1016E000808309C0E52FFF27E05EFB4F8091BD019D
:1016F0008083503A20F45F5F5093CB0102C0109278
:10170000CC012091BD018091C7019091C801820F49
:10171000911D9093C8018093C70102C01092CC0123
:10172000FF91EF91BF91AF919F918F915F914F91F9
:101730003F912F910F900FBE0F901F901895AC0105
:10174000A0E0B0E09D01A817B90748F4E2ECF4E08E
:101750008191280F311D1196A417B507C8F33F706A
:10176000FD01EE53FB4FC90156E0969587955A95BA
:10177000E1F7835C80831196FD01EE53FB4F2F73DD
:101780003070822F835C8083AD53BB4F8DE08C9390
:10179000109207018091C2048093C6000895A0E0D2
:1017A000B0E0E5EDFBE00C94377A2C859D850E8545
:1017B000BB2483E28093C2049F599093C304209377
:1017C000C40433E0E32EF12C002309F49EC0CF843F
:1017D000D888BE016D5E7F4FA989BA8901501097E4
:1017E00009F493C01097B9F0F601EB0DF11DB39415
:1017F0009081119791F4002349F1FB016E5F7F4FB7
:10180000DB01C080D1806E5F7F4F0D90BC91A02D19
:10181000BB24015002C090E019C01097B9F0F60146
:10182000EB0DF11DB3944081119791F4002341F128
:10183000FB016E5F7F4FDB01C080D1806E5F7F4F09
:101840000D90BC91A02DBB24015002C040E018C0F7
:101850001097B1F0F601EB0DF11DB39410811197C3
:1018600081F4002371F0FB013296DB01CD90DC9016
:10187000BF016E5F7F4FA081B181BB24015001C0C9
:1018800010E0F701EE53FB4F892F86958695835C18
:1018900080830894E11CF11CF701EE53FB4F892F64
:1018A00099278370907024E0880F991F2A95E1F79B
:1018B00055279A0194E0369527959A95E1F7822B62
:1018C000835C80830894E11CF11CF701EE53FB4F0D
:1018D0004F705070440F551F440F551F812F99278B
:1018E00026E0969587952A95E1F7842B835C808383
:1018F0000894E11CF11CF701EE53FB4F1F73135CBE
:1019000010830894E11CF11C6ACFC7010E949F0B51
:10191000E9E00C94537AA3E07A2F4091B901465044
:10192000442309F458C0E72FFF27E05EFB4F808176
:101930008D537F5FE72FFF27E05EFB4F20812D5304
:101940007F5FE72FFF27E05EFB4F30813D537F5FD6
:10195000E72FFF27E05EFB4F60816D537F5F992784
:10196000880F991F880F991F522F52955F70582B1F
:10197000822F99278F709070F4E0880F991FFA9545
:10198000E1F7232F26952695282B832F99278370FF
:101990009070E6E0880F991FEA95E1F7682B4150B7
:1019A0004F3FC9F0EA2FFF27E05EFB4F5083AF5F48
:1019B00041504F3F81F0EA2FFF27E05EFB4F20832D
:1019C000AF5F41504F3F39F0EA2FFF27E05EFB4FFA
:1019D0006083AF5FA5CF83E294E09093B8018093DA
:1019E000B701A350A093B6010895A2E0B0E0EBEFD9
:1019F000FCE00C943D7A8091BC01882309F485C3F6
:101A00000E948B0C80912104823609F081C2809162
:101A1000220499278137910509F4C0C082379105C6
:101A2000C4F48D36910509F482C08E36910544F4D4
:101A30008B34910531F18636910509F454C168C2A1
:101A40008E36910509F45BC08037910509F49FC07B
:101A50005FC28537910509F4E2C18637910544F4E8
:101A60008337910509F4DCC08437910539F150C200
:101A70008737910509F410C28937910509F46AC1C5
:101A800047C2E091B701F091B801808191819093B4
:101A9000DD028093DC022091DA023091DB02821BAE
:101AA000930B845E9D4F68E671E00E94DE79845B53
:101AB00090409093D9028093D8022AC28091B901B4
:101AC000A091B701B091B801853140F080E1EBEF12
:101AD000F3E00D9001928A95E1F70DC08D919D91F3
:101AE0000D90BC91A02D8093FB039093FC03A093D9
:101AF000FD03B093FE0380EF8093B4014BC080914F
:101B000007018823E1F38DE490E09F938F938AE2AD
:101B100096E09F938F9381E08F938F938EE48F93C2
:101B20000E94CF0B8DB79EB707968DBFF1C1A091D4
:101B3000B701B091B8011C91113081F48DE4EAE253
:101B4000F6E00D9001928A95E1F70E9470211983C9
:101B50008091F7038F7E8093F70301C019828091F3
:101B600007018823E1F381E090E09F938F93CE01FA
:101B700001969F938F9381E08F938F938DE48F9342
:101B80000E94CF0BADB7BEB71796ADBFC1C181E004
:101B90008093BF018FEF80930501BAC1E091B70137
:101BA000F091B80180818F3F39F40E94D521E091F6
:101BB000B701F091B8018083E091B701F091B801CD
:101BC0008081882311F481E003C0863010F085E025
:101BD0008083E091B701F091B80180810E94C82014
:101BE000E091B701F091B80180818983809107016C
:101BF0008823E1F380E790E09F938F9389EB95E052
:101C00009F938F9381E090E09F938F93CE010196F5
:101C10009F938F9382E08F9381E08F9381E571C1D1
:101C20002091B7013091B801D9018C918150853054
:101C300008F040C0F90181818435E1F52F5F3F4F05
:101C400080E7E9EBF5E0D9010D9001928A95E1F783
:101C5000F90182910E940C218091F8059927AA2709
:101C6000BB27BC01CD0124EC39E040E050E00E94EC
:101C70009F79DC01CB018093640190936501A0936F
:101C80006601B09367018091F9059927AA27BB27C0
:101C9000BC01CD010E949F79DC01CB0180936001E2
:101CA00090936101A0936201B09363010E94D521DA
:101CB000898301C01982809107018823E1F381E0C3
:101CC00090E09F938F93CE0101969F938F9381E035
:101CD0008F938F9383E58F930E94CF0B8DB79EB721
:101CE00007968DBF26C0E091B701F091B801E08161
:101CF0008E2F8150853018F48E2F0E94C8200E94AC
:101D0000D5218983809107018823E1F381E090E068
:101D10009F938F93CE0101969F938F9381E08F9332
:101D20008F9386E48F930E94CF0BADB7BEB7179603
:101D3000ADBF8091C102882329F46EE670E08981ED
:101D40000E94262B80E00E94C8058091E0050E9439
:101D50002D77DEC0E091B701F091B801808199271D
:101D600087FD90959093FC068093FB0681819927CF
:101D700087FD90959093FE068093FD0682819927BA
:101D800087FD9095909300078093FF0683819927A4
:101D900087FD90959093020780930107848199278E
:101DA00087FD909590930407809303078581992779
:101DB00087FD909590930607809305078681992764
:101DC00087FD90959093080780930707878199274F
:101DD00087FD909590930A0780930907808599273E
:101DE00087FD909590930C0780930B078185992729
:101DF00087FD909590930E0780930D078285992714
:101E000087FD90959093100780930F0783859927FE
:101E100087FD9095909312078093110779C0E09108
:101E2000B701F091B80180810E94A7268A83882398
:101E300019F481E0898301C0198280910701882308
:101E4000E1F388E090E09F938F9388E796E09F937B
:101E50008F9321E030E03F932F938091B7019091D1
:101E6000B8019F938F933F932F93CE0102969F9338
:101E70008F933F932F93CE01820F931F9F938F9346
:101E800084E08F9381E08F9385E58F930E94CF0B41
:101E9000EDB7FEB773963BC08091B6018930C0F1B3
:101EA0002091B7013091B8012F5F3F4F88E0A8E73C
:101EB000B6E0F90101900D928A95E1F7D9018E9172
:101EC0000E94FD258A83882319F481E0898301C05B
:101ED0001982809107018823E1F321E030E03F93EC
:101EE0002F93CE0102969F938F933F932F93CE0112
:101EF000820F931F9F938F9382E08F9381E08F9344
:101F000087E58F930E94CF0BEDB7FEB73B96EDBFF1
:101F10008091220499278436910509F4C9C0853639
:101F20009105ACF48136910509F47DC082369105A6
:101F30002CF48B34910509F459C0DFC08236910529
:101F400009F47EC08336910509F48DC0D6C0883669
:101F5000910509F4CBC0893691052CF4873691059B
:101F600009F4C8C0CAC08437910529F086379105A5
:101F700009F4BCC0C2C08091B901A091B701B09171
:101F8000B801803140F080E1EBEFF3E00D90019279
:101F90008A95E1F70DC08D919D910D90BC91A02D7A
:101FA0008093FB039093FC03A093FD03B093FE0387
:101FB000809107018823E1F31F92809104018F93A0
:101FC00084E58F930E94CF0B8AEF8093B4018FEF4B
:101FD0008093050180EA9FE00E940D149093AD016B
:101FE0008093AC010F900F900F9087C0E091B701E4
:101FF000F091B801808191819093DD028093DC02A1
:102000002091DA023091DB02821B930B845E9D4F9C
:1020100068E671E00E94DE79845B90409093D9027B
:102020008093D8026AC0E091B701F091B801808135
:1020300080930601803298F08FE1809306010FC0F3
:10204000A091B701B091B8018BE0E3E1F4E00D900D
:1020500001928A95E1F780911C048093A4058FEF8B
:10206000809305014AC08091B0019091B101892B04
:1020700089F4E091B701F091B801E081EE2351F0CD
:102080008AE0E89FC00111240E940D149093EE0392
:102090008093ED03E091B701F091B80190818AE05F
:1020A000989FC00111249093B1018093B00115C095
:1020B0008FEF80930501E091B701F091B801908115
:1020C0008AE0989FC00111249093B3018093B201DC
:1020D000892B19F081E08093C10180EA9FE00E9482
:1020E0000D149093AD018093AC0107C081E0809303
:1020F000C00103C081E08093C4011092BC01109222
:10210000B8011092B7011092B601E3E0CE5F0C94D3
:10211000597A982F8091C00085FFFCCF9093C6001C
:1021200008950F931F9388E18093C1008091C000B0
:1021300082608093C0008091C10080688093C1005C
:102140008091C10080648093C10000E010E00093A2
:10215000C5008AE290E08093C4008091B201909122
:10216000B3010E940D149093F0038093EF038CED64
:1021700090E00E940D1490931F0480931E0410920F
:10218000F10380E58093F20386E08093F5038BE012
:102190008093F3031092F4031093B8010093B701F6
:1021A0001092B6011F910F910895A0E1B0E0EBED00
:1021B000F0E10C943A7A80910701882309F41EC259
:1021C0008091AC019091AD010E941614882361F0BA
:1021D0001092AF011092AE011092B3011092B201B1
:1021E0001092B1011092B0018091C0018823D1F00A
:1021F000809107018823B1F08AE090E09F938F934C
:1022000081EF93E09F938F9381E08F938F9386E587
:102210008F930E94CF0B1092C0012DB73EB7295F5C
:102220003F4F2DBF8091C4018823D9F080910701D1
:102230008823B9F08BE090E09F938F9383E194E043
:102240009F938F9381E08F93809104018F9387E414
:102250008F930E94CF0B1092C4018DB79EB7079643
:102260008DBF80911E0490911F040E941614882334
:1022700009F461C080910701882309F45CC0809152
:10228000D5059927880F991F880F991F7C01002772
:10229000F7FC0095102F80911E0390911F03A091D1
:1022A0002003B0912103BC01CD01A80197010E9438
:1022B000137A30930C0420930B04809116039091B1
:1022C0001703A0911803B0911903BC01CD01A80117
:1022D00097010E94137A30930E0420930D0480918D
:1022E000AB0280930F048091AA028093100488E0CF
:1022F00090E09F938F938BE094E09F938F9381E086
:102300008F9383E08F938BE68F930E94CF0B809106
:1023100011042DB73EB7295F3F4F2DBF853018F010
:1023200086E08093110483E690E00E940D14909360
:102330001F0480931E048091B2019091B301892BF8
:1023400041F08091EF039091F0030E9416148823CE
:1023500021F48091C101882339F1809107018823FC
:1023600019F10E94F22982E490E09F938F9382E614
:1023700095E09F938F9381E08F938F9384E48F9365
:102380000E94CF0B1092C1018DB79EB707968DBFEB
:102390008091B2019091B301009731F00E940D1429
:1023A0009093F0038093EF038091B0019091B1017D
:1023B000892B09F4B8C08091ED039091EE030E943F
:1023C0001614882309F4AFC080910701882309F40B
:1023D000AAC08091D5059927880F991F880F991F4A
:1023E0007C010027F7FC0095102F80911E0390912F
:1023F0001F03A0912003B0912103BC01CD01A801CE
:1024000097010E94137A3093E0032093DF038091B9
:10241000160390911703A0911803B0911903BC0102
:10242000CD01A80197010E94137A3093E203209313
:10243000E1032091B4073091B5074091B607509160
:10244000B707DA01C90163E0880F991FAA1FBB1FF4
:102450006A95D1F7820F931FA41FB51F820F931F98
:10246000A41FB51F209144013091450140914601C0
:1024700050914701BC01CD010E94137A3093E403CF
:102480002093E3038091E6029091E702A091E80295
:10249000B091E90229E0B595A795979587952A957A
:1024A000D1F78093E5038091E2029091E302A0913D
:1024B000E402B091E50209E0B595A7959795879557
:1024C0000A95D1F78093E6038091EE029091EF0296
:1024D000A091F002B091F10219E0B595A7959795FA
:1024E00087951A95D1F78093E7038EE090E09F934C
:1024F0008F938FED93E09F938F9381E08F938F93D2
:1025000083E48F930E94CF0B8091B0019091B10131
:102510000E940D149093EE038093ED032DB73EB708
:10252000295F3F4F2DBF909106019F3F61F18DE0E4
:10253000989FC00111248B559E4F40E150E0BC0193
:10254000CE0101960E94CD7880E190E09F938F9319
:10255000CE0101969F938F9381E090E09F938F939C
:1025600086E091E09F938F9382E08F9381E08F9339
:1025700081E48F930E94CF0B8FEF809306018DB77C
:102580009EB70B968DBF8091A4058823D1F08091D2
:1025900007018823B1F081E090E09F938F9384EA54
:1025A00095E09F938F9381E08F938F9382E48F9335
:1025B0000E94CF0B1092A4052DB73EB7295F3F4F65
:1025C0002DBF8091BF018823C9F080910701882326
:1025D000A9F084E390E09F938F9381EE96E09F9320
:1025E0008F9381E08F938F9380E58F930E94CF0B21
:1025F0001092BF018DB79EB707968DBFE6E0C05F12
:102600000C94567A1F920F920FB60F9211242F93AB
:102610003F935F936F937F938F939F93AF93BF93FA
:10262000EF93FF9320E08091D201882329F08091DD
:10263000D20181508093D2018091BC03882319F08C
:1026400081508093BC038091DA0181508093DA013C
:102650008F3F09F05BC089E08093DA018091D80157
:102660009091D90101969093D9018093D8018091DE
:102670000A018F5F817080930A01882319F481E039
:102680008093D701349903C081E08093DB0180916E
:10269000D3019091D401892B21F18091D3019091A4
:1026A000D4010B9750F08091D3019091D4010A97F7
:1026B0009093D4018093D30104C01092D40110925E
:1026C000D3018091D3019091D401209108013091E0
:1026D000090182239323892B11F021E008C020E017
:1026E00006C08FEF9FEF90930901809308018091BE
:1026F0000201222331F08A3011F45A9A07C0479A16
:1027000005C08A3011F45A9801C047988091DB01C6
:10271000882309F472C020919B01222309F06DC027
:102720008091C60583FF69C086B19927FC01E071DD
:10273000F07084FF14C08091D5019091D60101966C
:102740009093D6018093D5018091D5019091D601C7
:10275000895E934008F451C02093DB014EC0809104
:10276000D5019091D601892B09F443C08091D50100
:102770009091D6018A569140E0F58091D5019091D3
:10278000D60169E270E00E94CA798091D5019091EA
:10279000D601860F971F9093D6018093D501809123
:1027A000D5019091D6010B9750F08091D501909171
:1027B000D6010A979093DD028093DC0204C0F09367
:1027C000DD02E093DC028091DC029091DD02209139
:1027D000DA023091DB02821B930B845E9D4F68E628
:1027E00071E00E94DE79845B90409093D9028093DF
:1027F000D8021092D6011092D501FF91EF91BF91AE
:10280000AF919F918F917F916F915F913F912F91A8
:102810000F900FBE0F901F9018952091D801309106
:10282000D901280F391FC901019608952091D801B7
:102830003091D901821B930B892F9927869580743B
:1028400090700895CF93DF930E940D14EC01CE0198
:102850000E9416148823D9F3DF91CF910895CF9366
:10286000DF930E940D14EC0109C080910F018823B1
:1028700029F090930F018FEC80937A00CE010E9493
:102880001614982F882389F3DF91CF9108959FB76D
:10289000F8945F983E9A469A8091B0008F7080932A
:1028A000B0008091B00083608093B0008091B1004F
:1028B0008B738093B1008091B1008B608093B100E5
:1028C0001092B2008FEF8093B3008091B0008068C7
:1028D0008093B000809170008A7F80937000809117
:1028E00070008260809370009FBF08958AE090E03E
:1028F0000E940D149093E3018093E20182E085BD74
:1029000083EA84BD17BC84EB88BD86E086BD8091D8
:102910006E00816080936E0008951F920F920FB633
:102920000F9211242F933F934F935F936F937F9355
:102930008F939F93AF93BF93CF93DF93EF93FF93C7
:10294000809102019091DC01843108F011C199233A
:1029500009F06AC38091B00086FFECC08091B0009E
:102960008F7B8093B00089EA93E09093DE0180939F
:10297000DD0180910B0190910C019C01220F331F0E
:10298000280F391F809150019927880F991F880FB0
:10299000991F280F391F37FF02C02D5F3F4FC90114
:1029A000959587959595879590930C0180930B014C
:1029B0009093D0018093CF0180911B066091E70531
:1029C00020911E0330911F03409120035091210359
:1029D00080FF2CC0772788279927EA01D90157FF64
:1029E00004C0A158BF4FCF4FDF4FE7E0D595C79543
:1029F000B795A795EA95D1F79D01AE010E949F7901
:102A00009B01AC0197FF04C0215C3F4F4F4F5F4FCC
:102A100066E055954795379527956A95D1F780914A
:102A2000CF019091D001820F931F2BC07727882769
:102A30009927EA01D90157FF04C0A158BF4FCF4FD2
:102A4000DF4F27E0D595C795B795A7952A95D1F77C
:102A50009D01AE010E949F799B01AC0197FF04C0CC
:102A6000215C3F4F4F4F5F4FF6E0559547953795A7
:102A70002795FA95D1F78091CF019091D001821BD3
:102A8000930B9093D0018093CF018091E805282F7C
:102A90003327220F331F220F331F8091CF019091D4
:102AA000D001821793077CF08091E905282F332706
:102AB000220F331F220F331F8091CF019091D0013D
:102AC0002817390724F43093D0012093CF012091A7
:102AD000DD013091DE018091CF019091D001280F6E
:102AE000391F205032403093DE012093DD01809168
:102AF000CF019091D00197FD039695958795959577
:102B000087959093D0018093CF0145E02D3D340708
:102B100018F08CED95E005C02757314030F487E779
:102B200091E09093DE018093DD018091DD01909131
:102B3000DE0143C28091B00080648093B000809138
:102B4000EE05282F33278DED96E0289FA001299FC1
:102B5000500D389F500D1124CA012091DF01309192
:102B6000E001821B930B9093DE018093DD0159C23B
:102B7000992309F059C28091B00086FF23C2809149
:102B8000B0008F7B8093B000E091E101EE23F1F47F
:102B90008091EE05282F33278DED96E0289FA00128
:102BA000299F500D389F500D1124CA012091DF013B
:102BB0003091E001821B930B9093DE018093DD0145
:102BC0001092E0011092DF01469A2BC289EA93E04D
:102BD0009093DE018093DD018E2F9927833091053C
:102BE00009F4A4C1843091053CF48130910561F071
:102BF000029709F4D2C0AAC18430910509F499C1A1
:102C0000059709F4A0C1A2C180910B0190910C011C
:102C10009C01220F331F280F391F809150019927E3
:102C2000880F991F880F991F280F391F37FF02C07F
:102C30002D5F3F4FC9019595879595958795909301
:102C40000C0180930B019093D0018093CF01809170
:102C50001B066091E70520911E0330911F034091F0
:102C600020035091210380FF2CC0772788279927C4
:102C7000EA01D90157FF04C0A158BF4FCF4FDF4F22
:102C800027E0D595C795B795A7952A95D1F79D01CA
:102C9000AE010E949F799B01AC0197FF04C0215CAB
:102CA0003F4F4F4F5F4FA6E0559547953795279576
:102CB000AA95D1F78091CF019091D001820F931FF7
:102CC00027C077278827992757FF04C021583F4FEF
:102CD0004F4F5F4FF7E05595479537952795FA95F4
:102CE000D1F70E949F799B01AC0197FF04C0215C42
:102CF0003F4F4F4F5F4FE6E05595479537952795E6
:102D0000EA95D1F78091CF019091D001821B930B6E
:102D10009093D0018093CF018091E805282F33272D
:102D2000220F331F220F331F8091CF019091D001CA
:102D3000821793077CF08091E905282F3327220F13
:102D4000331F220F331F8091CF019091D00128179C
:102D5000390724F43093D0012093CF018091DD0115
:102D60009091DE012091CF013091D001820F931F0D
:102D7000805092409093DE018093DD018091CF01DD
:102D80009091D00197FD0396959587959595879598
:102D90009093D0018093CF01ECC080910D01909170
:102DA0000E019C01220F331F280F391F80914F0104
:102DB0009927880F991F880F991F280F391F37FFF0
:102DC00002C02D5F3F4FC9019595879595958795D1
:102DD00090930E0180930D019093CE018093CD01CD
:102DE00080911B066091EB05A0911603B09117032B
:102DF000C0911803D091190381FF2AC07727882733
:102E000099279D01AE01D7FF04C021583F4F4F4F76
:102E10005F4FA7E05595479537952795AA95D1F728
:102E20000E949F799B01AC0197FF04C0215C3F4F3A
:102E30004F4F5F4FF6E05595479537952795FA9593
:102E4000D1F78091CD019091CE01820F931F29C0BF
:102E50007727882799279D01AE01D7FF04C0215805
:102E60003F4F4F4F5F4FE7E0559547953795279573
:102E7000EA95D1F70E949F799B01AC0197FF04C0AE
:102E8000215C3F4F4F4F5F4F76E055954795379503
:102E900027957A95D1F78091CD019091CE01821B33
:102EA000930B9093CE018093CD018091EC05282F58
:102EB0003327220F331F220F331F8091CD019091B2
:102EC000CE01821793077CF08091ED05282F3327E0
:102ED000220F331F220F331F8091CD019091CE011D
:102EE0002817390724F43093CE012093CD01809127
:102EF000DD019091DE012091CD013091CE01820F54
:102F0000931F805092409093DE018093DD01809169
:102F1000CD019091CE0197FD039695958795959556
:102F200087959093CE018093CD0123C0809178073F
:102F300002C080914F079927880F991F880F991F0A
:102F400087559E4F12C080918307F5CFFF27EE0F64
:102F5000FF1FEF51F94F20813181220F331F8091E4
:102F6000DD019091DE01820F931F9093DE0180932B
:102F7000DD018091DD019091DE0155E08D3D9507E9
:102F800018F08CED95E005C08757914030F487E745
:102F900091E09093DE018093DD012091DD0130917D
:102FA000DE012C5B30403093DE012093DD01809107
:102FB000DF019091E001820F931F9093E0018093D5
:102FC000DF012FC08091B00080648093B0008CEB53
:102FD00090E09093DE018093DD018091DF0190917C
:102FE000E00184549F4F9093E0018093DF01809132
:102FF000D101882321F08091CA02853B20F4809181
:10300000D101823011F4469801C0469A8091E101C5
:103010008F5F8093E1019091EE05981710F4109264
:10302000E10181E08093DC012091DD013091DE013E
:1030300041E02F37340730F08FEF8093B3002F5FDC
:1030400030400FC02F3F3105C9F0C0F0A9014F5FDC
:1030500050404F37510550F480E88093B30020581A
:1030600030403093DE012093DD0112C08FEF80935A
:10307000B3005093DE014093DD010AC08091DD0171
:103080008093B3001092DE011092DD011092DC01FA
:10309000FF91EF91DF91CF91BF91AF919F918F9170
:1030A0007F916F915F914F913F912F910F900FBE44
:1030B0000F901F90189510927C008FEC80937A00EF
:1030C0000895CF93DF931092E80183E090E00E948F
:1030D000B320C82FDD27C531D10508F02A97C7BD19
:1030E00084E690E00E942F148091130190911401C6
:1030F0008052934010F4C0E0D0E0CA3FD105F8F40C
:10310000C7BD82E390E00E942F1485E493E09F9373
:103110008F9389E890E19F938F93E091DA03F09188
:10312000DB03099580911301909114010F900F908A
:103130000F900F908052934010F02196DECFC093F5
:10314000B5056C2F83E090E00E94B9208091C60500
:1031500080FF0AC08091B5058A508B3E28F080918F
:10316000F60380648093F603C7BD8CE291E00E9471
:103170002F14DF91CF910895EF92FF921F93CF9379
:1031800010E080ED97E00E940D147C01CCE8133034
:1031900019F4CB3008F0C9E010E08091F80190916B
:1031A000F9018C5F934024F48091120181500AC090
:1031B0008091F8019091F9018750944034F080910A
:1031C00012018F5F8093120101C011E08091F6011E
:1031D0009091F7018C5F934024F48091110181500C
:1031E0000AC08091F6019091F7018750944034F025
:1031F000809111018F5F8093110101C01F5F809149
:10320000F4019091F5018C5F934024F480911001BA
:1032100081500AC08091F4019091F501875094404B
:10322000C4F0809110018F5F8093100113C087E478
:1032300093E09F938F9389E890E19F938F93E09120
:10324000DA03F091DB0309950F900F900F900F9028
:103250005FC01F5F82E180931F0280911A028E7F00
:1032600080931A0285EA8093BC00809112018A3013
:1032700040F48091F60381608093F6038AE08093A6
:10328000120180911201863F40F08091F603816027
:103290008093F60385EF80931201809111018A30AB
:1032A00040F48091F60382608093F6038AE0809375
:1032B000110180911101863F40F08091F6038260F8
:1032C0008093F60385EF80931101809110018A307D
:1032D00040F48091F60384608093F6038AE0809343
:1032E000100180911001863F40F08091F6038460C8
:1032F0008093F60385EF8093100180911F0288234D
:1033000039F0C7010E941614882309F090CFF5CF39
:1033100010920F018FEC80937A0080910F01882327
:10332000E1F3CA3020F48AE090E00E942F14C150EB
:1033300009F02DCF86E490E00E942F14CF911F91C9
:10334000FF90EF9008951F920F920FB60F921124E5
:10335000AF92BF92CF92DF92EF92FF920F931F93A3
:103360002F933F934F935F936F937F938F939F938D
:10337000AF93BF93EF93FF9380910102282F3327E0
:10338000442755278F5F80930102F90122313105CF
:1033900008F08CC3E25CFF4F0C94657A8091780052
:1033A0009091790046C080917800909179002CC16D
:1033B00080917800909179009093040280930302A9
:1033C00057C1809127039091280320917800309174
:1033D0007900821B930B9093A6058093A50580919D
:1033E000A5059091A60590930E0280930D025EC1F3
:1033F00080917800909179002091290330912A03DF
:10340000821B930B9093B4058093B3058091B30511
:103410009091B4059093100280930F0249C380915C
:103420000702909108022091780030917900820F74
:10343000931F909308028093070281E03AC3809122
:103440000502909106022091780030917900820F58
:10345000931F909306028093050284E02AC3809113
:103460001D0190911E019C01220F331F280F391F4F
:10347000809178009091790063E070E00E94CA79B1
:10348000260F371F369527953695279530931E01C1
:1034900020931D0185E00DC3809178009091790003
:1034A0004091230350912403841B950B9093EF01CB
:1034B0008093EE018091EE019091EF01029704F16B
:1034C00022E04E3E520784F4209102022B5F2093AB
:1034D000020225508091970290919802845F91405A
:1034E00018F4215F2093020280910202853684F154
:1034F0004F5F5F4F5093240340932303845626C0AD
:103500008091EE019091EF018F5F9F4F0CF532E0BB
:1035100047325307ECF0209102022550209302021B
:103520002B5F8091970290919802845F914018F4EC
:103530002F5020930202809102028C394CF44150AA
:10354000504050932403409323038C5980930202EC
:1035500081E08093ED0180917800909179009093C3
:10356000AC058093AB058091EE019091EF019C0139
:10357000442737FD4095542F8091DE029091DF0261
:10358000A091E002B091E102820F931FA41FB51F2A
:103590008093DE029093DF02A093E002B093E102F9
:1035A0002091DE023091DF024091E0025091E10271
:1035B00057FF04C021503C4F4F4F5F4F0AE05595D5
:1035C0004795379527950A95D1F78091DE0290911E
:1035D000DF02A091E002B091E102821B930BA40BE9
:1035E000B50B8093DE029093DF02A093E002B093CC
:1035F000E1022EC18091050290910602209178008F
:1036000030917900820F931F9093060280930502F8
:103610001092000250C2809102018A3071F48091B0
:103620007800909179002091030230910402820F7A
:10363000931F01969695879517C04091030250916C
:103640000402843158F02091780030917900240FE1
:10365000351F8FEF97E0821B930B06C08091780097
:1036600090917900840F951F9093F5018093F40158
:1036700086E01FC280912703909128032091780053
:1036800030917900821B930B9093A6058093A5053A
:103690008091A5059091A60520910D0230910E0212
:1036A000820F931F9093F3018093F20187E001C290
:1036B00080917800909179002091290330912A031C
:1036C000821B930B9093B4058093B3058091B3054F
:1036D0009091B40520910F0230911002820F931F38
:1036E0009093F1018093F001E3C1209107023091A2
:1036F00008028091780090917900280F391F30934B
:10370000080220930702809102018A3019F4220FE7
:10371000331F04C0220F331F220F331F30930802C0
:10372000209307022091070230910802C90137FD5A
:103730000796A3E095958795AA95E1F79093F901EF
:103740008093F8018091090290910A02820F931FE1
:1037500097FD01969595879590930A0280930902AB
:103760002091330330913403821B930B90931C01FF
:1037700080931B012091FE013091FF0180911B017C
:1037800090911C01280F391F37FF02C02F5F3F4F58
:10379000359527953093FF012093FE014ECE209161
:1037A0000502309106028091780090917900280FEF
:1037B000391F3093060220930502809102018A305E
:1037C00019F4220F331F04C0220F331F220F331F9F
:1037D00030930602209305022091050230910602E3
:1037E000C90137FD079663E0959587956A95E1F7DE
:1037F0009093F7018093F60180910B0290910C0257
:10380000820F931F97FD01969595879590930C02D3
:1038100080930B022091310330913203821B930B72
:1038200090931A01809319012091FC013091FD01C0
:103830008091190190911A01280F391F37FF02C09A
:103840002F5F3F4F359527953093FD012093FC0165
:1038500083E02FC11092010281E080930F018091DB
:10386000E4019091E50101969093E5018093E401D4
:1038700080917800909179009093140180931301C6
:103880008091130190911401AA27BB27A0901102E7
:10389000B0901202C0901302D0901402A80EB91E6C
:1038A000CA1EDB1EA0921102B0921202C092130235
:1038B000D0921402809115028F5F8093150282319D
:1038C00008F4F6C08091150190911601A09117019E
:1038D000B09118017C018D0123E0EE0CFF1C001F4C
:1038E000111F2A95D1F7E81AF90A0A0B1B0BEA0CEB
:1038F000FB1C0C1D1D1D8091E801992787FD9095EB
:10390000A92FB92FBC01CD0126EC34E240E050E0F4
:103910000E949F79DC01CB01E81AF90A0A0B1B0B04
:10392000D801C7010496A11DB11DB7FF05C0D8017C
:10393000C7010B96A11DB11D13E0B595A7959795ED
:1039400087951A95D1F78093150190931601A0934E
:103950001701B09318018091AD059091AE057C01DF
:103960000027F7FC0095102F80911501909116010A
:10397000A0911701B0911801E81AF90A0A0B1B0B64
:10398000E092BC02F092BD020093BE021093BF020F
:103990002091E9013091EA014091EB015091EC0155
:1039A00057FF04C0215F3F4F4F4F5F4FF4E05595E5
:1039B000479537952795FA95D1F78091E901909130
:1039C000EA01A091EB01B091EC01821B930BA40BD7
:1039D000B50B8093E9019093EA01A093EB01B093BA
:1039E000EC018091E9019091EA01A091EB01B09185
:1039F000EC018E0D9F1DA01FB11F8093E9019093D4
:103A0000EA01A093EB01B093EC018091E601909163
:103A1000E701AC01E5E0440F551FEA95E1F7481BCB
:103A2000590B8091E9019091EA01A091EB01B091CD
:103A3000EC01B7FF03C00F96A11DB11D74E0B59551
:103A4000A795979587957A95D1F72091BC023091EB
:103A5000BD02281B390B63E0220F331F6A95E1F783
:103A6000240F351F37FF02C0215E3F4F45E03595DB
:103A700027954A95E1F73093E7012093E601D601B7
:103A8000C501D7FE03C00196A11DB11DB595A7952F
:103A9000979587958093110290931202A093130239
:103AA000B093140289E08093150202C010920102C3
:103AB00082E0809300028091000280937C008091DC
:103AC0000102882319F08FEC80937A00FF91EF9127
:103AD000BF91AF919F918F917F916F915F914F9126
:103AE0003F912F911F910F91FF90EF90DF90CF901A
:103AF000BF90AF900F900FBE0F901F9018954AEA9D
:103B000020E030E02617370740F4FC018191480F90
:103B10002F5F3F4F26173707C8F3842F9927089543
:103B2000AC019AEA20E030E02617370750F4DA01BA
:103B3000A20FB31F0E946B7A802D980F2F5F3F4F0B
:103B4000F3CF892F9927089581E08093BC0582E007
:103B50008093BB0583E08093BA0584E08093BD0524
:103B600085E08093BE0586E08093BF0587E0809363
:103B7000C00588E08093C10589E08093C2058AE092
:103B80008093C3058BE08093C4058CE08093C505CA
:103B900008951F93CF93DF9384E58093B9058091B7
:103BA0000201843150F08AE08093D9051092FB0520
:103BB0008BE18093D5058EE40AC083E08093D9051C
:103BC00080E28093FB058EE18093D50585E58093A7
:103BD000F8058093F9058AE68093C60583E0809313
:103BE0001C06AEE1A093C7058FEF8093C905EFE0F7
:103BF000E093CA05A093C8051092CC05F8E0F093B5
:103C0000CD0580E48093CE051092CF0584E18093AA
:103C1000CB058EE08093D005B0E1B093D1051CE0D8
:103C20001093D205F093D30586EE8093D40580E8F7
:103C30008093D60550E55093D70586E98093D80543
:103C40005093DA058093DB0576E07093DC0581E222
:103C50008093DD058DE28093DE059AE59093DF0584
:103C600080E28093E1051092E2051092E305109244
:103C7000E4051092E5051092FD051092FE051092E4
:103C8000FF051092000634E63093E60548E24093C3
:103C9000E70561E060931B061092E80527EF20938B
:103CA000E9057093EE058DE78093EF058093F005AD
:103CB0008093F1053093EA054093EB051092EC05F3
:103CC0002093ED0582E38093F2059093F3058093B2
:103CD000F40510921A069093F5055093F60560933B
:103CE000F705B093FA053093FC058FE58093010644
:103CF00083EF809303068AEA809305068093060685
:103D0000E0930206E09304068EEF8093070630935B
:103D100008069093090690930A0690930B068BE48D
:103D200080930C0680930D0680930E0610920F066A
:103D300070931006F093110690931206A093130649
:103D4000309314063093150682E080931606609334
:103D5000E0051092180610921906ADE1B6E0EFE109
:103D6000F1E0ED01019009921A95E1F760E770E04A
:103D7000CD01845690400E947F1D80932906DF91DB
:103D8000CF911F910895CF93DF9384E58093B90578
:103D900080910201843150F08AE08093D90510921D
:103DA000FB058BE18093D5058EE40AC083E0809308
:103DB000D90580E28093FB058EE18093D50585E5EA
:103DC0008093F8058093F9058AE68093C60583E021
:103DD00080931C067EE17093C7058FEF8093C90521
:103DE0009FE09093CA057093C8051092CC0568E0D7
:103DF0006093CD0580E48093CE051092CF0590931B
:103E0000CB058AE08093D00580E18093D10556E010
:103E10005093D2056093D30586EE8093D40580E855
:103E20008093D6052AE52093D70588E78093D805A7
:103E30002093DA058093DB055093DC0581E28093C3
:103E4000DD058DE28093DE052093DF05E0E2E0935F
:103E5000E1051092E2051092E3051092E40510923C
:103E6000E5051092FD051092FE051092FF051092D7
:103E7000000644E64093E60538E23093E705F1E0BA
:103E8000F0931B061092E80597EF9093E905509385
:103E9000EE058DE78093EF058093F0058093F105A3
:103EA0004093EA053093EB051092EC059093ED05F5
:103EB00082E38093F2052093F3058093F40510923A
:103EC0001A062093F50580E58093F6058CE3809330
:103ED000F705E093FA059BE49093FC058FE580934A
:103EE000010683EF809303068AEA80930506809398
:103EF000060684E180930206809304068EEF809389
:103F00000706409308062093090620930A0620938B
:103F10000B0690930C0690930D0690930E0610924C
:103F20000F065093100660931106209312067093AB
:103F30001306409314064093150682E080931606FC
:103F4000F093E0051092180610921906ADE1B6E064
:103F50008CE0E6E2F1E0ED01019009928A95E1F74B
:103F600060E770E0CD01845690400E947F1D8093F1
:103F70002906DF91CF910895CF93DF9384E5809355
:103F8000B90580910201843150F08AE08093D9050F
:103F90001092FB058BE18093D5058EE40AC083E087
:103FA0008093D90580E28093FB058EE18093D5054F
:103FB00085E58093F8058093F9058AE68093C60528
:103FC00083E080931C066EE16093C7058FEF8093BA
:103FD000C9059FE09093CA056093C8051092CC056F
:103FE00078E07093CD0580E48093CE051092CF05E4
:103FF0009093CB057093D00590E19093D10556E056
:104000005093D2057093D30586EE8093D40580E853
:104010008093D60534E63093D70588E78093D8059A
:104020003093DA058093DB055093DC0581E28093C1
:10403000DD058DE28093DE052AE52093DF05909370
:10404000E1051092E2051092E3051092E40510924A
:10405000E5051092FD051092FE051092FF051092E5
:1040600000063093E60548E24093E705E1E0E0937F
:104070001B061092E80597EF9093E9055093EE0523
:104080008DE78093EF058093F0058093F1053093E1
:10409000EA054093EB051092EC059093ED0582E361
:1040A0008093F2052093F3058093F40510921A068D
:1040B0002093F50580E58093F60596E49093F70547
:1040C00080E28093FA059093FC058FE580930106CA
:1040D00083EF809303068AEA8093050680930606A1
:1040E00060930206609304068EEF80930706309378
:1040F00008062093090620930A0620930B068BE4FA
:1041000080930C0680930D0680930E0610920F0686
:1041100050931006709311062093120660931306B5
:10412000309314063093150682E080931606E093D0
:10413000E0051092180610921906ADE1B6E08CE089
:10414000EEE2F1E0ED01019009928A95E1F760E776
:1041500070E0CD01845690400E947F1D8093290617
:10416000DF91CF910895DC010E946B7A802D992711
:104170000895DC01062E0E947D7A0895DC010E94DC
:10418000787ACF010895DC010B010E94897A0895A5
:10419000FF920F931F93CF93DF93982F8150853019
:1041A00008F093E081E7F82E9F9D80011124E8013B
:1041B0002D9760E770E0CE010E94901D982FD801E6
:1041C000AD59BF4F0E946B7A802D891731F4DE0103
:1041D0000E946B7A802D843519F080E090E00AC04F
:1041E000E9EBF5E0DE011F2C0E94737A0E94C75AAA
:1041F00081E090E0E5E0CDB7DEB70C94577A8630E9
:1042000010F085E003C0882309F481E0A2E0B0E06B
:10421000082E0E947D7A08951F93CF93DF93182F65
:10422000C9EBD5E08091B905843591F5163010F0D1
:1042300015E002C0112361F160E770E089EB95E0C1
:104240000E947F1D8093290681E7189FD0011124C9
:104250001D97FE01182E0E948E7AEAEBF5E0A0E58C
:10426000B0E02CE030E0122E0E948E7AB9018AEB89
:1042700095E00E947F1DACE5B0E0082E0E947D7A9B
:10428000812F0E94FF200E94C75A81E090E002C067
:1042900080E090E0DF91CF911F9108956DE470E090
:1042A00088EE93E00E94901DA5E3B4E00E946B7A33
:1042B000902D981739F4A8EEB3E00E946B7A802D08
:1042C000813019F080E090E00895EAE2F6E0A8EE8F
:1042D000B3E08EE4182E0E94737A81E090E0089596
:1042E000CF93DF93CAE2D6E080912A06813089F429
:1042F0006DE470E0CE010E947F1D80937706A8EEEA
:10430000B3E08EE4FE01182E0E948E7A81E090E0E8
:1043100002C080E090E0DF91CF910895CF93DF93CA
:1043200081E080932A06EAE2F6E08FE015861686A1
:104330001786108A8150349687FFF8CF80E48093E7
:104340003706809338061092390680933A06809398
:104350003B0690EC90933C0610923D0680933E06FF
:1043600080933F0610924006909341069093420638
:104370008093430610924406809345069093460628
:10438000ABE2B6E087E0E8E3F1E0ED0101900992ED
:104390008A95E1F76DE470E0CD0101970E947F1DE1
:1043A00080937706DF91CF910895A2E0B0E00E945C
:1043B0006B7A802D863030F083E0A2E0B0E0082EEA
:1043C0000E947D7A99270895DF92EF92FF920F93D2
:1043D0001F93CF93FF24DF2CEF2C81E090E00E940D
:1043E000B320843539F031E0E32E64E581E090E0DC
:1043F0000E94B9206CE070E080E590E00E94901D82
:10440000C82FACE5B0E00E946B7A802D8C1711F4B8
:1044100021E0D22EC1E001E010E0EE2029F48C2F43
:104420000E94C8208823B1F591E0F92E1F930F93C5
:104430008EE793E09F938F9389E890E19F938F930A
:10444000E091DA03F091DB0309958DB79EB70696EC
:104450008DBF0230110549F0033011054CF40130D5
:10446000110531F40E94C91D05C00E94C31E02C07F
:104470000E94BC1FDD2049F0EAEBF5E0A0E5B0E0CA
:104480008CE0182E0E94737A02C00E94A41D8C2F0B
:104490000E940C21CF5F0F5F1F4FC63008F4BDCFC5
:1044A000FF2019F083E00E94FF200E94D521C82F31
:1044B0000E94C8208C2F99279F938F9384EA93E0C2
:1044C0009F938F9309E810E11F930F93E091DA0314
:1044D000F091DB0309958DB79EB706968DBFEE2050
:1044E00021F40E944E21882399F48DEB93E09F9351
:1044F0008F931F930F93E091DA03F091DB030995FB
:104500000E948E210E9470210F900F900F900F90AB
:104510001092B80590E0E7E3F6E0CFE080813496B2
:1045200018160CF49F5FC150C7FFF8CF9093B805E1
:10453000892F99279F938F938BE296E09F938F9378
:104540008EED93E09F938F931F930F93E091DA0387
:10455000F091DB0309958DB79EB708968DBF8FEF5D
:1045600093E09F938F931F930F93E091DA03F09161
:10457000DB0309950F900F900F900F90CF911F9133
:104580000F91FF90EF90DF9008959FB7F8943998BE
:10459000389A88B1836088B98091B9008C7F809304
:1045A000B9008AE28093B80010921F0210921D0297
:1045B00010921C02E0E8F6E08BE010821182128279
:1045C000138214821582168217828150389687FFD3
:1045D000F4CF9FBF089510921F0284E98093BC001E
:1045E00010921D0210921C0280E88093BC00109271
:1045F000BD001092BA001092BB001092B900109248
:10460000B8000E94C5221092BB0085E88093BC00D0
:1046100080911A02826080931A0208951F920F926D
:104620000FB60F9211242F933F934F935F938F9365
:104630009F93EF93FF9380911F02282F33274427E6
:1046400055278F5F80931F02F9012731310508F04C
:10465000B3C2E05BFF4F0C94657A80911D028C30F1
:1046600090F480911D028F5F80931D0280911D0246
:10467000E82FFF27EE0FFF1FEE0FFF1FE65DF94F3C
:104680008585181654F780911D028C3070F01092B9
:1046900019021092180210921D0285E080931F02E9
:1046A00080911C02880F8D5A04C080911D02880FD2
:1046B0008E5A8093BB0085E874C280911D02E82F5A
:1046C000FF2783E0EE0FFF1F8A95E1F7E058F94FCF
:1046D00081818093BB0085E88093BC0080911D029E
:1046E000E82FFF27EE0FFF1FEE0FFF1FEE0FFF1F3C
:1046F000E058F94F808180FF91C080911D02E82F22
:10470000FF27EE0FFF1FEE0FFF1FEE0FFF1FE058FA
:10471000F94F8281882329F08091B805873008F409
:104720005FC28091180290911902892B09F058C23A
:104730008091160290911702892B09F051C26EC028
:1047400080911D0221E030E002C0220F331F8A95C4
:10475000E2F7809116029091170228233923232B28
:1047600079F080911D02E82FFF27EE0FFF1FEE0F5B
:10477000FF1FEE0FFF1FE058F94F80E184830DC04B
:1047800080911D02E82FFF27EE0FFF1FEE0FFF1F86
:10479000EE0FFF1FE058F94F148280911D02E82FA1
:1047A000FF2753E0EE0FFF1F5A95E1F7E058F94F4E
:1047B0008481282F332743E0220F331F4A95E1F7E6
:1047C00080911D02E82FFF2793E0EE0FFF1F9A95BF
:1047D000E1F7E058F94F82818770822B8093BB000C
:1047E00085E88093BC0020911D0281E090E002C02A
:1047F000880F991F2A95E2F720911802309119022B
:1048000082239323892B51F088E796E0909323022B
:104810008093220288E080932402E2C184E080C178
:10482000E0912202F091230281918093BB0085E800
:104830008093BC00F0932302E09322028091240233
:10484000815080932402882309F4CAC183E068C19F
:104850008091B900803351F580912002882329F49A
:1048600080911D028F5F8093200280911D02E82FAE
:10487000FF2783E0EE0FFF1F8A95E1F7E058F94F1D
:10488000838199278F7790708F3791057CF4809181
:104890001D02E82FFF27EE0FFF1FEE0FFF1FEE0F89
:1048A000FF1FE058F94F83818F5F838310921F02AF
:1048B00084E98093BC008AE090E09093410180936A
:1048C000400180911D028F5F80931D0210921F0294
:1048D00062C18091B9008034A9F180911C02E82F57
:1048E000FF27EE0FFF1FEE0FFF1FEE0FFF1FE05819
:1048F000F94F83818F77838380911C028F5F809330
:104900001C0280911C028C30A0F010921C021092AC
:10491000170210921602809121028F5F809321026C
:104920008C3038F01092210280911A028D7F809392
:104930001A0280911A02816080931A0210921F025B
:1049400084E971C080911C02E82FFF27EE0FFF1F42
:10495000EE0FFF1FEE0FFF1FE058F94F83818068B5
:10496000838380911C02E82FFF27EE0FFF1FEE0FBD
:10497000FF1FEE0FFF1FE058F94F808180FF2FC00F
:1049800080911C02E82FFF2753E0EE0FFF1F5A957E
:10499000E1F7E058F94F84819927009751F040974B
:1049A000D9F588E796E0909323028093220288E06D
:1049B00031C080911C02992743E0880F991F4A95C6
:1049C000E1F78B57994F90932302809322029091A5
:1049D0001C02809121029817E1F483E01BC08091B2
:1049E0001C02992733E0880F991F3A95E1F78B57FE
:1049F000994F909323028093220280911A0281FDA5
:104A000006C090911C0280912102981711F482E057
:104A100001C081E08093240280912402813011F44E
:104A200085E801C085EC8093BC00809120028093D2
:104A30001B0210922002D4C0E0912202F0912302C6
:104A40008091BB0080838091220290912302019685
:104A500090932302809322028091240281508093BC
:104A60002402823010F085EC58C0813011F485E8C2
:104A700054C080911A0281FF2DC08091960280FD62
:104A80001DC080911C02E82FFF2723E0EE0FFF1FBF
:104A90002A95E1F7E058F94F86818A3F79F48091B1
:104AA0001C02E82FFF2793E0EE0FFF1F9A95E1F716
:104AB000E058F94F8081816080830CC080911C0296
:104AC000E82FFF2783E0EE0FFF1F8A95E1F7E058FC
:104AD000F94F108280911C028F5F80931C0280919D
:104AE0001C028C30A0F010921C021092170210923F
:104AF0001602809121028F5F809321028C3038F062
:104B00001092210280911A028D7F80931A021092D6
:104B10001F0284E98093BC0049C08093BC0086E0FA
:104B200080931F025DC088E9C4CD80911E02880F6A
:104B3000805FBFCD80911E0299278130910561F081
:104B4000823091051CF4892B21F04AC0029739F07C
:104B500047C080911201ADCD80911101AACD809105
:104B60001001A7CD80E8A5CD10921F0284E98093A3
:104B7000BC008AE090E090934101809340018091D5
:104B80001E02823088F480911E028F5F80931E0285
:104B900082E180931F0280911A028E7F80931A0215
:104BA00085EA8093BC001CC010921E0280911A02FC
:104BB000816080931A0214C010921F0284E98093CE
:104BC000BC0080911A02816080931A028AE090E012
:104BD000909341018093400110921D0210921C029B
:104BE000FF91EF919F918F915F914F913F912F9105
:104BF0000F900FBE0F901F9018951F93CF93DF93C8
:104C0000182F8091C102882321F48091B401882358
:104C100019F081E090E097C01D3008F092C0112398
:104C2000B1F0E12FFF2723E0EE0FFF1F2A95E1F7F8
:104C3000E058F94F35978081359688230CF081C074
:104C40003897808180FD03C083E090E07CC0809134
:104C50007806823019F084E090E075C067E070E07B
:104C600088E796E00E947F1D90917F06891719F0D2
:104C700085E090E068C080ED97E00E940D14EC01A3
:104C800080911A0280FD05C0CE010E94161488236F
:104C9000B9F3112319F48FEF90E00BC0212F3327C4
:104CA0002150304081E090E002C0880F991F2A9582
:104CB000E2F79093190280931802A1E0B0E0E0E8D7
:104CC000F6E040E050E06BE0CD01042E02C0880F1A
:104CD000991F0A94E2F72091180230911902822359
:104CE0009323892B11F01182128261504F5F5F4F25
:104CF000389667FFE9CF10921D0210921F02809133
:104D00001A028E7F80931A0285EA8093BC008091FC
:104D10001A0280FD05C0CE010E9416148823B9F343
:104D20008091180290911902892B29F0CE010E94DE
:104D30001614882311F3809118029091190200979C
:104D400011F082E090E0DF91CF911F9108950F93D1
:104D50001F93CF93DF93982F8091C102882321F472
:104D60008091B401882319F081E090E092C09D30D9
:104D7000A0F4992319F486E090E08BC0C92FDD27B9
:104D8000FE0133E0EE0FFF1F3A95E1F7E058F94FCF
:104D900035978081359687FD03C082E090E079C029
:104DA0003897808180FD03C083E090E072C080ED81
:104DB00097E00E940D148C0180911A0280FD05C0BD
:104DC000C8010E9416148823B9F3219721E030E02E
:104DD000C90102C0880F991FCA95E2F79093170284
:104DE00080931602D901E0E8F6E040E050E06BE085
:104DF000CD01042E02C0880F991F0A94E2F720917A
:104E000016023091170282239323892B11F011820D
:104E1000128261504F5F5F4F389667FFE9CF109263
:104E20001C021092780610927F0610921F02809149
:104E30001A028E7F80931A0285EA8093BC008091CB
:104E40001A0280FD05C0C8010E9416148823B9F318
:104E50008091160290911702892B29F0C8010E94B7
:104E60001614882311F380917806823019F084E0BB
:104E700090E00FC067E070E088E796E00E947F1D39
:104E800090917F06891719F085E090E002C080E0DC
:104E900090E0DF91CF911F910F91089589E1A5E1F5
:104EA000B7E0E1EEF6E011821082329611961C9284
:104EB0001E921296815087FFF6CF8091FB0690914B
:104EC000FC068F5790409093FC068093FB068091E0
:104ED000FD069091FE068F5790409093FE068093BA
:104EE000FD068091FF06909100078F5790409093A8
:104EF000FC068093FB0680910107909102078F5773
:104F000090409093FE068093FD061092300310921D
:104F10002F03109232031092310310923403109237
:104F2000330308951F920F920FB60F9211240F931F
:104F30001F932F933F934F935F936F937F938F9321
:104F40009F93AF93BF93CF93DF93EF93FF938091A2
:104F50001C0682FDCFC04091860050918700809151
:104F6000260290912702481B590B80918600909150
:104F700087009093270280932602CA018D549440A3
:104F8000A0912802B0912902835F9A4178F4809120
:104F900028028093E006149714F01092420181E0F9
:104FA00090E0909329028093280207C2AD30B105AA
:104FB0000CF003C2CA018B5F9040845B914008F003
:104FC00074C0425D5140FD01EA0FFB1FEF51F94FE4
:104FD00080819181FA01E81BF90BCF01F7FF03C033
:104FE000909581959F4F06975CF48091CA02883C0A
:104FF00020F48091CA02865F01C088EC8093CA02C7
:10500000FD01EA0FFB1FEF51F94F808191819C0157
:10501000220F331F280F391F240F351F37FF02C0FF
:105020002D5F3F4FE901D595C795D595C795CA0125
:1050300001968C179D0714F4219706C041505040EB
:10504000C417D5070CF421968091CA02833CE0F086
:105050008D010A0F1B1FF801EF51F94F80819181DB
:105060009E01281B390BC90163E070E00E94DE79C4
:10507000CB01880F991F860F971F0B5E184FD80121
:1050800011969C938E9307C0AA0FBB1FAB5EB84FBF
:1050900011961C921E92E0912802F0912902EE0FC7
:1050A000FF1FEF51F94FD183C08320912802309127
:1050B00029022F5F3F4F30932902209328028091CD
:1050C0000201843108F079C12530310511F45D9A6F
:1050D00001C05D9880912802909129028630910547
:1050E00011F45C9A01C05C98079711F45B9A65C152
:1050F0005B9863C1409186005091870080912A029D
:1051000090912B02481B590B80918600909187004B
:1051100090932B0280932A02CA018D54944060918F
:105120009402835F9A4108F07AC0609325028091CF
:105130002502843008F453C09091E0068091250246
:10514000981709F04CC0509195025B3008F43FC0AD
:10515000109242011092940240E05F31C0F0E42FBF
:10516000FF27EE0FFF1F9F01205A3D4FDF01AF5178
:10517000B94F8D919C91D9018D939C93DF01AB5ECA
:10518000B84F8D919C91E658FD4F91838083E42F19
:10519000FF27EE0FFF1F9F012F51394FDF01A45D45
:1051A000BD4F8D919C91D90111969C938E93DF01F7
:1051B000AA5BBD4F8D919C91EB5EF84F91838083EC
:1051C000842F8F5F482F8D3040F28093940280911E
:1051D00095028F3FB9F08F5F8093950213C0809145
:1051E0009502853620F08AE08093950202C01092E5
:1051F0009502809102018A3011F0843110F0289AD2
:1052000001C0289881E0809394028091C102882394
:1052100009F0D3C0809125028093E006CEC06D30A6
:1052200008F0A3C0CA018B5F9040845B914008F0F6
:105230007EC0425D5140E62FFF27EE0FFF1FE45D69
:10524000FD4F80819181FA01E81BF90BCF01059692
:105250000B97B0F4809195028A3120F08091CA02B8
:10526000865F05C08B3028F08091CA028E5F8093E4
:10527000CA028091CA02893C18F088EC8093CA0265
:10528000E62FFF27EE0FFF1FE45DFD4F8081918128
:105290009C01220F331F280F391F240F351F37FFA2
:1052A00002C02D5F3F4FE901D595C795D595C795AC
:1052B000CA0101968C179D0714F4219706C041502E
:1052C0005040C417D5070CF421968091CA028E3B3A
:1052D000D8F0E62FFF27EE0FFF1FDF01A45DBD4FC3
:1052E0008D919C919E01281B390BC90163E070E0F0
:1052F0000E94DE79CB01880F991F860F971FEA5B0A
:10530000FD4F9183808308C0E62FFF27EE0FFF1F1C
:10531000EA5BFD4F1182108280919402E82FFF27F3
:10532000EE0FFF1FE45DFD4FD183C08309C0809164
:1053300002018A3011F0843110F0289A01C02898B7
:1053400080910201843188F480919402853011F4B7
:105350005D9A05C05D98863011F45C9A05C05C9832
:10536000873011F45B9A01C05B988091940284317C
:1053700020F48F5F8093940220C08431F1F48091F7
:1053800002018A3011F0843110F0289A01C0289867
:105390008EE1809394022CE0C5E1D7E0A0E6B2E074
:1053A000E1EEF6E08D919D91918380833296198292
:1053B00018822296215027FFF5CFFF91EF91DF91C0
:1053C000CF91BF91AF919F918F917F916F915F919D
:1053D0004F913F912F911F910F910F900FBE0F9002
:1053E0001F901895EF92FF920F931F938091D50510
:1053F0009927880F991F880F991F7C010027F7FCB8
:105400000095102F80911E0390911F03A0912003FF
:10541000B0912103BC01CD01A80197010E94137A2C
:1054200030936505209364058091160390911703CE
:10543000A0911803B0911903BC01CD01A8019701F7
:105440000E94137A30936705209366058091A60722
:105450009091A70797FD03969595879595958795C4
:1054600090936905809368058091B8079091B9077A
:1054700097FD0396959587959595879590936B05E0
:1054800080936A0580912F03909130032091F4015D
:105490003091F501821B930B90936D0580936C0501
:1054A0008091BC029091BD02A091BE02B091BF025A
:1054B000BC01CD0125E030E040E050E00E94137ACD
:1054C00030936F0520936E058091EE019091EF016E
:1054D00090937105809370058091DC029091DD02BC
:1054E000909375058093740580911D0190911E0124
:1054F00090937705809376058091CA0299279093BF
:105500007905809378058091B4079091B507A091B3
:10551000B607B091B7072091440130914501409101
:10552000460150914701BC01CD010E94137A30938E
:105530007B0520937A0580918106992790937D05BC
:1055400080937C0580918906992790937F058093AD
:105550007E0580919106992790938105809380051F
:105560008091990699279093830580938205809175
:10557000A106992790938505809384058091A906BB
:10558000992790938705809386058091B106992786
:1055900090939505809394058091B90699279093EF
:1055A0009705809396058091C10699279093990558
:1055B000809398058091C906992790939B058093C5
:1055C0009A058091CF019091D00190938D058093A1
:1055D0008C0580912C0890912D08909391058093D3
:1055E00090058091300890913108909393058093B5
:1055F000920580913208992790939F0580939E058C
:105600008091AA039091AB039093A1058093A0058C
:105610008091A8039091A9039093A3058093A2057C
:105620008091F603882321F48091F703882321F0E9
:1056300080916305816003C0809163058E7F8093B4
:1056400063051F910F91FF90EF9008951F93CF93E3
:10565000DF93182FEB018091C1028823A1F4115030
:105660001F3F89F0D093D401C093D3018091D3011F
:105670009091D401892BD1F7CE018C0F9D1F0E94F0
:105680002214115078F7DF91CF911F910895CF9395
:10569000DF93809102018D3011F40E94BC181092AA
:1056A0007A008091F8019091F901909364078093BA
:1056B00063078091F6019091F701909353078093CF
:1056C00052078091F4019091F5019093AE07809379
:1056D000AD072091F0013091F101C901880F991FA8
:1056E000880F991F820F931F820F931F9093A70714
:1056F0008093A6072091F2013091F301C901880F30
:10570000991F880F991F820F931F820F931F9093E9
:10571000B9078093B8078FEC80937A00ABECB2E0C6
:10572000CEEBD5E097E08991E82FFF27EE0FFF1F22
:10573000EF51F94F0190F081E02DE259FF4F1E1615
:105740001F061CF0E0E0F0E005C0EF3FF10514F0AB
:10575000EFEFF0E08C91282F3327E217F30714F4D2
:10576000815004C02E173F0714F48F5F8C93915023
:10577000119697FFD8CF8091F8059927AA27BB27C4
:10578000BC01CD0124EC39E040E050E00E949F795B
:10579000DC01CB018093640190936501A0936601C5
:1057A000B09367018091F9059927AA27BB27BC010F
:1057B000CD010E949F79DC01CB0180936001909321
:1057C0006101A0936201B0936301DF91CF910895CD
:1057D000A0E0B0E0EEEEFBE20C94347A882EC0E05C
:1057E000D0E07E016E011092F603469AD0932A0310
:1057F000C0932903D0932803C0932703D093240395
:10580000C0932303D0933403C0933303D093320364
:10581000C0933103D0933003C0932F0310924D01F6
:1058200010924C011092E8010E94472B84E690E010
:105830000E942F140E94472B8091C60580FF10C044
:105840008091130190911401875B934038F480910B
:105850001301909114018E5E924010F40E94611821
:105860000FE18AE090E00E942F148091F401909162
:10587000F501C80FD91F8091F8019091F901E80E48
:10588000F91E8091F6019091F701C80ED91E0150C2
:1058900007FFE7CF9701205F3F4F36952795369555
:1058A00027953093340320933303C6014096969591
:1058B00087959695879590933203809331036096F0
:1058C000F5E0D695C795FA95E1F7D0933003C093EC
:1058D0002F0390932E0380932D0330932C0320935A
:1058E0002B03882009F441C08091A6079091A70757
:1058F00097FF03C0909581959F4F6CE070E00E94E8
:10590000DE799B0170932A03609329038091B80785
:105910009091B90797FF03C0909581959F4F6CE0D8
:1059200070E00E94DE7970932803609327038091D2
:10593000AB059091AC059093240380932303B901A8
:1059400084E090E00E94C3206091270370912803B7
:1059500086E090E00E94C3206091230370912403AD
:1059600088E090E00E94C32065C084E090E00E943F
:10597000BE2090932A038093290386E090E00E9442
:10598000BE20909328038093270388E090E00E9434
:10599000BE209C01909324038093230380912903CC
:1059A00090912A038150984050F480912703909160
:1059B00028038150984018F421503440D8F183E0F6
:1059C00094E09F938F9389E890E19F938F93E09168
:1059D000DA03F091DB0309958091A6079091A70760
:1059E00097FF03C0909581959F4F6CE070E00E94F7
:1059F000DE7970932A03609329038091B807909110
:105A0000B90797FF03C0909581959F4F6CE070E0B8
:105A10000E94DE7970932803609327038091AB0581
:105A20009091AC0590932403809323030F900F90E3
:105A30000F900F9010926407109263071092530713
:105A4000109252071092AE071092AD0784E690E0D4
:105A50000E942F148091F0019091F1019C01220F7E
:105A6000331F220F331F280F391F280F391F309380
:105A7000A7072093A6078091F2019091F3018C0172
:105A8000000F111F000F111F080F191F080F191FFA
:105A90001093B9070093B8078091D505C82EDD246F
:105AA000EE24FF24442737FD4095542FC701B6014B
:105AB0000E949F794B015C0160931E0370931F034A
:105AC00080932003909321039801442737FD40954C
:105AD000542FC701B6010E949F79DC01CB0180934E
:105AE000160390931703A0931803B09319038092A1
:105AF000FA029092FB02A092FC02B092FD02809307
:105B0000F2029093F302A093F402B093F502109284
:105B1000EE021092EF021092F0021092F1028091C8
:105B2000150190911601A0911701B0911801909361
:105B3000AE058093AD051092E7011092E601109238
:105B4000DE021092DF021092E0021092E1028091D8
:105B5000DC029091DD029093DB028093DA020E94D6
:105B60005E5682E390E09093D4018093D3018091BC
:105B7000F8059927AA27BB27BC01CD0124EC39E001
:105B800040E050E00E949F79DC01CB018856954CA3
:105B9000AF4FBF4F8093640190936501A09366015E
:105BA000B09367018091F9059927AA27BB27BC010B
:105BB000CD010E949F79DC01CB018856954CAF4FF7
:105BC000BF4F8093600190936101A0936201B093F5
:105BD000630110924901109248018091DC0290917A
:105BE000DD02AA2797FDA095BA2F2091440130919C
:105BF00045014091460150914701BC01CD010E94F1
:105C00009F79DC01CB018093B4079093B507A093F3
:105C1000B607B093B7071092D5021092D40281E074
:105C2000809301010E94C75A8091960284608093FC
:105C300096028FEF809327081092280880E28093C5
:105C40002908CBECD2E0AEEBB5E007E08D91E82F70
:105C5000FF27EE0FFF1FEF51F94F8081918182598D
:105C60008993015007FFF2CF84E68093CA028091A6
:105C7000D101882311F0469A579A8091330390916D
:105C8000340380569940815C9B4228F08091F60352
:105C900081608093F60380913103909132038056A6
:105CA0009940815C9B4228F08091F603826080934A
:105CB000F60380912F03909130038C5291408957C5
:105CC000954028F08091F60384608093F6038091DC
:105CD000290390912A038C529140835C914028F0D3
:105CE0008091F60388608093F6038091270390915A
:105CF00028038C529140835C914028F08091F603F8
:105D000080618093F6038091230390912403805057
:105D100092408355914028F08091F60380628093F1
:105D2000F603ECE0CDB7DEB70C94507AA3E1B0E017
:105D3000ECE9FEE20C942E7A80912F0390913003CF
:105D40002091F4013091F501821B930B9093AE07E3
:105D50008093AD078091FE019091FF0197FD07961A
:105D60009C0153E0359527955A95E1F730936407E8
:105D7000209363078091FC019091FD0197FD0796A8
:105D800043E0959587954A95E1F790935307809363
:105D900052073093700720936F07909368078093A2
:105DA00067078091A6079091A707AC01440F551F84
:105DB000480F591F2091F0013091F101C901880F5E
:105DC000991F880F991F820F931F820F931F480FEF
:105DD000591F57FF02C04D5F5F4F55954795559529
:105DE00047955093A7074093A6078091B8079091D5
:105DF000B907AC01440F551F480F591F2091F201FC
:105E00003091F301C901880F991F880F991F820FE4
:105E1000931F820F931F480F591F57FF02C04D5FFA
:105E20005F4F55954795559547955093B9074093C2
:105E3000B8072091F0013091F101C901880F991F35
:105E4000880F991F820F931F820F931F9C01442775
:105E500037FD4095542F80910E0390910F03A09130
:105E60001003B0911103820F931FA41FB51F8093DD
:105E70000E0390930F03A0931003B093110320918E
:105E8000F2013091F301C901880F991F880F991F02
:105E9000820F931F820F931F9C01442737FD40956B
:105EA000542F80910A0390910B03A0910C03B091A1
:105EB0000D03820F931FA41FB51F80930A039093B5
:105EC0000B03A0930C03B0930D0380917B0790917B
:105ED0007C072091F0013091F101820F931F909384
:105EE0007C0780937B078091B0079091B107209148
:105EF000F2013091F301820F931F9093B1078093C9
:105F0000B007809125039091260301969093260374
:105F1000809325038091AB059091AC0520912303DC
:105F200030912403821B930B9C01442737FD40953D
:105F3000542F8091060390910703A0910803B0911C
:105F40000903820F931FA41FB51F8093060390932C
:105F50000703A0930803B09309038FEC80937A00A2
:105F600010920F012091F6023091F7024091F80251
:105F70005091F90229873A874B875C8729543B4621
:105F8000414050402CF028E43BE641E050E00DC099
:105F900089859A85AB85BC85885B9449AE4FBF4F98
:105FA0004CF428EB34E94EEF5FEF2D833E834F83B3
:105FB000588708C089859A85AB85BC858D839E836B
:105FC000AF83B8872091FE023091FF024091000319
:105FD000509101032D873E874F87588B29543B46AC
:105FE000414050402CF028E43BE641E050E00DC039
:105FF0008D859E85AF85B889885B9449AE4FBF4F2C
:106000004CF428EB34E94EEF5FEF29833A834B835E
:106010005C8308C08D859E85AF85B88989839A8306
:10602000AB83BC83A091AD07B091AE07BB8BAA8BAD
:10603000FD01CF01AA2797FDA095BA2FA090EE02EF
:10604000B090EF02C090F002D090F102A80EB91EFD
:10605000CA1EDB1EA092EE02B092EF02C092F002C6
:10606000D092F102E090B407F090B5070091B60726
:106070001091B707E80EF91E0A1F1B1FE092B40724
:10608000F092B5070093B6071093B707F091B102ED
:10609000F98BFF2309F098C18091B002882309F0A1
:1060A00093C18091C60586FF8FC180915207909160
:1060B0005307AA2797FDA095BA2FBC01CD012981CE
:1060C0003A814B815C810E949F799B01AC0197FFD3
:1060D00004C02150384F4F4F5F4F6BE055954795A7
:1060E000379527956A95D1F780914C01682E7724D2
:1060F00088249924CA01B901A40193010E949F79BF
:10610000DC01CB018093420390934303A0934403AB
:10611000B0934503B7FF04C08150904FAF4FBF4FBE
:106120001C012D013CE055944794379427943A95EF
:10613000D1F720924203309243034092440350929D
:1061400045038091630790916407AA2797FDA09566
:10615000BA2FBC01CD012D813E814F8158850E940F
:106160009F7997FF04C06150784F8F4F9F4F2BE06E
:1061700095958795779567952A95D1F7A401930111
:106180000E949F79DC01CB018093460390934703E3
:10619000A0934803B0934903B7FF04C08150904FC8
:1061A000AF4FBF4F9C01AD018CE05595479537959A
:1061B00027958A95D1F72093460330934703409360
:1061C0004803509349038091420390914303909375
:1061D0004A07809349078091460390914703909323
:1061E0004E0780934D07221933094409550920931E
:1061F0004603309347034093480350934903E20E0C
:10620000F31E041F151FE092B407F092B507009328
:10621000B6071093B70780914B018823B1F457FF5D
:1062200004C02F5F3F4F4F4F5F4F559547953795B0
:106230002795A21AB30AC40AD50AA092EE02B09218
:10624000EF02C092F002D092F1022A893B897901D3
:106250000027F7FC0095102F80914603909147038B
:10626000A0914803B0914903E80EF91E0A1F1B1FB5
:10627000C801B70129813A814B815C810E949F79D5
:106280009B01AC0197FF04C02150384F4F4F5F4F27
:10629000BBE05595479537952795BA95D1F78091ED
:1062A0004D01A82EBB24CC24DD24CA01B901A601CE
:1062B00095010E949F79DC01CB0180933A03909372
:1062C0003B03A0933C03B0933D03B7FF04C0815050
:1062D000904FAF4FBF4F3C014D01ACE09594879478
:1062E00077946794AA95D1F760923A0370923B0332
:1062F00080923C0390923D03C801B7012D813E81FD
:106300004F8158850E949F7997FF04C06150784F54
:106310008F4F9F4FFBE09595879577956795FA95F9
:10632000D1F7A60195010E949F79DC01CB018093F2
:106330003E0390933F03A0934003B0934103B7FF04
:1063400004C08150904FAF4FBF4FAC01BD01ECE096
:106350007595679557954795EA95D1F740933E0314
:1063600050933F0360934003709341032A893B8914
:1063700037FF03C0309521953F4F21343105E4F1BB
:10638000D401C30197FE07C0B095A0959095819563
:106390009F4FAF4FBF4F81389105A105B10584F4E0
:1063A000DB01CA0177FF07C0B095A0959095819554
:1063B0009F4FAF4FBF4F81389105A105B105E4F064
:1063C00081E08093D60218C010924E0710924D07BC
:1063D00010924A071092490710923E0310923F0311
:1063E000109240031092410310923A0310923B0323
:1063F00010923C0310923D0380913E0390913F0325
:10640000A0914003B0914103BC01CD0124E630E0EE
:1064100040E050E00E94137AE0903A03F0903B0392
:10642000E21AF30AF0926207E092610780913A0360
:1064300090913B03A0913C03B0913D03BC01CD0181
:1064400024E630E040E050E00E94137ADA01C9010E
:1064500020913E0330913F038C01021B130B1093DC
:106460005607009355078091440190914501A091F2
:106470004601B0914701BC01CD0128E631E040E082
:1064800050E00E949F792091B4073091B507409168
:10649000B6075091B707261737074807590764F022
:1064A000261B370B480B590B2093B4073093B507C5
:1064B0004093B6075093B7072091B4073091B507C2
:1064C0004091B6075091B70757FF0CC0260F371FF2
:1064D000481F591F2093B4073093B5074093B60760
:1064E0005093B70760915207709153076E0D7F1D4F
:1064F0009B01442737FD4095542F8091F2029091E3
:10650000F302A091F402B091F502820F931FA41F31
:10651000B51F8093F2029093F302A093F402B0931C
:10652000F5028091B6029091B702681B790BCB01FE
:10653000AA2797FDA095BA2F29853A854B855C85BA
:10654000820F931FA41FB51F8093F6029093F7024A
:10655000A093F802B093F902C0906001D09061015D
:10656000E0906201F0906301C816D906EA06FB06C6
:10657000C4F488EA91E6A0E0B0E08C199D09AE0968
:10658000BF098093F6029093F702A093F802B093AC
:10659000F9028093F2029093F302A093F402B09375
:1065A000F50222273327A9012C193D094E095F095D
:1065B0008091F6029091F702A091F802B091F90251
:1065C00082179307A407B507B4F4D701C601885A08
:1065D0009146A040B0408093F6029093F702A093BA
:1065E000F802B093F9028093F2029093F302A09321
:1065F000F402B093F5026091630770916407600F35
:10660000711F9B01442737FD4095542F8091FA025A
:106610009091FB02A091FC02B091FD02820F931FAA
:10662000A41FB51F8093FA029093FB02A093FC0273
:10663000B093FD028091B4029091B502681B790B72
:10664000CB01AA2797FDA095BA2F2D853E854F85B2
:106650005889820F931FA41FB51F8093FE02909349
:10666000FF02A0930003B0930103E0906401F09057
:1066700065010091660110916701E816F9060A07A5
:106680001B07C4F488EA91E6A0E0B0E08E199F09E8
:10669000A00BB10B8093FE029093FF02A093000326
:1066A000B09301038093FA029093FB02A093FC0243
:1066B000B093FD0222273327A9012E193F09400B71
:1066C000510B8091FE029091FF02A0910003B091C6
:1066D000010382179307A407B507B4F4D801C701D3
:1066E000885A9146A040B0408093FE029093FF02EA
:1066F000A0930003B09301038093FA029093FB02EE
:10670000A093FC02B093FD028091EE029091EF0203
:10671000A091F002B091F1028093020390930303E1
:10672000A0930403B09305038091FE029091FF02B1
:10673000A0910003B091010380931E0390931F0367
:10674000A0932003B09321038091F6029091F70269
:10675000A091F802B091F902809316039093170369
:10676000A0931803B09319038091FA029091FB0251
:10677000A091FC02B091FD0280931A0390931B0339
:10678000A0931C03B0931D038091F2029091F30239
:10679000A091F402B091F502809312039093130339
:1067A000A0931403B093150380911B0190911C01D9
:1067B00097FD079633E0959587953A95E1F7909385
:1067C0006407809363078091190190911A0197FDE6
:1067D000079623E0959587952A95E1F790935307BF
:1067E000809352078091F8019091F9010F9734F44A
:1067F00088E19CEF90936407809363078091F80190
:106800009091F901079734F480E398EF909364072F
:1068100080936307209102012A30A9F48091F80146
:106820009091F901835F934034F088EE93E0909368
:106830006407809363078091F8019091F9018A5F62
:106840009340DCF014C08091F8019091F901815DD2
:10685000974034F088EE93E0909364078093630749
:106860008091F8019091F901805E974034F080EDBD
:1068700097E090936407809363078091F60190916D
:10688000F7010F9734F488E19CEF909353078093BE
:1068900052078091F6019091F701079734F480E355
:1068A00098EF90935307809352072A30A9F4809170
:1068B000F6019091F701835F934034F088EE93E006
:1068C00090935307809352078091F6019091F701BE
:1068D0008A5F9340DCF014C08091F6019091F7013B
:1068E000815D974034F088EE93E090935307809356
:1068F00052078091F6019091F701805E974034F045
:1069000080ED97E09093530780935207E0915701F1
:10691000EE2309F4B7C040911B0150911C018091F6
:106920004A0390914B03481B590B509351034093DA
:10693000500320911B0130911C01280F391F37FF94
:1069400002C02F5F3F4F3595279530934B0320931F
:106950004A03413851051CF080E890E005C04058DA
:106960005F4F34F480E89FEF90935103809350037E
:106970008E2F9927A0915003B0915103A89FA00199
:10698000A99F500DB89F500D112457FF02C0415FC1
:106990005F4F14E0559547951A95E1F7809163078D
:1069A00090916407840F951F909364078093630709
:1069B0006091190170911A0180914C0390914D03DF
:1069C000681B790B70934F0360934E03409119013C
:1069D00050911A01480F591F57FF02C04F5F5F4F78
:1069E0005595479550934D0340934C03613871057D
:1069F0001CF080E890E005C060587F4F34F480E8D8
:106A00009FEF90934F0380934E032E2F3327809157
:106A10004E0390914F03829FB001839F700D929F10
:106A2000700D1124AB0177FF02C0415F5F4FE4E0BE
:106A300055954795EA95E1F7809152079091530754
:106A4000840F951F9093530780935207A29FC00114
:106A5000A39F900DB29F900D11249C0180911B016A
:106A600090911C01820F931F90931C0180931B0136
:106A70008091190190911A01860F971F90931A0126
:106A80008093190100916707109168078091490769
:106A900090914A07101611065CF59C0197FF04C0FF
:106AA00022273327281B390BC901AA2797FDA09558
:106AB000BA2F20914B01332744275527BC01CD0124
:106AC0000E949F799B01AC0197FF04C0215C3F4F5E
:106AD0004F4F5F4F76E055954795379527957A95B7
:106AE000D1F78091610790916207820F931F27C0B1
:106AF00097FF03C0909581959F4FAA2797FDA0957A
:106B0000BA2F20914B01332744275527BC01CD01D3
:106B10000E949F799B01AC0197FF04C0215C3F4F0D
:106B20004F4F5F4F66E055954795379527956A9586
:106B3000D1F78091610790916207821B930B90932C
:106B4000620780936107E0906F07F0907007809173
:106B50004D0790914E071E141F045CF59C0197FF92
:106B600004C022273327281B390BC901AA2797FD08
:106B7000A095BA2F20914B01332744275527BC01FC
:106B8000CD010E949F799B01AC0197FF04C0215C5D
:106B90003F4F4F4F5F4F96E0559547953795279557
:106BA0009A95D1F78091550790915607820F931FC0
:106BB00027C097FF03C0909581959F4FAA2797FD07
:106BC000A095BA2F20914B01332744275527BC01AC
:106BD000CD010E949F799B01AC0197FF04C0215C0D
:106BE0003F4F4F4F5F4F86E0559547953795279517
:106BF0008A95D1F78091550790915607821B930B88
:106C000090935607809355078091C60587FF44C02F
:106C10009989992309F040C08091B0028823E1F559
:106C2000A1E0EA16A1E0FA064CF08091630790918A
:106C300064078E0D9F1D805091400DC0B0E0EB1693
:106C4000BFEFFB0664F480916307909164078E0D9B
:106C50009F1D80509F4F9093640780936307E1E0EE
:106C600001301E074CF08091520790915307800F1E
:106C7000911F805091400CC0FFEF00301F0764F45B
:106C80008091520790915307800F911F80509F4F22
:106C90009093530780935207ABECB2E06EEB75E034
:106CA00057E0FB018191BF01E82FFF27EE0FFF1F87
:106CB000EF51F94F0190F081E02DE259FF4FEF3F86
:106CC000F10521F01CF0EFEFF0E004C0F7FF02C087
:106CD000E0E0F0E04C91242F3327E217F307B1F006
:106CE000CF01821B930B97FD079613E0959587952F
:106CF0001A95E1F7242F280F2C93822F9927E81754
:106D0000F90714F4215001C02F5F2C9351501196B4
:106D100057FFC7CFE2E1CD5E0C944A7A8091C10261
:106D2000882301F5809196028C7F80939602ABEFC9
:106D3000B3E0E0E8F6E09BE08091B401882309F439
:106D40008C938D91818312829150389697FFF4CF66
:106D50008091B401882359F08091B40181508093CF
:106D6000B40105C0809196028160809396021092D2
:106D70001D0210921F0280911A028E7F80931A02C8
:106D800085EA8093BC0008958091C805883F38F05B
:106D9000EFEFF0E0E81BF109E553FD4F80818093B0
:106DA0005D0180915D01882329F0843618F084E626
:106DB00080935D018091CA05883F38F0EFEFF0E0E5
:106DC000E81BF109E553FD4F808180935B018091C1
:106DD0005B01882329F0843618F084E680935B01F8
:106DE0008091D705883F38F0EFEFF0E0E81BF1091C
:106DF000E553FD4F808180935601809156018B3081
:106E000010F48AE002C08F3F11F480935601809104
:106E10000206883F38F0EFEFF0E0E81BF109E55398
:106E2000FD4F808180937D0780917D07823010F433
:106E300081E002C08F3F11F480937D0780910406AA
:106E4000883F38F0EFEFF0E0E81BF109E553FD4F24
:106E500080818093A9078091A907823010F481E096
:106E600002C08F3F11F48093A9078091EF05883FFE
:106E700038F0EFEFF0E0E81BF109E553FD4F8081BA
:106E8000809378078091F005883F38F0EFEFF0E0CD
:106E9000E81BF109E553FD4F808180934F078091F6
:106EA000F105883F38F0EFEFF0E0E81BF109E5531A
:106EB000FD4F8081809383079091C905983F18F416
:106EC00090935C0109C0EFEFF0E0E91BF109E55395
:106ED000FD4F808180935C01983F18F490935C0192
:106EE00009C0EFEFF0E0E91BF109E553FD4F8081A8
:106EF00080935C018091CC05883F38F0EFEFF0E0A3
:106F0000E81BF109E553FD4F808180935A01809180
:106F1000CE05883F38F0EFEFF0E0E81BF109E553CC
:106F2000FD4F8081809358018091D605883F38F0CD
:106F3000EFEFF0E0E81BF109E553FD4F808180930E
:106F400059018091D805883F38F0EFEFF0E0E81B59
:106F5000F109E553FD4F8081809355018091D9055A
:106F6000883F38F0EFEFF0E0E81BF109E553FD4F03
:106F70008081809357018091DA05883F38F0EFEFE8
:106F8000F0E0E81BF109E553FD4F80818093540147
:106F90008091DB05883F38F0EFEFF0E0E81BF10966
:106FA000E553FD4F8081809353018091E105883F37
:106FB00038F0EFEFF0E0E81BF109E553FD4F808179
:106FC000809351018091E205883F38F0EFEFF0E0C7
:106FD000E81BF109E553FD4F80818093AB0280915E
:106FE000E305883F38F0EFEFF0E0E81BF109E553E7
:106FF000FD4F80818093AA028091E405883F38F09C
:10700000EFEFF0E0E81BF109E553FD4F808180933D
:10701000A9028091E505883F38F0EFEFF0E0E81B2A
:10702000F109E553FD4F80818093A8028091FD0511
:10703000883F38F0EFEFF0E0E81BF109E553FD4F32
:1070400080818093A7028091FE05883F38F0EFEFA2
:10705000F0E0E81BF109E553FD4F80818093A60223
:107060008091FF05883F38F0EFEFF0E0E81BF10971
:10707000E553FD4F80818093A50280910006883FF3
:1070800038F0EFEFF0E0E81BF109E553FD4F8081A8
:107090008093A4028091E605883F38F0EFEFF0E09E
:1070A000E81BF109E553FD4F8081809350018091E9
:1070B000EA05883F38F0EFEFF0E0E81BF109E5530F
:1070C000FD4F808180934F018091F205883F38F019
:1070D000EFEFF0E0E81BF109E553FD4F808180936D
:1070E0004E018091F505883F38F0EFEFF0E0E81BA6
:1070F000F109E553FD4F808180934D018091F605A4
:10710000883F38F0EFEFF0E0E81BF109E553FD4F61
:10711000808180934C018091F705883F38F0EFEF34
:10712000F0E0E81BF109E553FD4F808180934B01AE
:107130008091FC05883F38F0EFEFF0E0E81BF109A3
:10714000E553FD4F808180934A0180911706883F67
:1071500038F0EFEFF0E0E81BF109E553FD4F8081D7
:107160008093BB0780915101282F33272F5F3F4F1A
:107170008CE398E2B9010E94DE7970935F0160931D
:107180005E018091D4058093AA078091D3058093F6
:10719000690790911906933320F181E08093A3024F
:1071A000983F58F0EFEFF0E0E91BF109E553FD4F90
:1071B0008081823310F41092A3028091FA0790919B
:1071C000FB0797FF08C08091A302882321F08091DC
:1071D000F603806803C08091F6038F778093F603EF
:1071E00002C01092A3028091FA079091FB0797FFCB
:1071F0001DC08091C1028823C9F08091A302882319
:10720000A9F080910801909109018F5F9F4F71F45F
:1072100088E99AE39093D4018093D30180E094EAC3
:1072200090930901809308011092A3028091A30218
:10723000882339F080914D01823D18F4825E80935D
:107240004D010895A5E3B0E0E8E2F9E30C942E7A4D
:107250000E94962E309102013C3010F4299A01C010
:107260002998E090C202F090C302F9A2E8A28091AE
:10727000690799270A96E816F90614F499A388A3D2
:107280008091CA02843608F05CC0809166039091B8
:107290006703009731F0019790936703809366032B
:1072A00007C01092C102809196028F7E8093960251
:1072B0003A3011F0343110F0289A01C028988091AA
:1072C000970290919802895E9340C0F18091DE050B
:1072D000282F332739A328A38091960280618093B9
:1072E00096028091BA05A82FBB27AA0FBB1FFD01EC
:1072F000EB5EF84F118210828091BB05282F332757
:10730000220F331FC9018B5E984FFC01118210823E
:10731000AF51B94F11961C921E922F51394FD9017E
:1073200011961C921E928091BD05E82FFF27EE0F4B
:10733000FF1FEF51F94F11821082AAC21092C102B1
:10734000A7C28091CA028D3808F4A2C28091960229
:107350008F7E809396029091DF0582E3989FC00113
:1073600011249093670380936603E8A1F9A1B9976C
:107370008CF08091C102882369F0809197029091EE
:107380009802FFEF8F3F9F0729F001969093980294
:107390008093970280919702909198028F3F910578
:1073A00009F038F51092E6021092E7021092E80216
:1073B0001092E9021092E2021092E3021092E402AB
:1073C0001092E5021092520310925303109254034C
:1073D000109255031092EE021092EF021092F002FA
:1073E0001092F1028A3F910549F481E080936C0389
:1073F00005C0809196028260809396028091BC05C0
:10740000E82FFF27EE0FFF1FEF51F94F8081918189
:10741000813591050CF441C12091C102222309F06C
:107420003CC18091BD05E82FFF27EE0FFF1FEF51F4
:10743000F94F808191818C3491050CF406C18091C3
:1074400068038F5F80936803893C08F426C13C3051
:1074500010F4299801C0299A1092C1021092680371
:1074600010929802109297023091BA05E32FFF27ED
:10747000EE0FFF1FEF51F94F808191818734910505
:10748000B4F48091BB05E82FFF27EE0FFF1FEF51EB
:10749000F94F808191810190F081E02DF7FF03C0C9
:1074A000F095E195FF4FE734F1050CF478C041E029
:1074B0002091BB05A22FBB27AA0FBB1FAF51B94F0D
:1074C0008D919C9111978734910544F0E32FFF270C
:1074D000EE0FFF1FEF51F94F808191818D919C91AB
:1074E0008734910574F08091BA05E82FFF27EE0FDD
:1074F000FF1FEF51F94F80819181873491050CF086
:1075000042E0E22FFF27EE0FFF1FEF51F94F80817E
:1075100091818634910574F48091BA05E82FFF2794
:10752000EE0FFF1FEF51F94F808191818734910554
:107530000CF043E0E22FFF27EE0FFF1FEF51F94F52
:10754000808191818A5B9F4F74F48091BA05E82F06
:10755000FF27EE0FFF1FEF51F94F80819181873494
:1075600091050CF044E0E22FFF27EE0FFF1FEF51D3
:10757000F94F808191818A5B9F4F74F48091BA05A5
:10758000E82FFF27EE0FFF1FEF51F94F8081918108
:10759000863491050CF445E0842F0E94FF208091F1
:1075A000BB05E82FFF27EE0FFF1FEF51F94F80813A
:1075B00091810190F081E02DF7FF03C0F095E195F6
:1075C000FF4F7E97BCF48091BA05E82FFF27EE0F9E
:1075D000FF1FEF51F94F808191818A5B9F4F54F4D7
:1075E00081E08093110488EE93E09093D40180931E
:1075F000D30153C00E94D5210E94C82080E00E9480
:10760000C8058091E0050E942D778091C60580FF16
:1076100010C08091130190911401875B934038F45E
:1076200080911301909114018E5E924010F40E949B
:1076300061181092D10180E00E94E82B81E08093D4
:107640006B038093D101579A1FC080819181855B24
:107650009F4F0CF5809168038F5F80936803893C8E
:10766000E0F03C3010F4299801C0299A1092C10230
:1076700010926803109298021092970281E00E9483
:10768000E82B81E080936B030E94D52168E770E0CE
:107690000E94262B02C0209368038091BC05E82F2E
:1076A000FF27EE0FFF1FEF51F94F808191818B5A19
:1076B0009F4F0CF0EDC02091C102E091BD05222347
:1076C00009F0CAC0FF27EE0FFF1FEF51F94F80816D
:1076D0009181855B9F4F0CF0BCC0809169038F5FE7
:1076E00080936903893C08F4D3C020936903809197
:1076F000F603882309F0A6C080916B03882309F460
:10770000A1C081E090E0909398028093970281E07D
:107710008093C102109252031092530310925403AB
:10772000109255031092EE021092EF021092F002A6
:107730001092F1021092EA021092EB021092EC0207
:107740001092ED028091D505E82EFF240027112725
:107750008091A6079091A7079C01442737FD40958B
:10776000542FC801B7010E949F79DC01CB0180939F
:10777000FE029093FF02A0930003B0930103809157
:10778000B8079091B9079C01442737FD4095542FC5
:10779000C801B7010E949F79DC01CB018093F602FA
:1077A0009093F702A093F802B093F90280911E0320
:1077B00090911F03A0912003B09121038093FA02BE
:1077C0009093FB02A093FC02B093FD0280911603FC
:1077D00090911703A0911803B09119038093F202BE
:1077E0009093F302A093F402B093F5021092E60294
:1077F0001092E7021092E8021092E9021092E2025F
:107800001092E3021092E4021092E5028091960237
:10781000886080939602909118068FE0989F90015F
:1078200011248091DC029091DD02820F931F68E6A3
:1078300071E00E94DE7997FD01969595879580937A
:10784000220326C08CED95E09093D4018093D30160
:107850001FC0209369031CC0FF27EE0FFF1FEF51CD
:10786000F94F808191818C34910584F080916A0375
:107870008F5F80936A03893C58F01092C102109286
:107880006A03109298021092970202C010926A0343
:1078900080914201815080934201809142018F3F4B
:1078A00021F08091960284FF82C30E94C4368091A9
:1078B0007503909176039C01220F331F280F391F07
:1078C000A090BA05AA2DBB27AA0FBB1FFD01EF513F
:1078D000F94F9090D005492D552780819181849F43
:1078E000F001859FF00D949FF00D11242E0F3F1F86
:1078F00037FF02C02D5F3F4FB901759567957595AC
:107900006795AB5EB84F8091D105082F11278D91F7
:107910009C91809F7001819FF00C909FF00C11242E
:107920006E0D7F1D709376036093750380917703CE
:10793000909178039C01220F331F280F391FB090BC
:10794000BB05AB2DBB27AA0FBB1FFD01EF51F94FA4
:1079500080819181849FF001859FF00D949FF00DAF
:1079600011242E0F3F1F37FF02C02D5F3F4FA9018B
:107970005595479555954795AB5EB84F8D919C9120
:10798000809F7001819FF00C909FF00C11244E0D90
:107990005F1D50937803409377039E012F5F3F4F05
:1079A0008FE1E3E7F1E0D90101900D928A95E1F7CB
:1079B0008091A302882309F448C0CB0177FD039688
:1079C000DC01B595A795B595A795CA0157FD039616
:1079D000FC01F595E795F595E79580919C01682F59
:1079E000772767FD70956A9F90016B9F300D7A9F96
:1079F000300D11248091AE03482F552747FD509537
:107A00004E9FC0014F9F900D5E9F900D1124280F37
:107A1000391F37FF02C0295F3F4F03E03595279597
:107A20000A95E1F73093C9022093C8026E9F900136
:107A30006F9F300D7E9F300D11244A9FC0014B9FD8
:107A4000900D5A9F900D112444C080911806082F64
:107A50001127DE01A00FB11FFD01978190939C01BA
:107A6000020F131FD8018C918093AE03A92FBB275F
:107A7000A7FDB095A69F9001A79F300DB69F300D32
:107A80001124E82FFF27E7FDF095E49FC001E59F53
:107A9000900DF49F900D1124280F391F37FF02C05D
:107AA000295F3F4F13E0359527951A95E1F73093FD
:107AB000C9022093C802A49F9001A59F300DB49FD6
:107AC000300D1124E69FC001E79F900DF69F900DA9
:107AD0001124281B390B37FF02C0295F3F4FF3E009
:107AE00035952795FA95E1F73093C7022093C602A2
:107AF0008091BD05E82FFF27EE0FFF1FEF51F94FD3
:107B000080819181909581959F4F9093C50280933C
:107B1000C4028330910514F0029705C0BFEF8E3F79
:107B20009B0734F402969093C5028093C40204C06C
:107B30001092C5021092C4028091AA039091AB03E7
:107B40002091A6033091A703820F931FC090C80213
:107B5000D090C902C81AD90AD092C902C092C802EC
:107B60008091A8039091A9032091A4033091A503CB
:107B7000820F931F0091C6021091C702081B190BB8
:107B80001093C7020093C6028091BC05E82FFF271F
:107B9000EE0FFF1FEF51F94FE080F180E8E7F0E0D2
:107BA000EE0EFF1EF092C302E092C20280915601D7
:107BB0009927AA2797FDA095BA2FBC01CD010E9455
:107BC0004779DC01CB0120E030E040E251E4BC0128
:107BD000CD010E94E878DC01CB01BC01CD010E94FF
:107BE0002A79DC01CB018093B20780915501809303
:107BF0008507809154019927AA2797FDA095BA2F50
:107C0000BC01CD010E944779DC01CB0120E030E0CE
:107C100040E251E4BC01CD010E94E878DC01CB01D7
:107C2000BC01CD010E942A79DC01CB0180935B0766
:107C3000809153018093710780911D0480FF59C08A
:107C40008091BB07813808F454C0809116049927AD
:107C500087FD9095292D3327829FA001839F500D8A
:107C6000929F500D1124C40ED51ED092C902C0920D
:107C7000C80280911704992787FD9095829FB001D3
:107C8000839F700D929F700D1124060F171F109384
:107C9000C7020093C60280911804282F332727FDBE
:107CA00030958091C4029091C502820F931F9093EA
:107CB000C5028093C40280911A04282F332727FD20
:107CC00030958091CB059927289FD001299FB00D31
:107CD000389FB00D1124B0934901A09348018091C1
:107CE000190499278E159F0524F49093C30280935D
:107CF000C2028091C2029091C30297FF04C0109209
:107D0000C3021092C2028091C60582FF02C0109287
:107D100085074091C8025091C902CA0157FD0396D8
:107D20009C01359527953595279537FF03C03095EC
:107D300021953F4F80919B0290919C02821793075F
:107D4000B4F4CA0157FF03C0909581959F4F97FDEA
:107D50000396959587959595879590939C0280932A
:107D60009B028536910544F084E690E001C00197BE
:107D700090939C0280939B024091C6025091C7024F
:107D8000CA0157FD03969C01359527953595279592
:107D900037FF03C0309521953F4F80919902909114
:107DA0009A0282179307B4F4CA0157FF03C0909553
:107DB00081959F4F97FD0396959587959595879506
:107DC00090939A02809399028536910544F084E657
:107DD00090E001C0019790939A028093990280915C
:107DE000960284FF08C010929C0210929B0210928F
:107DF0009A0210929902EB2DFF27EE0FFF1FEF5111
:107E0000F94F4091F305242F332780819181281762
:107E1000390744F480911A0682FF04C081E0809300
:107E2000AF0213C0EB2DFF27EE0FFF1FEF51F94FED
:107E3000842F99272091F405821B9109208131819B
:107E40002817390714F41092AF024091BB05E42FB4
:107E5000FF27EE0FFF1FEF51F94F5091F305852FCC
:107E6000992722273327281B390B8081918182177C
:107E7000930744F480911A0683FF04C081E0809345
:107E8000AE0216C08091AE02882391F0E42FFF2746
:107E9000EE0FFF1FEF51F94F8091F4059927851BD5
:107EA0009109208131818217930714F41092AE0258
:107EB000EA2DFF27EE0FFF1FEF51F94F4091F30519
:107EC000242F3327808191812817390744F480912A
:107ED0001A0680FF04C081E08093AC0217C0809135
:107EE000AC02882399F0EA2DFF27EE0FFF1FEF5118
:107EF000F94F842F99272091F405821B9109208145
:107F000031812817390714F41092AC024091BA0558
:107F1000E42FFF27EE0FFF1FEF51F94F5091F305AC
:107F2000852F992722273327281B390B80819181A0
:107F30008217930744F480911A0681FF04C081E000
:107F40008093AD0216C08091AD02882391F0E42F9A
:107F5000FF27EE0FFF1FEF51F94F8091F40599278E
:107F6000851B9109208131818217930714F41092A7
:107F7000AD028091AF02882319F48091AE02811185
:107F800081E08093B0028091AC02882321F480913B
:107F9000AD02882351F081E08093B1021092B002CB
:107FA0001092AF021092AE0202C08093B102809193
:107FB000B002882321F48091B102882369F0809176
:107FC000F2059927E8A1F9A18E179F0714F499A348
:107FD00088A381E08093D6028091960284FF1AC024
:107FE0001092C5021092C4021092C9021092C802E7
:107FF0001092C7021092C6029AE59093B20788E7E2
:108000008093850790935B07809371071092B0026D
:108010001092B1028091740790917507A091760734
:10802000B091770720911E0330911F0340912003E8
:1080300050912103820F931FA41FB51F80937407D3
:1080400090937507A0937607B093770780917E078A
:1080500090917F07A0918007B0918107209016032F
:10806000309017034090180350901903820D931D10
:10807000A41DB51D80937E0790937F07A093800772
:10808000B093810780916B0790916C07A0916D0769
:10809000B0916E07E0901A03F0901B0300911C034F
:1080A00010911D03EAA2FBA20CA31DA38E0D9F1D20
:1080B000A01FB11F80936B0790936C07A0936D076F
:1080C000B0936E0780915C0790915D07A0915E0769
:1080D000B0915F07E0901203F09013030091140336
:1080E00010911503EEA2FFA208A719A78E0D9F1DE0
:1080F000A01FB11F80935C0790935D07A0935E075C
:10810000B0935F07F090B102FAA6FF2029F48091A6
:10811000B002882309F460C010920E0310920F037E
:10812000109210031092110310920A0310920B0385
:1081300010920C0310920D031092740710927507A1
:10814000109276071092770710927E0710927F07A1
:10815000109280071092810710926B0710926C07A3
:1081600010926D0710926E0710925C0710925D07D7
:1081700010925E0710925F078091FE029091FF02BD
:10818000A0910003B09101038093FA029093FB0247
:10819000A093FC02B093FD028091F6029091F70249
:1081A000A091F802B091F9028093F2029093F30249
:1081B000A093F402B093F5021092E5011092E4014D
:1081C0001092B5021092B4021092B7021092B60249
:1081D0000AA5002309F0F2C18091B002882309F0BA
:1081E000EDC18091AB059091AC05815092402CF48B
:1081F0008091C102882309F4E1C190902708A090E2
:10820000D5056091A6077091A7077BAB6AAB8091FB
:10821000B8079091B9079DAB8CAB9FEF991609F405
:10822000D9C0BB24CC24DD24CA01B901A601950123
:108230000E94137A79018A01EAA9FBA9CF01AA2732
:1082400097FDA095BA2FE81AF90A0A0B1B0BC20179
:10825000B101A60195010E94137A59016A012CA966
:108260003DA9C901AA2797FDA095BA2FA81AB90A56
:10827000CA0ADB0A292C332427FC3094432C532CC4
:10828000C801B701A20191010E949F7997FF04C024
:1082900061507E4F8F4F9F4F3B014C0109E09594F9
:1082A0008794779467940A95D1F7C601B501A20126
:1082B00091010E949F7997FF04C061507E4F8F4FBC
:1082C0009F4F5B016C0119E0D594C794B794A794B4
:1082D0001A95D1F780919B0290919C02813491056F
:1082E0003CF48091990290919A0281349105D4F0E6
:1082F000D401C30197FE03C00196A11DB11D3C012D
:108300004D019594879477946794D601C501D7FE63
:1083100003C00196A11DB11D5C016D01D594C794E8
:10832000B794A7948091BD05E82FFF27EE0FFF1F9C
:10833000EF51F94F808191810190F081E02DF7FF9D
:1083400003C0F095E195FF4F7A97A4F0C401B30103
:1083500023E030E040E050E00E94137A39014A0106
:10836000C601B50123E030E040E050E00E94137AFE
:1083700059016A0180912908282F332727FD30955C
:10838000432F532F261537054805590514F4390195
:108390004A01992787FD9095909581959F4FAA272F
:1083A00097FDA095BA2F681679068A069B0614F4E5
:1083B0003C014D012A153B054C055D0514F459019E
:1083C0006A01A816B906CA06DB060CF0CFC05C012C
:1083D0006D01CCC0EA2CFF2400271127CA01B90186
:1083E000A80197010E94137A39014A014AA95BA9A1
:1083F000CA01AA2797FDA095BA2F681A790A8A0A96
:108400009B0AC201B101A80197010E94137A590188
:108410006A016CA97DA9CB01AA2797FDA095BA2F67
:10842000A81AB90ACA0ADB0AD401C30197FE03C01D
:108430000F96A11DB11D3C014D01F4E09594879468
:1084400077946794FA95D1F7D601C501D7FE03C09A
:108450000F96A11DB11D5C016D01E4E0D594C79498
:10846000B794A794EA95D1F780919B0290919C02D2
:10847000813491053CF48091990290919A02813463
:108480009105A4F0C401B30123E030E040E050E0E6
:108490000E94137A39014A01C601B50123E030E098
:1084A00040E050E00E94137A59016A018091BD05B5
:1084B000E82FFF27EE0FFF1FEF51F94F80819181C9
:1084C0000190F081E02DF7FF03C0F095E195FF4F9B
:1084D0007A97A4F0C401B30123E030E040E050E01B
:1084E0000E94137A39014A01C601B50123E030E048
:1084F00040E050E00E94137A59016A0171E2671668
:108500007104810491042CF070E2672E712C812C8F
:10851000912C80EE68168FEF78068FEF88068FEF2C
:10852000980644F460EE662E6FEF762E6FEF862E7F
:108530006FEF962E91E2A916B104C104D1042CF07C
:1085400050E2A52EB12CC12CD12CA0EEAA16AFEF73
:10855000BA06AFEFCA06AFEFDA0644F440EEA42E37
:108560004FEFB42E4FEFC42E4FEFD42E8091FE026A
:108570009091FF02A0910003B09101038619970921
:10858000A809B9098093FE029093FF02A09300030B
:10859000B09301038091F6029091F702A091F80246
:1085A000B091F9028A199B09AC09BD098093F602C2
:1085B0009093F702A093F802B093F9028091E4013E
:1085C0009091E5018F3F910509F008F4C4C5BAA563
:1085D000BB2309F04EC58091B002882309F049C53C
:1085E0008091D602882309F044C5E091FB05EBA7F2
:1085F000EE2309F43EC58091740790917507A09110
:108600007607B0917707B7FF04C081509F4FAF4FF7
:10861000BF4FE92EFA2E0B2F112707FD1A95E09276
:108620007407F0927507009376071093770780918F
:108630007E0790917F07A0918007B0918107B7FFD7
:1086400004C081509F4FAF4FBF4F892F9A2FAB2F40
:10865000BB27A7FDBA958CA79DA7AEA7BFA7809300
:108660007E0790937F07A0938007B0938107809146
:10867000D505A82EBB24CC24DD2420910E033091F7
:108680000F034091100350911103C601B5010E94E0
:108690009F7997FF04C061507F4F8F4F9F4F672E88
:1086A000782E892E992487FC9A9460920E037092FA
:1086B0000F03809210039092110320910A033091CE
:1086C0000B0340910C0350910D03C601B5010E94AC
:1086D0009F7997FF04C061507F4F8F4F9F4F272E88
:1086E000382E492E552447FC5A9420920A03309282
:1086F0000B0340920C0350920D038091060390915E
:108700000703A0910803B0910903B7FF04C081508B
:108710009F4FAF4FBF4F892F9A2FAB2FBB27A7FD7E
:10872000BA958093060390930703A0930803B09330
:108730000903D801C70186199709A809B9098093C7
:108740005E0390935F03A0936003B0936103209155
:10875000FA05E22EFF2400271127BC01CD01A80154
:1087600097010E94137A59016A0120936D03309397
:108770006E0340936F03509370038CA59DA5AEA527
:10878000BFA582199309A409B50980936203909348
:108790006303A0936403B0936503BC01CD01A801FA
:1087A00097010E94137A20937103309372034093D0
:1087B000730350937403D601C501D7FE04C08150E2
:1087C0009F4FAF4FBF4F892F9A2FAB2FBB27A7FDCE
:1087D000BA959093B5028093B40257FF04C021501C
:1087E0003F4F4F4F5F4FBB2757FDBA95A52F942F93
:1087F000832F9093B7028093B60280919B02909151
:108800009C0281349105DCF48091990290919A0246
:1088100081349105A4F48091BD05E82FFF27EE0F68
:10882000FF1FEF51F94F808191810190F081E02D80
:10883000F7FF03C0F095E195FF4F7A97E4F0809140
:1088400027088F3FC1F48091B4029091B50297FD43
:108850000196959587959093B5028093B402809187
:10886000B6029091B70297FD0196959587959093E2
:10887000B7028093B60280916B0790916C07A0912C
:108880006D07B0916E07B7FF04C081509F4FAF4F87
:10889000BF4F892F9A2FAB2FBB27A7FDBA95809387
:1088A0006B0790936C07A0936D07B0936E07809150
:1088B0005C0790915D07A0915E07B0915F07B7FFDD
:1088C00004C081509F4FAF4FBF4F892F9A2FAB2FBE
:1088D000BB27A7FDBA9580935C0790935D07A09393
:1088E0005E07B0935F0780911E0390911F03A091D4
:1088F0002003B09121032AA13BA14CA15DA1281B1B
:10890000390B4A0B5B0B209356033093570340936C
:108910005803509359038091160390911703A09127
:108920001803B0911903EEA0FFA008A519A5E81A35
:10893000F90A0A0B1B0BE0925A03F0925B030093B7
:108940005C0310935D0320935E0330935F034093B9
:10895000600350936103E0926203F092630300931B
:108960006403109365038091FA029091FB02A09139
:10897000FC02B091FD02821B930BA40BB50B8093FC
:10898000FA029093FB02A093FC02B093FD02809147
:10899000F2029091F302A091F402B091F5028E19C7
:1089A0009F09A00BB10B8093F2029093F302A09366
:1089B000F402B093F502FBA5FF23E1F02091D4026D
:1089C0003091D502213831054CF080912F039091E0
:1089D000300301969093300380932F0320583F4F2C
:1089E0004CF480912F0390913003019790933003C2
:1089F00080932F031092D5021092D40281E090E070
:108A000090937A0380937903A0905E03B0905F0304
:108A1000C0906003D0906103D601C501D7FE07C0A6
:108A200088279927DC018A199B09AC09BD09815067
:108A30009240A040B04034F084E090E090937A03FC
:108A40008093790380917F0390918003A0918103AB
:108A5000B091820320917407309175074091760799
:108A600050917707821B930BA40BB50B815E914B42
:108A7000AF4FBF4F8F539C49A040B04028F080912A
:108A8000280889310CF4FFC031E0A31630E1B306A9
:108A900030E0C30630E0D3060CF473C080917B0352
:108AA000882309F46AC0D601C501D7FE07C088270C
:108AB0009927DC018A199B09AC09BD099C01AD010C
:108AC000B7FF04C021503E4F4F4F5F4FF9E055951F
:108AD000479537952795FA95D1F78091790390912D
:108AE0007A03820F931F90937A0380937903D601C0
:108AF000C501D7FE03C00796A11DB11DE3E0B595E2
:108B0000A79597958795EA95D1F780936D039093F4
:108B10006E03A0936F03B093700389589341A040F4
:108B2000B04064F088E893E1A0E0B0E080936D038A
:108B300090936E03A0936F03B093700320916D0325
:108B400030916E0340916F035091700357FF04C042
:108B500021503F4F4F4F5F4F232F342F452F552725
:108B600047FD5A958091B4029091B502820F931FF0
:108B70009093B5028093B40206C081E080937B039A
:108B800002C010927B0350E0A51650EFB5065FEFD0
:108B9000C5065FEFD5060CF073C080917C03882377
:108BA00009F46AC0D601C501D7FE07C088279927F6
:108BB000DC018A199B09AC09BD099C01AD01B7FF15
:108BC00004C021503E4F4F4F5F4F69E05595479588
:108BD000379527956A95D1F78091790390917A031B
:108BE000820F931F90937A0380937903D601C50176
:108BF000D7FE03C00796A11DB11D23E0B595A7952B
:108C0000979587952A95D1F780936D0390936E037E
:108C1000A0936F03B093700388579C4EAF4FBF4F24
:108C200064F488E79CEEAFEFBFEF80936D03909301
:108C30006E03A0936F03B093700320916D03309186
:108C40006E0340916F035091700357FF04C0215091
:108C50003F4F4F4F5F4F232F342F452F552747FD51
:108C60005A958091B4029091B502820F931F909310
:108C7000B5028093B40211C081E080937C030DC0E3
:108C800010927C030AC010927A031092790388EE46
:108C900093E090936901809368017BA5272F332788
:108CA0008091790390917A032817390724F430933F
:108CB0007A0320937903E0912808EE2379F02E2F90
:108CC000332727FD30958091790390917A032817F7
:108CD000390724F430937A032093790340915E039B
:108CE00050915F03609160037091610341385105B9
:108CF0006105710574F080913303909134032091E4
:108D0000790330917A03820F931F909334038093F9
:108D1000330340585F4F6F4F7F4F74F4809133039C
:108D2000909134032091790330917A03821B930B45
:108D3000909334038093330381E090E090937A031F
:108D400080937903A0906203B0906303C0906403A2
:108D5000D0906503D601C501D7FE07C088279927A3
:108D6000DC018A199B09AC09BD0981509240A040E1
:108D7000B04034F084E090E090937A0380937903DC
:108D80008091830390918403A0918503B091860321
:108D900020917E0730917F07409180075091810795
:108DA000821B930BA40BB50B815E914BAF4FBF4F52
:108DB0008F539C49A040B04018F0E9310CF4FFC03B
:108DC00011E0A11610E1B10610E0C10610E0D106D5
:108DD0000CF473C080917D03882309F46AC0D60126
:108DE000C501D7FE07C088279927DC018A199B098E
:108DF000AC09BD099C01AD01B7FF04C021503E4F35
:108E00004F4F5F4F09E055954795379527950A9540
:108E1000D1F78091790390917A03820F931F9093F9
:108E20007A0380937903D601C501D7FE03C0079664
:108E3000A11DB11D13E0B595A795979587951A9536
:108E4000D1F78093710390937203A0937303B0934F
:108E5000740389589341A040B04064F088E893E1DE
:108E6000A0E0B0E08093710390937203A09373032A
:108E7000B093740320917103309172034091730396
:108E80005091740357FF04C021503F4F4F4F5F4F25
:108E9000232F342F452F552747FD5A958091B60231
:108EA0009091B702820F931F9093B7028093B602FE
:108EB00006C081E080937D0302C010927D0330E004
:108EC000A31630EFB3063FEFC3063FEFD3060CF017
:108ED00073C080917E03882309F46AC0D601C5015E
:108EE000D7FE07C088279927DC018A199B09AC099E
:108EF000BD099C01AD01B7FF04C021503E4F4F4F4B
:108F00005F4FE9E05595479537952795EA95D1F755
:108F10008091790390917A03820F931F90937A0343
:108F200080937903D601C501D7FE03C00796A11D22
:108F3000B11D73E0B595A795979587957A95D1F76B
:108F40008093710390937203A0937303B09374039F
:108F500088579C4EAF4FBF4F64F488E79CEEAFEF4D
:108F6000BFEF8093710390937203A0937303B09348
:108F700074032091710330917203409173035091F7
:108F8000740357FF04C021503F4F4F4F5F4F232FB3
:108F9000342F452F552747FD5A958091B602909161
:108FA000B702820F931F9093B7028093B60211C04D
:108FB00081E080937E030DC010927E030AC0109260
:108FC0007A031092790388EE93E09093690180937D
:108FD00068015BA5252F33278091790390917A034F
:108FE0002817390724F430937A032093790380916A
:108FF0002808882379F0282F332727FD3095809182
:10900000790390917A032817390724F430937A036F
:10901000209379034091620350916303609164034C
:1090200070916503413851056105710574F08091B7
:109030003103909132032091790330917A03820FAA
:10904000931F909332038093310340585F4F6F4FCB
:109050007F4FCCF4809131039091320320917903BA
:1090600030917A03821B930B9093320380933103E8
:109070000AC01092B7021092B6021092B502109276
:10908000B4021092D60280918507882341F4109291
:10909000B7021092B6021092B5021092B4028091FB
:1090A000740790917507A0917607B0917707809328
:1090B0007F0390938003A0938103B09382038091F8
:1090C0007E0790917F07A0918007B09181078093E0
:1090D000830390938403A0938503B0938603109237
:1090E0000E0310920F0310921003109211031092AE
:1090F0000A0310920B0310920C0310920D031092AE
:1091000006031092070310920803109209031092AD
:1091100074071092750710927607109277071092D5
:109120007E0710927F07109280071092810710929D
:109130006B0710926C0710926D0710926E071092D9
:109140005C0710925D0710925E0710925F07109205
:10915000E5011092E4010091C4021091C502C8011A
:1091600017FF04C088279927801B910B40976CF04C
:1091700088EE93E090936901809368018091C60521
:1091800084FD03C081E080936C03F090D205AF2C86
:10919000BB24CC24DD24B801882777FD8095982F47
:1091A000980117FF04C022273327201B310B4427C7
:1091B00037FD4095542F0E949F799B01AC01C60159
:1091C000B5010E949F7997FF04C061507E4F8F4F79
:1091D0009F4F59E095958795779567955A95D1F763
:1091E0009B018F2D9927809FD001819FB00D909F6B
:1091F000B00D1124CD01B7FD0396959587959595F2
:109200008795280F391F442737FD4095542F209309
:10921000520330935303409354035093550380916A
:10922000EE029091EF02A091F002B091F102821B48
:10923000930BA40BB50B8093EE029093EF02A093D7
:10924000F002B093F1028155934CA040B04064F01D
:1092500080E593ECA0E0B0E08093EE029093EF0203
:10926000A093F002B093F1028091EE029091EF0290
:10927000A091F002B091F102805B9C43AF4FBF4FD1
:1092800064F480EB9CE3AFEFBFEF8093EE0290932A
:10929000EF02A093F002B093F102A090DC02B09034
:1092A000DD02A114B10409F478C18091C60583FFE1
:1092B00074C180911E0390911F03A0912003B0916F
:1092C0002103B7FF04C081509E4FAF4FBF4F29E02D
:1092D000B595A795979587952A95D1F76C0197FF36
:1092E00004C0D094C194D108D39480911603909176
:1092F0001703A0911803B0911903B7FF04C0815060
:109300009E4FAF4FBF4F09E0B595A79597958795AD
:109310000A95D1F7BC0197FF03C0709561957F4F07
:10932000C616D7060CF46B01B601D7FE02C0695F02
:109330007F4F2B0113E0559447941A95E1F7B2E063
:10934000EB2EF12C4E0C5F1C0CE112E0A00EB11EB6
:1093500075010027F7FC0095102F24EE3DEFA20EBB
:10936000B31E8091B4079091B507A091B607B09154
:10937000B70760904401709045018090460190903D
:109380004701BC01CD01A40193010E94137AE21AA6
:10939000F30A040B150BC801B70128E631E040E0E1
:1093A00050E00E94137ADC01CB01ACE4EA2EAFEF6F
:1093B000FA2EE80EF91E009168011091690101155D
:1093C000110589F539E1C316D1046CF58091D402F9
:1093D0009091D5028E0D9F1D9093D5028093D4025B
:1093E00080916C038823F9F0C501AA2797FDA09509
:1093F000BA2FBC01CD01A40193010E949F79DC0129
:10940000CB018093B4079093B507A093B607B093B0
:10941000B707BC01CD010E94137A3093DB02209381
:10942000DA0210926C03C701F4E0880F991FFA95D5
:10943000E1F7B2010E94DE79CB01AA2797FDA09542
:10944000BA2F2091B4073091B5074091B6075091DB
:10945000B707280F391F4A1F5B1F2093B4073093AB
:10946000B5074093B6075093B707F09059016F2D99
:109470007727C69EC001C79E900DD69E900D1124E1
:1094800097FD4F966C01E5E0D594C794EA95E1F716
:109490006C197D096B0177FD7AC00115110509F082
:1094A0006FC000919B0210919C0280919902909153
:1094B0009A02080F191F17FF02C0095F1F4F73E0C0
:1094C000159507957A95E1F7005C1F4FCA01B90120
:1094D000A40193010E94137ADA01C9012091DA02F2
:1094E0003091DB02442737FD4095542F821B930BAC
:1094F000A40BB50B845E9D4FAF4FBF4FBC01CD0198
:1095000028E631E040E050E00E94137ADC01CB0114
:10951000845B90408C9DA0018D9D500D9C9D500DB5
:109520001124CA01B8010E94DE7983E0F89E60012F
:109530001124C616D70614F4B60108C08827992747
:109540008C199D09681779070CF4BC019B0144270D
:1095500037FD4095542F8091EE029091EF02A0913B
:10956000F002B091F102820F931FA41FB51F8093E8
:10957000EE029093EF02A093F002B093F1020DC0BF
:1095800001501040109369010093680106C084EFF8
:1095900091E090936901809368018091D6028823BD
:1095A00081F01092E2021092E3021092E402109213
:1095B000E5021092E6021092E7021092E802109281
:1095C000E9027090B1027720F1F480918507282F8D
:1095D00033274427552780911E0390911F03A091A4
:1095E0002003B0912103BC01CD010E949F79DC01D1
:1095F000CB01BC01CD0128EF3AE240E050E00E94EF
:10960000137A290102C0442455249090B002992075
:10961000F1F480918507282F33274427552780911F
:10962000160390911703A0911803B0911903BC0180
:10963000CD010E949F79DC01CB01BC01CD0128EF57
:109640003AE240E050E00E94137A190102C022245D
:1096500033248091550790915607893C91051CF061
:1096600088EC90E005C088539F4F34F488E39FEF67
:1096700090935607809355078091610790916207F8
:10968000893C91051CF088EC90E005C088539F4F01
:1096900034F488E39FEF9093620780936107809191
:1096A000630790916407AA2797FDA095BA2F209190
:1096B000B207A22EBB24CC24DD24BC01CD01A6011F
:1096C00095010E949F799B01AC0180915507909173
:1096D0005607AA2797FDA095BA2F67E0880F991F14
:1096E000AA1FBB1F6A95D1F7280F391F4A1F5B1F9E
:1096F00057FF04C0215C3F4F4F4F5F4F06E0559529
:109700004795379527950A95D1F77201E20EF31E1A
:10971000F0926407E092630780915207909153079B
:10972000AA2797FDA095BA2FBC01CD01A6019501EE
:109730000E949F799B01AC01809161079091620723
:10974000AA2797FDA095BA2F17E0880F991FAA1F87
:10975000BB1F1A95D1F7280F391F4A1F5B1F57FFF0
:1097600004C0215C3F4F4F4F5F4FB6E05595479582
:1097700037952795BA95D1F78101020F131F1093E2
:109780005307009352078091AD079091AE07880F61
:10979000991FAA2797FDA095BA2F20915B07332721
:1097A00044275527BC01CD010E949F795B016C01C4
:1097B00097FF08C08FE390E0A0E0B0E0A80EB91ECC
:1097C000CA1EDB1EA6E0D594C794B794A794AA95A9
:1097D000D1F780917107282F33274427552780918F
:1097E000020390910303A0910403B0910503BC010F
:1097F000CD010E949F79DC01CB01BC01CD0120EF9E
:1098000035E540E050E00E94137AB501620F731F06
:109810007093AE076093AD0791E0E91690E1F90609
:1098200034F080E090E19093640780936307809127
:109830006307909164078050904F34F480E090EF7C
:1098400090936407809363070150104134F080E0E7
:1098500090E1909353078093520780915207909123
:1098600053078050904F34F480E090EF909353076B
:10987000809352076150704134F080E090E1909302
:10988000AE078093AD078091AD079091AE078050F1
:10989000904F34F480E090EF9093AE078093AD0743
:1098A00080910001482F552780911D0190911E0144
:1098B0004817590794F420911D0130911E0168A1A9
:1098C00079A1649FC001659F900D749F900D112434
:1098D000B9010E94CA7979A368A388A199A1880FC8
:1098E000991F880F991F99A388A34091C60540FF2F
:1098F000ABC6992009F0A8C6772009F0A5C6CC24EC
:10990000DD2446018091960281FF08C08091B20259
:109910009091B30290938F0580938E05209135032B
:10992000309136032115310509F03FC080911301B4
:10993000909114018959934058F087B5853F20F4E0
:109940008091E801815011C081E0809392034EC064
:1099500080911301909114018436910508F587B523
:109960008B30D0F08091E8018F5F8093E8019AE01E
:109970008902900111248091B505821B87BD8CE27C
:1099800091E09093D4018093D3018EE591E0909380
:109990003603809335032AC081E08093910326C06B
:1099A000709291037092920321C08091BC029091B9
:1099B000BD02A091BE02B091BF02E4E0880F991FE2
:1099C000AA1FBB1FEA95D1F78093E9019093EA01A2
:1099D000A093EB01B093EC01D092E701C092E601B5
:1099E00021503040309336032093350320915C01A1
:1099F00041FF24C02233D8F48091720181508093BA
:109A000072018F3FD9F51092D7028091BC029091DC
:109A1000BD02A091BE02B091BF028093B8029093A4
:109A2000B902A093BA02B093BB0281E004C081E006
:109A30008093D70288EC8093720120C08091480106
:109A400090914901820F911D2091CB053327829F70
:109A5000F001839FF00D929FF00D1124CF01AA27F2
:109A600097FDA095BA2F8093B8029093B902A09366
:109A7000BA02B093BB0281E08093D70280911E03AB
:109A800090911F03A0912003B0912103E090440125
:109A9000F09045010091460110914701BC01CD01B4
:109AA000A80197010E94137A59016A018091160357
:109AB00090911703A0911803B0911903BC01CD0137
:109AC000A80197010E94137AB901C5010E94E570AF
:109AD0003C01CC971CF07CE3672E712CC3010E94E3
:109AE000285C3C0180E2809343018091D702882367
:109AF00009F436C48091960299279C012071307038
:109B000084FD2EC460911C0660FD04C08091C605D2
:109B100081FD07C008A119A1309388032093870312
:109B200097C18091960281FF69C140916E01509169
:109B30006F01CA010F962091C2023091C3028217B1
:109B40009307ACF580919103882389F58091930365
:109B500081FF13C08D7F809393038091BC0290910D
:109B6000BD02A091BE02B091BF028093B802909353
:109B7000B902A093BA02B093BB02809193038160B3
:109B800080939303241B350B2F50304037FF03C0C5
:109B9000309521953F4F8091870390918803820FE4
:109BA000931F90938803809387038BE26EC0CA0152
:109BB0000F9728173907ACF580919203882389F510
:109BC0008091930380FF13C08E7F809393038091D5
:109BD000BC029091BD02A091BE02B091BF028093E1
:109BE000B8029093B902A093BA02B093BB028091DD
:109BF0009303826080939303241B350B215F3F4FB7
:109C000037FF03C0309521953F4F80918703909196
:109C10008803821B930B90938803809387038DE2C4
:109C200034C020919303822F992783709070892BE1
:109C300059F12C7F2093930310928803109287038D
:109C40002091BC023091BD024091BE025091BF02F2
:109C50002093B8023093B9024093BA025093BB02EA
:109C600061FF06C084EF91E09093D4018093D3010B
:109C70008091C002882341F4233331054105510509
:109C80001CF081E08093C0028DE38093430120911A
:109C9000870330918803C90137FF04C088279927BB
:109CA000821B930B815092400CF491C08091CB05A4
:109CB0009927289FA001299F500D389F500D1124EE
:109CC000CA0160E075E00E94DE79CB01AA2797FD0A
:109CD000A095BA2F2091B8023091B9024091BA02F2
:109CE0005091BB02280F391F4A1F5B1F2093B802F7
:109CF0003093B9024093BA025093BB02109288038A
:109D000010928703A090BC02B090BD02C090BE022A
:109D1000D090BF02D601C50180509440A040B04011
:109D200082179307A407B5075CF4D601C5018050DC
:109D30009C4FAF4FBF4F281739074A075B0744F0C6
:109D40008093B8029093B902A093BA02B093BB0279
:109D500080911C0681FF06C084E690E09093D401B8
:109D60008093D3018091CF05882389F54091B20279
:109D70005091B30257FF02C04D5F5F4F5595479515
:109D80005595479580911D0190911E0120910001EC
:109D90003327489FB001499F700D589F700D1124C3
:109DA000CB01B9010E94DE7970936F0160936E015F
:109DB000663471051CF486E490E005C067397105CE
:109DC00034F086E990E090936F0180936E0180916A
:109DD000350390913603892BB9F18091BC029091A3
:109DE000BD02A091BE02B091BF028093B8029093D1
:109DF000B902A093BA02B093BB0226C08091BC0204
:109E00009091BD02A091BE02B091BF0280599140D5
:109E1000A040B0408093B8029093B902A093BA02D8
:109E2000B093BB028091CF05882311F0992702C01F
:109E300088E790E090936F0180936E0188A199A1CB
:109E40009093B3028093B2020091B2021091B302D8
:109E5000A090BC02B090BD02C090BE02D090BF02E4
:109E60002091B8023091B9024091BA025091BB02E0
:109E70002A153B054C055D0524F080911C0680FDEC
:109E8000B1C28091350390913603892B39F000914E
:109E9000B2021091B302CC24DD24D7C0D601C50193
:109EA000821B930BA40BB50B80935603909357031F
:109EB000A0935803B09359038230E0E89E07EFEF78
:109EC000AE07EFEFBE072CF481E090E8AFEFBFEFF5
:109ED00009C08F5F9F47A040B04064F08FEF9FE7BD
:109EE000A0E0B0E08093560390935703A0935803EB
:109EF000B0935903C0905603D090570380915B01F3
:109F0000282F3327442755278091560390915703D4
:109F1000A0915803B0915903BC01CD010E949F79D3
:109F200097FF04C0615E7F4F8F4F9F4F55E095951F
:109F30008795779567955A95D1F7609356037093F7
:109F40005703809358039093590365302EEF72079F
:109F50002FEF82072FEF92072CF484E09EEFAFEFF4
:109F6000BFEF09C0605074408040904064F080E0D2
:109F700094E0A0E0B0E08093560390935703A09341
:109F80005803B09359038090560390905703209143
:109F9000E6013091E70137FF02C0295F3F4F43E000
:109FA000359527954A95E1F74FEF223834071CF491
:109FB00021E83FEF05C02038310514F020E830E0FB
:109FC000C901AA2797FDA095BA2F20915D013327DB
:109FD00044275527BC01CD010E949F7997FF04C0FB
:109FE0006D5F7F4F8F4F9F4F22E0959587957795B7
:109FF00067952A95D1F79B015FEF613075071CF4D7
:10A0000020E03FEF06C06F3F710519F014F020E02B
:10A0100031E080919303882349F0C90137FD03960D
:10A020009C0135952795359527950DC080911C0687
:10A0300080FF09C0C90137FD07969C01A3E0359553
:10A040002795AA95E1F7820E931E20915A012223AB
:10A0500009F454C06091DE027091DF028091E00249
:10A060009091E10297FF04C061587F4F8F4F9F4F3F
:10A07000F7E09595879577956795FA95D1F733270A
:10A08000442755270E949F7997FF04C0615E7F4F48
:10A090008F4F9F4FE5E09595879577956795EA9562
:10A0A000D1F76093560370935703809358039093AE
:10A0B00059036138AFEF7A07AFEF8A07AFEF9A071E
:10A0C0002CF480E89FEFAFEFBFEF0AC06F3F710540
:10A0D0008105910569F064F080E091E0A0E0B0E0D6
:10A0E0008093560390935703A0935803B09359035A
:10A0F0008091560390915703880E991E80915801C4
:10A10000282F332780912B08992787FD9095289F2A
:10A11000F001299FF00D389FF00D11249F01F7FFEA
:10A1200002C021583F4F220F232F221F330BFFEF76
:10A1300021383F071CF420E83FEF06C02F3F3105D0
:10A1400019F014F020E031E0820E931EC401AA271A
:10A1500097FDA095BA2FE090B202F090B30297015C
:10A16000442737FD4095542FBC01CD010E949F79B3
:10A1700097FF04C061507E4F8F4F9F4F59E09595D8
:10A180008795779567955A95D1F7061B170B8091A0
:10A19000870390918803892B09F060C01E141F0467
:10A1A0000CF05CC09601D7FE03C0309521953F4F5F
:10A1B0002D33310540F480918B0390918C038017EF
:10A1C000910774F526C02C53304045E0369527950D
:10A1D0004A95E1F72031310510F02FE030E0409151
:10A1E0008B0350918C031C141D04E4F480E190E077
:10A1F000821B930B489F9001499F300D589F300D53
:10A20000112494E0369527959A95E1F720173107A8
:10A2100020F5809170019091710108171907F4F0F1
:10A220008C011CC0205F3F4F8091700190917101A3
:10A23000829FB001839F700D929F700D11249B012E
:10A2400084E0369527958A95E1F74017510714F079
:10A250008A0104C00217130708F08901C801AA2760
:10A2600097FDA095BA2F1DE0880F991FAA1FBB1F4D
:10A270001A95D1F79301442737FD4095542FBC011F
:10A28000CD010E94137A20935A0330935B034093CD
:10A290005C0350935D0300915A0310915B0380911E
:10A2A000890390918A039C01220F331F280F391FC5
:10A2B000200F311F37FF02C02D5F3F4FA901559579
:10A2C00047955595479550938A034093890380910C
:10A2D000C705282F3327220F331F220F331F2417C0
:10A2E00035076CF48091AA07282F3327220F331FDC
:10A2F000220F331F205530404217530724F030936C
:10A300008A032093890380911C0680FF14C08091EA
:10A31000890390918A03A8A1B9A18A179B0724F009
:10A32000B0938A03A0938903E0918903F0918A0393
:10A33000F9A3E8A357C028A139A12E193F0937FF77
:10A3400002C02D5F3F4F3595279535952795E090B5
:10A350008903F0908A03E20EF31EF9A2E8A242C03C
:10A360008091CF05882301F56091B2027091B3020C
:10A3700077FF02C06D5F7F4F7595679575956795FF
:10A3800040911D0150911E0180910001282F33271B
:10A39000649FC001659F900D749F900D1124B901B9
:10A3A0000E94DE79CB0101C0992790936F018093C1
:10A3B0006E0180916E0190916F01873491051CF4BC
:10A3C00086E490E005C08639910534F086E990E096
:10A3D00090936F0180936E0108A119A110938A03D5
:10A3E000009389038091960299279C012270307016
:10A3F00081FF1CC180918D0390918E03A0918F03EA
:10A40000B09190030097A105B10521F08091C002A1
:10A410008130B1F428A139A1C901AA2797FDA095DF
:10A42000BA2F2EE0880F991FAA1FBB1F2A95D1F7BC
:10A4300080938D0390938E03A0938F03B09390032A
:10A440008091C002813019F482E08093C00248A15B
:10A4500059A1CA01AA2797FDA095BA2F93014427B5
:10A4600037FD4095542FBC01CD010E949F79DC013E
:10A47000CB0180935A0390935B03A0935C03B0934A
:10A480005D03B7FF04C08150904EAF4FBF4F5C01DA
:10A490006D018DE0D594C794B794A7948A95D1F7B0
:10A4A000A0925A03B0925B03C0925C03D0925D030A
:10A4B00060919702709198025FE0603A750750F5DD
:10A4C00080918D0390918E03A0918F03B0919003A2
:10A4D0009C01AD010AE056954795379527950A9559
:10A4E000D1F7821B930BA40BB50BA601950114E0C9
:10A4F000220F331F441F551F1A95D1F7820F931F48
:10A50000A41FB51F80938D0390938E03A0938F0398
:10A51000B093900360547F4118F580918D03909122
:10A520008E03A0918F03B09190039C01AD01FCE0DC
:10A530005695479537952795FA95D1F7821B930B3A
:10A54000A40BB50BA6019501E2E0220F331F441FB7
:10A55000551FEA95D1F7820F931FA41FB51F29C07D
:10A560008091E6019091E7018091E6019091E701E9
:10A5700097FF03C0909581959F4F843691050CF508
:10A5800080918D0390918E03A0918F03B0919003E1
:10A590009C01AD017EE056954795379527957A95B4
:10A5A000D1F7821B930BA40BB50B8A0D9B1DAC1D21
:10A5B000BD1D80938D0390938E03A0938F03B09362
:10A5C000900380918D0390918E03A0918F03B091A1
:10A5D00090036EE0B695A795979587956A95D1F704
:10A5E0009093B3028093B2024091CD05442399F039
:10A5F00055279C01BA010E94DE79C901861B970B81
:10A6000090938C0380938B03260F371F3093710137
:10A610002093700119C010928C0310928B038FEF5E
:10A6200093E090937101809370010EC01092C0026C
:10A6300010928D0310928E0310928F03109290034C
:10A640003093B3022093B2029091690798AB292FFF
:10A650003327220F331F220F331F285D3F4FA8A13E
:10A66000B9A12A173B0714F039A328A3B091AA0770
:10A67000B9AB8B2F9927880F991F880F991F805589
:10A680009040E8A1F9A18E179F0714F499A388A31D
:10A6900080911B02882321F4809132088F3FA1F022
:10A6A00080919702909198020297C09768F4E8A071
:10A6B000F9A01E141F0444F481E090E090939802E6
:10A6C0008093970239A328A308A119A110937305B9
:10A6D000009372058091520390915303A09154030B
:10A6E000B091550322E0880F991FAA1FBB1F2A951E
:10A6F000D1F7C090AD07D090AE07C81AD90A013A79
:10A7000011058CF0C80117FD0196959587958C155C
:10A710009D050CF46C01909581959F4FC816D90644
:10A7200094F46C0110C011E5C116D1041CF0E0E5F1
:10A73000CE2ED12C20EBC2162FEFD20624F470EBD4
:10A74000C72E7FEFD72E49A9242F3327220F331F7F
:10A75000220F331FC90168A179A1861B970B8C15A5
:10A760009D050CF46C0188A199A1821B930BC8165E
:10A77000D9060CF46C018091630790916407609195
:10A78000C8027091C902861B970B90937307809340
:10A790007207A09085072091E6023091E702409170
:10A7A000E8025091E902AA2041F0461A570AC20174
:10A7B000AA2797FDA095BA2F04C0AA2797FDA095B8
:10A7C000BA2F280F391F4A1F5B1F2093E6023093D0
:10A7D000E7024093E8025093E9028091E6029091EB
:10A7E000E702A091E802B091E90281509A4FA0409F
:10A7F000B04064F080E09AEFA0E0B0E08093E60221
:10A800009093E702A093E802B093E9028091E602F8
:10A810009091E702A091E802B091E9028050964041
:10A82000AF4FBF4F64F480E096E0AFEFBFEF80938F
:10A83000E6029093E702A093E802B093E902B09099
:10A84000DC052B2D33278091720790917307289F89
:10A850007001299FF00C389FF00C11249701F7FE2E
:10A8600002C0295F3F4F790153E0F594E7945A9570
:10A87000E1F700915E0110915F019801442737FDD7
:10A880004095542F8091E6029091E702A091E80252
:10A89000B091E902BC01CD010E94137AE20EF31ED1
:10A8A00090904A01692D7727882799279601D7FE2E
:10A8B00004C0222733272C193D0937FF02C02F5F20
:10A8C0003F4F3595279548A159A1240F351F44279F
:10A8D00037FD4095542F0E949F7997FF04C0615C1B
:10A8E0007F4F8F4F9F4F26E095958795779567957A
:10A8F0002A95D1F79B016E157F050CF47B013095ED
:10A9000021953F4FE216F3060CF47901809152072E
:10A91000909153076091C6027091C702861B970BF6
:10A9200090935107809350072091E2023091E30207
:10A930004091E4025091E502AA2041F0261A370A1C
:10A94000C101AA2797FDA095BA2F04C0AA2797FD99
:10A95000A095BA2F280F391F4A1F5B1F2093E202D0
:10A960003093E3024093E4025093E5028091E202C7
:10A970009091E302A091E402B091E50281509A4FD8
:10A98000A040B04064F080E09AEFA0E0B0E0809397
:10A99000E2029093E302A093E402B093E502809177
:10A9A000E2029091E302A091E402B091E5028050AE
:10A9B0009640AF4FBF4F64F480E096E0AFEFBFEF3B
:10A9C0008093E2029093E302A093E402B093E50245
:10A9D0002B2D33278091500790915107289FD0014C
:10A9E000299FB00D389FB00D11249D01B7FF02C003
:10A9F000295F3F4F5901B3E0B594A794BA95E1F7A9
:10AA00009801442737FD4095542F8091E2029091A0
:10AA1000E302A091E402B091E502BC01CD010E94E5
:10AA2000137AA20EB31E692D7727882799279601DE
:10AA3000D7FE04C0222733272C193D0937FF02C057
:10AA40002F5F3F4F35952795E8A1F9A12E0F3F1FA6
:10AA5000442737FD4095542F0E949F7997FF04C0EB
:10AA6000615C7F4F8F4F9F4FF6E095958795779567
:10AA70006795FA95D1F79B016A157B050CF45B018C
:10AA8000309521953F4FA216B3060CF45901209042
:10AA9000A502E0E86E2EE6E07E2E77E3872E76E0D4
:10AAA000972E6BE0362E58E8452E57E0552ED401F0
:10AAB0002C9112160CF0ECC0203419F408A119A145
:10AAC0001EC0E8A1F9A1CF01AA2797FDA095BA2F32
:10AAD000332727FD3095432F532FBC01CD010E9412
:10AAE0009F7997FF04C0615C7F4F8F4F9F4F46E077
:10AAF00095958795779567954A95D1F78B01F401E0
:10AB00002181203419F40E0D1F1D22C0203C19F4A0
:10AB10000E191F091DC0C701AA2797FDA095BA2FBE
:10AB2000332727FD3095432F532FBC01CD010E94C1
:10AB30009F7997FF04C0615C7F4F8F4F9F4F36E036
:10AB400095958795779567953A95D1F7060F171FD5
:10AB5000F4012281203419F40A0D1B1D22C0203C6F
:10AB600019F40A191B091DC0C501AA2797FDA09554
:10AB7000BA2F332727FD3095432F532FBC01CD012A
:10AB80000E949F7997FF04C0615C7F4F8F4F9F4F5A
:10AB900026E095958795779567952A95D1F7060FC5
:10ABA000171FF4012381203419F40C0D1D1D22C040
:10ABB000203C19F40C191D091DC0C601AA2797FDD8
:10ABC000A095BA2F332727FD3095432F532FBC0173
:10ABD000CD010E949F7997FF04C0615C7F4F8F4F2A
:10ABE0009F4FB6E09595879577956795BA95D1F77C
:10ABF000060F171FD2018D919C91801791075CF46D
:10AC0000BC01600F711F77FF02C06F5F7F4F8B0128
:10AC10001595079511C0B1E0B21528F0000F111F6E
:10AC2000081B190B09C0222D3327801B910BB9017A
:10AC30000E94DE79060F171FE8A98E2F9927880F2B
:10AC4000991F880F991F8017910754F4F9A98F2F26
:10AC50009927880F991F880F991F081719070CF05B
:10AC60008C01C80117FD0396959587959595879555
:10AC7000F3018183880F991F880F991F9801281B62
:10AC8000390BC901880F8283D2010D931C9303C035
:10AC9000F301118212823A9402E010E0400E511E3C
:10ACA00024E030E0820E931E48E050E0640E751EF2
:10ACB00037FEFDCEE2E1CB5C0C944A7A8091A00392
:10ACC0009091A103A091A203B091A3038093980354
:10ACD00090939903A0939A03B0939B0380919C0354
:10ACE00090919D03A0919E03B0919F038093940344
:10ACF00090939503A0939603B093970308951092B1
:10AD0000AB031092AA031092A9031092A80308950E
:10AD100084B1806A84B93D9A82E58CBD1DBC459A98
:10AD200081E08093BF078AEA8093D00783E880930D
:10AD3000D1078AE08093D2071092D4071092D307EC
:10AD40001092D6071092D50710922A081092F20797
:10AD500008953091BF07332309F085C00DB407FE75
:10AD600082C084E08093D201459A2EB58091AF03D2
:10AD700099278130910589F0823091051CF4892B47
:10AD800021F03EC00297B9F03BC03093F107209309
:10AD9000B0032138A9F581E008C0253549F4809138
:10ADA000B003820F8093B00382E08093AF0328C08A
:10ADB0003093AF0325C08091F107E82FFF27E35FB1
:10ADC000F74F20838F5F8093F1079091B0038A3112
:10ADD000A0F0291769F48AE1ADE0B8E0E3EFF7E00D
:10ADE0000D9001928A95E1F781E08093F20702C00D
:10ADF0003093F2071092AF0303C0920F9093B00309
:10AE00002091CF07203208F028C0459800000000AC
:10AE10000000000000000000000000000000000032
:10AE20000000000000000000000000000000000022
:10AE3000000000000000000000000000E091C807D2
:10AE4000F091C907E20FF11D80818EBD8091EF075F
:10AE50009081890F8093EF0703C081E08093BF0743
:10AE60002F5F2093CF070895EF92FF920F931F93C8
:10AE70008091D5059927880F991F880F991F7C010C
:10AE80000027F7FC0095102F80911E0390911F035F
:10AE9000A0912003B0912103BC01CD01A80197012D
:10AEA0000E94137A3093D4072093D307809116031E
:10AEB00090911703A0911803B0911903BC01CD0123
:10AEC000A80197010E94137A3093D6072093D507E3
:10AED0002091B4073091B5074091B6075091B7075C
:10AEE000DA01C901E3E0880F991FAA1FBB1FEA9589
:10AEF000D1F7820F931FA41FB51F820F931FA41FAA
:10AF0000B51F209144013091450140914601509177
:10AF10004701BC01CD010E94137A3093DC072093D6
:10AF2000DB0780912F03909130032091F401309141
:10AF3000F501821B930B9093E2078093E107E09168
:10AF40002503F091260380917B0790917C07BF0138
:10AF50000E94DE79CB019B01220F331F220F331F8A
:10AF6000280F391F280F391F37FF02C02D5F3F4FB1
:10AF700035952795359527953093D8072093D70792
:10AF80008091B0079091B107BF010E94DE799B01CB
:10AF9000220F331F220F331F260F371F260F371F95
:10AFA00037FF02C02D5F3F4F359527953595279583
:10AFB0003093DA072093D9071092260310922503C5
:10AFC00010927C0710927B071092B1071092B00785
:10AFD0008091D20799278D30910509F466C08E3093
:10AFE00091055CF48B30910509F48EC08C3091058D
:10AFF0000CF00FC10A9761F0A8C18F30910509F4D8
:10B000007CC18F3091050CF45CC1409799F19DC1D2
:10B010008091AB028093E3078091AA028093E407BA
:10B020008091A9028093E5078091A8028093E607AA
:10B030008091A7028093E7078091A6028093E8079A
:10B040008091A5028093E9078091A4028093EA078A
:10B05000809196028093EB0780919602837F809384
:10B0600096020E94D5218093EC0780912203809361
:10B07000ED076BC180912C0890912D089093E40707
:10B080008093E30780913008909131089093E60710
:10B090008093E50780911D0190911E018093E70741
:10B0A000809100018093E80750C18091070680934A
:10B0B000E307809108068093E40780910906809356
:10B0C000E50780910A068093E60780910B0680933E
:10B0D000E70780910F068093E80780911006809320
:10B0E000E907809111068093EA0780911406809306
:10B0F000EB07809112068093EC07809113068093F2
:10B10000ED0780911506DAC0F8948091BC05E82F10
:10B11000FF27EE0FFF1FEF51F94F0190F081E02D57
:10B12000E038F1051CF0EFE7F0E006C02FEFE13862
:10B13000F20714F4E1E8FFEFE093E3078091BD0527
:10B14000E82FFF27EE0FFF1FEF51F94F0190F0811D
:10B15000E02DE038F1051CF0EFE7F0E006C06FEFFE
:10B16000E138F60714F4E1E8FFEFE093E40780919B
:10B17000BB05E82FFF27EE0FFF1FEF51F94F01909E
:10B18000F081E02DE038F1051CF0EFE7F0E006C0BB
:10B190008FEFE138F80714F4E1E8FFEFE093E507FB
:10B1A0008091BA05E82FFF27EE0FFF1FEF51F94FEF
:10B1B0000190F081E02DE038F1051CF0EFE7F0E0C0
:10B1C00006C02FEFE138F20714F4E1E8FFEF7894BE
:10B1D000E093E6078091CB028093E7078091CC0251
:10B1E0008093E8078091CD028093E9078091CE0299
:10B1F0008093EA078091CF028093EB078091D00281
:10B200008093EC078091D1028093ED078091D20268
:10B2100055C080911104863018F01092110485E019
:10B220008093E307809116068093E4078091BC0227
:10B230009091BD02A091BE02B091BF02BC01CD01B0
:10B2400025E030E040E050E00E94137A3093E607BA
:10B250002093E5078091B8029091B902A091BA02BB
:10B26000B091BB02BC01CD0125E030E040E050E0F0
:10B270000E94137A3093E8072093E70780910C0629
:10B280008093E90780910D068093EA0780910E066E
:10B290008093EB078091CA028093EC078091E106CE
:10B2A0009091E2068093ED0780917205909173056D
:10B2B00097FD039695958795959587958093EE07CD
:10B2C00044C01092E30780E58093E40786E0809312
:10B2D000E5078EE08093E607809102018093E707FF
:10B2E0008091F6038093E8078091F7038093E90744
:10B2F0008091F8038093EA0728C08091EE0580933F
:10B30000E30780911B068093E407809150018093AE
:10B31000E5078091E7058093E6078091E805809333
:10B32000E7078091E9058093E80780914F018093BA
:10B33000E9078091EB058093EA078091EC05809303
:10B34000EB078091ED058093EC078091F20788234D
:10B3500009F4CFC08AEF80939B014091F40750918C
:10B36000F507CA0181509E4F8F5F9340B0F4209142
:10B37000F6073091F707C90181509E4F8F5F9340C8
:10B3800060F48091C60585FF08C05093AB034093DD
:10B39000AA033093A9032093A8038091FA07909100
:10B3A000FB0721E08936920724F49093DD02809315
:10B3B000DC028091DC029091DD022091DA02309172
:10B3C000DB02821B930B845E9D4F68E671E00E9456
:10B3D000DE79845B90409093D9028093D8022091CB
:10B3E000FE073091FF078091D3019091D40182171D
:10B3F000930740F480911104882321F43093D40101
:10B400002093D3018091F30799278836910549F15C
:10B410008936910524F48736910531F072C089365A
:10B42000910509F445C06DC08091000880932708FC
:10B430008091010880932908809102088093280850
:10B440008091030880932A088091040880932B0838
:10B450008091050880939C01809106088093AE033B
:10B4600050C0809100088093CA07809101088093A2
:10B47000CB07809102088093CC07809103088093CA
:10B48000CD07809104088093CE078091620590914A
:10B490000508892B80936205909106089093AC0370
:10B4A0008091630583709C70892B8093630529C00C
:10B4B000809100088093C007809101088093C107A4
:10B4C000809102088093C207809103088093C3078C
:10B4D00080910408909105089093C5078093C40754
:10B4E00080910608909107089093C7078093C6073C
:10B4F00008C01092AB031092AA031092A9031092F5
:10B50000A8031F910F91FF90EF9008958091BF07BE
:10B51000882309F43BC0459880ED97E09093C907D4
:10B520008093C8079091AD03E92FFF27EE56FE4F99
:10B530009F5F9093AD0380818093D207993010F084
:10B540001092AD031092BF070E94345781E08093A0
:10B55000CF07000000000000000000000000000015
:10B5600000000000000000000000000000000000DB
:10B5700000000000000000000000000000000000CB
:10B5800000008091D0078093EF078EBD089587B1AA
:10B590008C6087B9429843981092B20380E88093F8
:10B5A0009E011092B10380939D0108958091B7038D
:10B5B00081508093B7038F3F09F0FBC094E09093D4
:10B5C000B70380910006882319F081E08093B703C8
:10B5D00080919602807BE1F080910506882349F0F6
:10B5E0008091BA03882311F49093B20381E0809391
:10B5F000BA03809106068823B9F08091BB038823A3
:10B6000019F484E08093B10381E08093BB030CC004
:10B610008093BA038093BB03809101068093B803A3
:10B62000809103068093B9038091BA03882309F0BF
:10B6300040C080911A06282F332724FF07C080912D
:10B64000C102882319F425FD4DC04EC09091020619
:10B65000983F50F080917D078D3D30F08091B80388
:10B6600088230CF43FC040C0983F48F080917D078C
:10B670008A3028F48091B8038823B4F133C08091D4
:10B68000B20381508093B2038F3F79F580917D079B
:10B6900081508093B20380919E01813011F480E843
:10B6A00001C0869580939E0180919E019091B80380
:10B6B00017C08091B20381508093B2038F3FA9F4E9
:10B6C00089E08093B20380919E01813011F480E87B
:10B6D00001C0869580939E0180919E019091050600
:10B6E000892311F0429A01C042988091BB038823BC
:10B6F00009F043C080911A06282F332724FF07C082
:10B700008091C102882319F426FD50C034C0909165
:10B710000406983F50F08091A9078D3D30F080914C
:10B72000B90388230CF442C026C0983F48F08091AA
:10B73000A9078A3028F48091B9038823E4F036C041
:10B740008091B10381508093B1038F3F91F5809137
:10B75000A90781508093B10380919D01813011F43C
:10B7600080E801C0869580939D0180919D01909114
:10B77000B9038923D9F4439808958091B103815086
:10B780008093B1038F3FA9F489E08093B103809146
:10B790009D01813011F480E801C0869580939D0160
:10B7A00080919D0190910606892311F0439A089596
:10B7B0004398089508950895CF93FC0197FF05C01D
:10B7C000CFEFF095E195FF4F01C0C1E028E631E0F1
:10B7D000CF01B9010E94DE79FC018B35910554F04F
:10B7E0008B5590408A35910538F484EB90E08E1BA0
:10B7F0009F0BFC0141E00DC0CF01855B90408A3575
:10B80000910518F4E45BF04003C02E1B3F0BF901D7
:10B810004FEFEE0FFF1FE55EFB4F259134918C2F0C
:10B82000992787FD9095289FB001299F700D389F1B
:10B83000700D1124842F992787FD9095689FA00192
:10B84000699F500D789F500D1124CA01CF91089522
:10B850002AE530E0281B390BC9010E94DC5B089502
:10B86000CF93DF9380E00E94C97280911D01909177
:10B870001E016AE070E00E94DE799F938F938091B1
:10B880001D0190911E016AE070E00E94DE797F93B5
:10B890006F938BE595E09F938F93CCEBD2E7DF938B
:10B8A000CF93E091DA03F091DB0309952DB73EB712
:10B8B000285F3F4F2DBF80919B018823B9F186E01F
:10B8C0000E94C9728091C4079091C5076AE070E038
:10B8D0000E94CA797F936F938FED90E09F938F932F
:10B8E0008091B4079091B507A091B607B091B707C2
:10B8F000209144013091450140914601509147010A
:10B90000BC01CD010E94137A3F932F9384E695E00A
:10B910009F938F93DF93CF93E091DA03F091DB0352
:10B9200009958DB79EB70A968DBF12C086E00E941A
:10B93000C97280E795E09F938F93DF93CF93E09157
:10B94000DA03F091DB0309950F900F900F900F90A1
:10B950008091AC038823C1F086E00E94C972809177
:10B96000AC0399279F938F9387E795E09F938F93DD
:10B97000DF93CF93E091DA03F091DB0309952DB7C4
:10B980003EB72A5F3F4F2DBF80E10E94C972809170
:10B99000A5019091A6016CE370E00E94CA799F9383
:10B9A0008F938091A5019091A6016CE370E00E94B5
:10B9B000CA797F936F9380913008909131089F935B
:10B9C0008F9382E895E09F938F93CCEBD2E7DF9340
:10B9D000CF93E091DA03F091DB0309958091C605DE
:10B9E0002DB73EB7265F3F4F2DBF80FF29C08AE1AC
:10B9F0000E94C9728091430199279F938F938091F0
:10BA0000BC029091BD02A091BE02B091BF02BC01E8
:10BA1000CD0124E630E040E050E00E94137A3F93ED
:10BA20002F938FE895E09F938F93DF93CF93E091CF
:10BA3000DA03F091DB0309958DB79EB708968DBFA9
:10BA4000DF91CF910895CF93DF9380E00E94C97278
:10BA500080919F06992787FD90959F938F93809162
:10BA60009706992787FD90959F938F9380918F06D6
:10BA7000992787FD90959F938F93809187069927AB
:10BA800087FD90959F938F9386E995E09F938F9381
:10BA9000CCEBD2E7DF93CF93E091DA03F091DB03B5
:10BAA000099580E10E94C9722DB73EB7245F3F4FD0
:10BAB0002DBF8091BF06992787FD90959F938F9307
:10BAC0008091B706992787FD90959F938F938091DA
:10BAD000AF06992787FD90959F938F938091A70636
:10BAE000992787FD90959F938F9386EA95E09F9382
:10BAF0008F93DF93CF93E091DA03F091DB03099505
:10BB00008091B8052DB73EB7245F3F4F2DBF8530DC
:10BB100098F480E10E94C97286EB95E09F938F9321
:10BB2000DF93CF93E091DA03F091DB0309950F9057
:10BB30000F900F900F9018C08730B0F488E10E94EA
:10BB4000C9728FED90E09F938F9387EC95E09F9360
:10BB50008F93DF93CF93E091DA03F091DB030995A4
:10BB60008DB79EB706968DBFDF91CF910895CF9385
:10BB7000DF9320912C0830912D088091D40390916F
:10BB8000D5038217930720F43093D5032093D40371
:10BB900080E00E94C97280911D0190911E016AE0AF
:10BBA00070E00E94DE799F938F9380911D019091A8
:10BBB0001E016AE070E00E94DE797F936F9380ED52
:10BBC00095E09F938F93CCEBD2E7DF93CF93E091F7
:10BBD000DA03F091DB0309958DB79EB708968DBF08
:10BBE0008091C1028823D1F48AE00E94C9728091B9
:10BBF000D4039091D5036AE070E00E94CA799F93C4
:10BC00008F938091D4039091D5036AE070E00E94F5
:10BC1000CA797F936F9389ED95E019C08AE00E94FD
:10BC2000C97280912C0890912D086AE070E00E9402
:10BC3000CA799F938F9380912C0890912D086AE088
:10BC400070E00E94CA797F936F9382EE95E09F9394
:10BC50008F93DF93CF93E091DA03F091DB030995A3
:10BC60008DB79EB708968DBF80E10E94C972809102
:10BC70003008909131089F938F9380912E08909176
:10BC80002F089F938F938BEE95E09F938F93DF9375
:10BC9000CF93E091DA03F091DB0309958DB79EB75E
:10BCA00008968DBFDF91CF9108950F931F93CF9387
:10BCB000DF9380919B01CCEBD2E7882309F478C015
:10BCC00080E00E94C9728091C10799279F938F934A
:10BCD0008091C30799279F938F9387EF95E09F9358
:10BCE0008F938E01DF93CF93E091DA03F091DB0322
:10BCF00009958DB79EB708968DBF8091C207833096
:10BD000031F48CE00E94C97286E096E005C08CE0B8
:10BD10000E94C9728BE096E09F938F93DF93CF933D
:10BD2000E091DA03F091DB0309950F900F900F90EB
:10BD30000F908091C00781FF12C08CE00E94C972F1
:10BD400080E196E09F938F931F930F93E091DA0326
:10BD5000F091DB0309950F900F900F900F9080E109
:10BD60000E94C9728FED90E09F938F938091C607D8
:10BD70009091C7079F938F938091C4079091C507B7
:10BD80006AE070E00E94CA797F936F9385E196E044
:10BD90009F938F938CEB92E79F938F93E091DA03BD
:10BDA000F091DB0309958DB79EB70A968DBF12C03F
:10BDB00082E00E94C97285E296E09F938F93DF93A1
:10BDC000CF93E091DA03F091DB0309950F900F9088
:10BDD0000F900F90DF91CF911F910F9108951F93B6
:10BDE000CF93DF93182F8091AC078F5F8093AC07C0
:10BDF00090916A01891710F11092AC078091850625
:10BE000080937A0780918D068093AB078091950689
:10BE10008093790780919D06809387078091A5067E
:10BE20008093A5078091AD06809365078091B50644
:10BE3000809382078091BD06809386079091850646
:10BE40008091D803891710F49093D80390918D06B0
:10BE50008091DC03891710F49093DC039091950690
:10BE60008091D603891710F49093D60390919D0684
:10BE70008091D703891710F49093D7039091A5066A
:10BE80008091D903891710F49093D9039091AD064E
:10BE90008091D303891710F49093D3039091B50642
:10BEA0008091DD03891710F49093DD039091BD0616
:10BEB0008091DE03891710F49093DE038091C10214
:10BEC000882301F58091D80380937A078091DC0361
:10BED0008093AB078091D603809379078091D70335
:10BEE000809387078091D9038093A5078091D3031E
:10BEF000809365078091DD03809382078091DE0344
:10BF00008093860780E00E94C97280918707282F5E
:10BF100033278091B805482F552780913803909199
:10BF20003903BA010E94CA79261B370B3F932F931E
:10BF300080917907282F33278091B805482F5527FE
:10BF40008091380390913903BA010E94CA79261B67
:10BF5000370B3F932F938091AB07282F3327809186
:10BF6000B805482F55278091380390913903BA01BD
:10BF70000E94CA79261B370B3F932F9380917A0733
:10BF8000282F33278091B805482F552780913803F3
:10BF900090913903BA010E94CA79261B370B3F934F
:10BFA0002F9382E396E09F938F93CCEBD2E7DF93BE
:10BFB000CF93E091DA03F091DB03099580E10E94D1
:10BFC000C9722DB73EB7245F3F4F2DBF80918207C6
:10BFD000282F33278091B805482F552780913803A3
:10BFE00090913903BA010E94CA79261B370B3F93FF
:10BFF0002F9380918207282F33278091B805482FEF
:10C0000055278091380390913903BA010E94CA796B
:10C01000261B370B3F932F9380916507282F3327DB
:10C020008091B805482F55278091380390913903A6
:10C03000BA010E94CA79261B370B3F932F93809138
:10C04000A507282F33278091B805482F55278091C1
:10C05000380390913903BA010E94CA79261B370B25
:10C060003F932F9382E496E09F938F93DF93CF9338
:10C07000E091DA03F091DB0309958091B8052DB7C3
:10C080003EB7245F3F4F2DBF853038F580E10E94D9
:10C09000C97280912C0890912D086AE070E00E948E
:10C0A000CA799F938F9380912C0890912D086AE014
:10C0B00070E00E94CA797F936F9382E596E09F9328
:10C0C0008F93DF93CF93E091DA03F091DB0309952F
:10C0D0008DB79EB708968DBF29C0873038F588E1A7
:10C0E0000E94C97280912C0890912D086AE070E03E
:10C0F0000E94CA799F938F9380912C0890912D086C
:10C100006AE070E00E94CA797F936F9385E696E0BB
:10C110009F938F93DF93CF93E091DA03F091DB034A
:10C1200009952DB73EB7285F3F4F2DBF1F3221F431
:10C1300080916A018F5F05C01F3429F480916A01E4
:10C14000815080936A01DF91CF911F910895482F0C
:10C1500010928407109254071092A107109237038F
:10C1600080916B0190916C011816190634F081E0F2
:10C1700090E090936C0180936B0180916B019091A2
:10C180006C01059734F081E090E090936C0180930E
:10C190006B0120916B0130916C012130310519F454
:10C1A0008EE3809384072230310519F48EE3809367
:10C1B00054072330310519F48EE38093A10724300E
:10C1C000310519F48EE3809337034F3839F4215049
:10C1D000304030936C0120936B0108954F3131F45E
:10C1E0002F5F3F4F30936C0120936B0108950F93A5
:10C1F0001F9380E00E94C97280919B0699278F77D8
:10C2000090709F938F938091930699278F7790706A
:10C210009F938F9380918B0699278F7790709F9330
:10C220008F938091830699278F7790709F938F9338
:10C230008FE696E09F938F930CEB12E71F930F937B
:10C24000E091DA03F091DB03099580E10E94C97265
:10C250008DB79EB70C968DBF8091BB0699278F77BF
:10C2600090709F938F938091B30699278F779070EA
:10C270009F938F938091AB0699278F7790709F93B0
:10C280008F938091A30699278F7790709F938F93B8
:10C290008FE796E09F938F931F930F93E091DA03BC
:10C2A000F091DB0309958DB79EB70C968DBF1F915A
:10C2B0000F9108951F93CF93DF93182F8091AC07B0
:10C2C0008F5F8093AC0790916A01891710F11092EB
:10C2D000AC078091810680937A07809189068093CC
:10C2E000AB0780919106809379078091990680939E
:10C2F00087078091A1068093A5078091A906809366
:10C3000065078091B106809382078091B90680937A
:10C31000860780E00E94C9728091870799279F93C2
:10C320008F938091790799279F938F938091AB0783
:10C3300099279F938F9380917A0799279F938F9343
:10C340008FE896E09F938F93CCEBD2E7DF93CF9368
:10C35000E091DA03F091DB03099580E10E94C97254
:10C360002DB73EB7245F3F4F2DBF80918607992799
:10C370009F938F938091820799279F938F938091AA
:10C38000650799279F938F938091A50799279F937E
:10C390008F938FE996E09F938F93DF93CF93E091F4
:10C3A000DA03F091DB0309958091B8052DB73EB70C
:10C3B000245F3F4F2DBF853098F480E10E94C97201
:10C3C0008FEA96E09F938F93DF93CF93E091DA0308
:10C3D000F091DB0309950F900F900F900F9019C00B
:10C3E0008730B8F488E10E94C97280916A01992768
:10C3F0009F938F9380EC96E09F938F93DF93CF93DF
:10C40000E091DA03F091DB0309958DB79EB70696AC
:10C410008DBF1F3221F480916A018F5F05C01F34E8
:10C4200029F480916A01815080936A01DF91CF9154
:10C430001F9108956F927F928F929F92AF92BF92B9
:10C44000CF92DF92EF92FF920F931F93A090E6029C
:10C45000B090E702C090E802D090E90229E0D594BC
:10C46000C794B794A7942A95D1F7E090E202F09090
:10C47000E3020091E4021091E50299E01595079519
:10C48000F794E7949A95D1F76090EE027090EF02DE
:10C490008090F0029090F10289E0959487947794CF
:10C4A00067948A95D1F780E00E94C972FF92EF925B
:10C4B000BF92AF9289EC96E09F938F930CEB12E7BB
:10C4C0001F930F93E091DA03F091DB03099580E16C
:10C4D0000E94C9728DB79EB708968DBF7F926F92EA
:10C4E00087ED96E09F938F931F930F93E091DA036C
:10C4F000F091DB0309958DB79EB706968DBF1F910E
:10C500000F91FF90EF90DF90CF90BF90AF909F90F2
:10C510008F907F906F900895CF93DF9380E00E947B
:10C52000C9728091E6019091E7019F938F9388EE05
:10C5300096E09F938F93CCEBD2E7DF93CF93E0917C
:10C54000DA03F091DB03099580E10E94C9728DB78F
:10C550009EB706968DBF8091C2029091C3029F93B1
:10C560008F938091B2029091B30297FD03969595B7
:10C570008795959587959F938F9383EF96E09F93EB
:10C580008F93DF93CF93E091DA03F091DB0309956A
:10C590008DB79EB708968DBFDF91CF9108950F9309
:10C5A0001F93CF93C82F0E94A76080E00E94C9729A
:10C5B0008091FF069091000781589F4F9F938F9322
:10C5C0008091A10799279F938F938091FB0690916B
:10C5D000FC0681589F4F9F938F93809184079927E2
:10C5E0009F938F9384E097E09F938F930CEB12E7D8
:10C5F0001F930F93E091DA03F091DB03099580E13B
:10C600000E94C9722DB73EB7245F3F4F2DBF809166
:10C6100001079091020781589F4F9F938F938091BC
:10C62000370399279F938F938091FD069091FE0683
:10C6300081589F4F9F938F938091540799279F9381
:10C640008F9387E197E09F938F931F930F93E091D0
:10C65000DA03F091DB03099580E090E02DB73EB757
:10C66000245F3F4F2DBFCF3211F481E090E040E0D6
:10C6700050E020916B0130916C012130310509F4BB
:10C68000A90184239523892B49F08091FB06909181
:10C69000FC0601969093FC068093FB0680E090E0F8
:10C6A000CF3411F481E090E040E050E021303105DA
:10C6B00009F4A90184239523892B49F08091FB0675
:10C6C0009091FC0601979093FC068093FB0680E016
:10C6D00090E0CF3211F481E090E040E050E0223071
:10C6E000310511F441E050E084239523892B49F072
:10C6F0008091FD069091FE0601969093FE06809330
:10C70000FD0680E090E0CF3411F481E090E040E05D
:10C7100050E02230310511F441E050E084239523AC
:10C72000892B49F08091FD069091FE060197909328
:10C73000FE068093FD0680E090E0CF3211F481E0A8
:10C7400090E040E050E02330310511F441E050E04A
:10C7500084239523892B49F08091FF06909100074F
:10C760000196909300078093FF0680E090E0CF341D
:10C7700011F481E090E040E050E02330310511F405
:10C7800041E050E084239523892B49F08091FF06F6
:10C79000909100070197909300078093FF0680E037
:10C7A00090E0CF3211F481E090E040E050E024309E
:10C7B000310511F441E050E084239523892B49F0A1
:10C7C0008091010790910207019690930207809350
:10C7D000010780E090E0CF3411F481E090E040E088
:10C7E00050E02430310511F441E050E084239523DA
:10C7F000892B49F08091010790910207019790934E
:10C80000020780930107CF911F910F910895CF9355
:10C81000C82F80911C0680FF14C080E00E94C9725E
:10C820008AE297E09F938F938CEB92E79F938F938D
:10C83000E091DA03F091DB0309950F900F900F90D0
:10C840000F9080911C0680FD14C080E10E94C97287
:10C850008BE397E09F938F938CEB92E79F938F935B
:10C86000E091DA03F091DB0309950F900F900F90A0
:10C870000F90CF3221F480911C06816006C0CF3426
:10C8800031F480911C068E7F826080931C06CF91CC
:10C8900008950F931F93CF93C82F0E94A76080E045
:10C8A0000E94C9728091CC0599279F938F938091A4
:10C8B000A10799279F938F938091C80599279F93EC
:10C8C0008F938091840799279F938F938CE497E0AF
:10C8D0009F938F930CEB12E71F930F93E091DA0372
:10C8E000F091DB03099580E10E94C9722DB73EB734
:10C8F000245F3F4F2DBF8091C70599279F938F934A
:10C900008091370399279F938F938091CA05992728
:10C910009F938F938091540799279F938F938EE5D0
:10C9200097E09F938F931F930F93E091DA03F09119
:10C93000DB03099580E090E02DB73EB7245F3F4FC1
:10C940002DBFCF3211F481E090E040E050E0209123
:10C950006B0130916C012130310509F4A901842368
:10C960009523892B29F08091C8058F5F8093C80596
:10C9700080E090E0CF3411F481E090E040E050E0BE
:10C980002130310509F4A90184239523892B29F04D
:10C990008091C80581508093C80580E090E0CF3237
:10C9A00011F481E090E040E050E02230310511F4D4
:10C9B00041E050E084239523892B29F08091CA051A
:10C9C0008F5F8093CA0580E090E0CF3411F481E05E
:10C9D00090E040E050E02230310511F441E050E0B9
:10C9E00084239523892B29F08091CA058150809357
:10C9F000CA0580E090E0CF3211F481E090E040E0A1
:10CA000050E02330310511F441E050E084239523B8
:10CA1000892B29F08091CC058F5F8093CC0580E035
:10CA200090E0CF3411F481E090E040E050E023301A
:10CA3000310511F441E050E084239523892B29F03E
:10CA40008091CC0581508093CC0580E090E0CF327E
:10CA500011F481E090E040E050E02430310511F421
:10CA600041E050E084239523892B29F08091C7056C
:10CA70008F5F8093C70580E090E0CF3411F481E0B0
:10CA800090E040E050E02430310511F441E050E006
:10CA900084239523892B29F08091C70581508093A9
:10CAA000C705CF911F910F9108950F931F93CF93B7
:10CAB000C82F0E94A76080E00E94C9728091CE05B5
:10CAC00099279F938F938091A10799279F938F9385
:10CAD0008091CD0599279F938F9380918407992703
:10CAE0009F938F9380E797E09F938F930CEB12E7D0
:10CAF0001F930F93E091DA03F091DB03099580E136
:10CB00000E94C9722DB73EB7245F3F4F2DBF809161
:10CB1000C90599279F938F938091370399279F93F6
:10CB20008F938091CB0599279F938F938091540782
:10CB300099279F938F9382E897E09F938F931F93FA
:10CB40000F93E091DA03F091DB03099580E090E028
:10CB50002DB73EB7245F3F4F2DBFCF3211F481E098
:10CB600090E040E050E020916B0130916C01213069
:10CB7000310509F4A90184239523892B29F080919B
:10CB8000CD058F5F8093CD0580E090E0CF3411F428
:10CB900081E090E040E050E02130310509F4A90146
:10CBA00084239523892B29F08091CD058150809392
:10CBB000CD0580E090E0CF3211F481E090E040E0DC
:10CBC00050E02230310511F441E050E084239523F8
:10CBD000892B29F08091CB058F5F8093CB0580E076
:10CBE00090E0CF3411F481E090E040E050E022305A
:10CBF000310511F441E050E084239523892B29F07D
:10CC00008091CB0581508093CB0580E090E0CF32BE
:10CC100011F481E090E040E050E02330310511F460
:10CC200041E050E084239523892B29F08091CE05A3
:10CC30008F5F8093CE0580E090E0CF3411F481E0E7
:10CC400090E040E050E02330310511F441E050E045
:10CC500084239523892B29F08091CE0581508093E0
:10CC6000CE05CF911F910F9108950F931F93CF93EE
:10CC7000C82F0E94A76080E00E94C9728091D205EF
:10CC800099279F938F938091A10799279F938F93C3
:10CC90008091D00599279F938F938091840799273E
:10CCA0009F938F9384E997E09F938F930CEB12E708
:10CCB0001F930F93E091DA03F091DB03099580E174
:10CCC0000E94C9722DB73EB7245F3F4F2DBF8091A0
:10CCD000FB0599279F938F938091370399279F9303
:10CCE0008F938091D10599279F938F9380915407BB
:10CCF00099279F938F9387EA97E09F938F931F9332
:10CD00000F93E091DA03F091DB03099580E090E066
:10CD10002DB73EB7245F3F4F2DBFCF3211F481E0D6
:10CD200090E040E050E020916B0130916C012130A7
:10CD3000310509F4A90184239523892B29F08091D9
:10CD4000D0058F5F8093D00580E090E0CF3411F460
:10CD500081E090E040E050E02130310509F4A90184
:10CD600084239523892B29F08091D00581508093CD
:10CD7000D00580E090E0CF3211F481E090E040E017
:10CD800050E02230310511F441E050E08423952336
:10CD9000892B29F08091D1058F5F8093D10580E0A8
:10CDA00090E0CF3411F481E090E040E050E0223098
:10CDB000310511F441E050E084239523892B29F0BB
:10CDC0008091D10581508093D10580E090E0CF32F1
:10CDD00011F481E090E040E050E02330310511F49F
:10CDE00041E050E084239523892B29F08091D205DE
:10CDF0008F5F8093D20580E090E0CF3411F481E022
:10CE000090E040E050E02330310511F441E050E083
:10CE100084239523892B29F08091D205815080931A
:10CE2000D20580E090E0CF3211F481E090E040E064
:10CE300050E02430310511F441E050E08423952383
:10CE4000892B29F08091FB058F5F8093FB0580E0A3
:10CE500090E0CF3411F481E090E040E050E02430E5
:10CE6000310511F441E050E084239523892B29F00A
:10CE70008091FB0581508093FB05CF911F910F910D
:10CE800008950F931F93CF93C82F0E94A76080E04F
:10CE90000E94C9728091D80599279F938F938091A2
:10CEA000A10799279F938F938091D70599279F93E7
:10CEB0008F938091840799279F938F938AEB97E0B4
:10CEC0009F938F930CEB12E71F930F93E091DA037C
:10CED000F091DB03099580E10E94C9722DB73EB73E
:10CEE000245F3F4F2DBF8091E10599279F938F933A
:10CEF0008091370399279F938F938091D905992724
:10CF00009F938F938091540799279F938F938DECD4
:10CF100097E09F938F931F930F93E091DA03F09123
:10CF2000DB03099580E090E02DB73EB7245F3F4FCB
:10CF30002DBFCF3211F481E090E040E050E020912D
:10CF40006B0130916C012130310509F4A901842372
:10CF50009523892B29F08091D7058F5F8093D70582
:10CF600080E090E0CF3411F481E090E040E050E0C8
:10CF70002130310509F4A90184239523892B29F057
:10CF80008091D70581508093D70580E090E0CF3223
:10CF900011F481E090E040E050E02230310511F4DE
:10CFA00041E050E084239523892B29F08091D90515
:10CFB0008F5F8093D90580E090E0CF3411F481E059
:10CFC00090E040E050E02230310511F441E050E0C3
:10CFD00084239523892B29F08091D9058150809352
:10CFE000D90580E090E0CF3211F481E090E040E09C
:10CFF00050E02330310511F441E050E084239523C3
:10D00000892B29F08091D8058F5F8093D80580E027
:10D0100090E0CF3411F481E090E040E050E0233024
:10D02000310511F441E050E084239523892B29F048
:10D030008091D80581508093D80580E090E0CF3270
:10D0400011F481E090E040E050E02430310511F42B
:10D0500041E050E084239523892B29F08091E1055C
:10D060008F5F8093E10580E090E0CF3411F481E0A0
:10D0700090E040E050E02430310511F441E050E010
:10D0800084239523892B29F08091E1058150809399
:10D09000E105CF911F910F9108950F931F93CF93A7
:10D0A000C82F0E94A76080E00E94C9728091130679
:10D0B00099279F938F938091A10799279F938F938F
:10D0C0008091080699279F938F93809184079927D1
:10D0D0009F938F9380EE97E09F938F930CEB12E7D3
:10D0E0001F930F93E091DA03F091DB03099580E140
:10D0F0000E94C9722DB73EB7245F3F4F2DBF80916C
:10D10000150699279F938F938091370399279F93B3
:10D110008F938091120699279F938F938091540744
:10D1200099279F938F9383EF97E09F938F931F93FC
:10D130000F93E091DA03F091DB03099580E090E032
:10D140002DB73EB7245F3F4F2DBFCF3211F481E0A2
:10D1500090E040E050E020916B0130916C01213073
:10D16000310509F4A90184239523892B29F08091A5
:10D1700008068F5F8093080680E090E0CF3411F4BA
:10D1800081E090E040E050E02130310509F4A90150
:10D1900084239523892B29F0809108068150809360
:10D1A000080680E090E0CF3211F481E090E040E0AA
:10D1B00050E02230310511F441E050E08423952302
:10D1C000892B29F0809112068F5F8093120680E0F0
:10D1D00090E0CF3411F481E090E040E050E0223064
:10D1E000310511F441E050E084239523892B29F087
:10D1F0008091120681508093120680E090E0CF3239
:10D2000011F481E090E040E050E02330310511F46A
:10D2100041E050E084239523892B29F08091130667
:10D220008F5F8093130680E090E0CF3411F481E0AB
:10D2300090E040E050E02330310511F441E050E04F
:10D2400084239523892B29F08091130681508093A4
:10D25000130680E090E0CF3211F481E090E040E0EE
:10D2600050E02430310511F441E050E0842395234F
:10D27000892B29F0809115068F5F8093150680E039
:10D2800090E0CF3411F481E090E040E050E02430B1
:10D29000310511F441E050E084239523892B29F0D6
:10D2A00080911506815080931506CF911F910F91A3
:10D2B00008951F93CF93DF93182F80E00E94C972C7
:10D2C00086E098E09F938F93CCEBD2E7DF93CF93E8
:10D2D000E091DA03F091DB03099580911A060F9033
:10D2E0000F900F900F9082FF06C08CE30E94BC72DB
:10D2F00080E00E94BC7280911A0680FF06C08EE515
:10D300000E94BC7280E00E94BC7280911A0681FF6C
:10D3100006C086E70E94BC7280E00E94BC728091C9
:10D320001A0683FF03C08EE30E94BC7280E10E9454
:10D33000C97280911A0699279F938F9388E098E08D
:10D340009F938F93DF93CF93E091DA03F091DB0308
:10D35000099520E030E08DB79EB706968DBF1F324D
:10D3600011F421E030E040E050E080911A068F3067
:10D3700010F441E050E024233523232B19F08F5F74
:10D3800080931A0620E030E01F3411F421E030E0F1
:10D3900040E050E080911A06882311F041E050E00F
:10D3A00024233523232B19F0815080931A06DF9113
:10D3B000CF911F9108950F931F93CF93C82F0E9471
:10D3C000A76080E00E94C9728091F40599279F931D
:10D3D0008F938091A10799279F938F938091F20556
:10D3E00099279F938F938091840799279F938F9379
:10D3F0008AE198E09F938F930CEB12E71F930F93B2
:10D40000E091DA03F091DB03099580E10E94C97293
:10D410002DB73EB7245F3F4F2DBF8091370399272B
:10D420009F938F938091F30599279F938F9380917A
:10D43000540799279F938F938DE298E09F938F9342
:10D440001F930F93E091DA03F091DB03099580E0DD
:10D4500090E02DB73EB7265F3F4F2DBFCF3211F47E
:10D4600081E090E040E050E020916B0130916C0150
:10D470002130310509F4A90184239523892B29F052
:10D480008091F2058F5F8093F20580E090E0CF34C9
:10D4900011F481E090E040E050E02130310509F4E2
:10D4A000A90184239523892B29F08091F2058150CD
:10D4B0008093F20580E090E0CF3211F481E090E0BB
:10D4C00040E050E02230310511F441E050E0842387
:10D4D0009523892B29F08091F3058F5F8093F305C5
:10D4E00080E090E0CF3411F481E090E040E050E043
:10D4F0002230310511F441E050E084239523892B3B
:10D5000029F08091F30581508093F30580E090E04D
:10D51000CF3211F481E090E040E050E0233031055B
:10D5200011F441E050E084239523892B29F0809168
:10D53000F4058F5F8093F40580E090E0CF3411F420
:10D5400081E090E040E050E02330310511F441E00B
:10D5500050E084239523892B29F08091F405815094
:10D560008093F405CF911F910F9108950F931F930E
:10D57000CF93C82F0E94A76080E00E94C97280915B
:10D58000F70599279F938F938091A10799279F93E0
:10D590008F938091F50599279F938F9380918407AE
:10D5A00099279F938F9389E398E09F938F930CEB38
:10D5B00012E71F930F93E091DA03F091DB030995D3
:10D5C00080E10E94C9722DB73EB7245F3F4F2DBF47
:10D5D0008091FF0599279F938F9380913703992717
:10D5E0009F938F938091F60599279F938F938091B6
:10D5F000540799279F938F938CE498E09F938F9380
:10D600001F930F93E091DA03F091DB03099580E01B
:10D6100090E02DB73EB7245F3F4F2DBFCF3211F4BE
:10D6200081E090E040E050E020916B0130916C018E
:10D630002130310509F4A90184239523892B29F090
:10D640008091F5058F5F8093F50580E090E0CF3401
:10D6500011F481E090E040E050E02130310509F420
:10D66000A90184239523892B29F08091F505815008
:10D670008093F50580E090E0CF3211F481E090E0F6
:10D6800040E050E02230310511F441E050E08423C5
:10D690009523892B29F08091F6058F5F8093F605FD
:10D6A00080E090E0CF3411F481E090E040E050E081
:10D6B0002230310511F441E050E084239523892B79
:10D6C00029F08091F60581508093F60580E090E086
:10D6D000CF3211F481E090E040E050E0233031059A
:10D6E00011F441E050E084239523892B29F08091A7
:10D6F000F7058F5F8093F70580E090E0CF3411F459
:10D7000081E090E040E050E02330310511F441E049
:10D7100050E084239523892B29F08091F7058150CF
:10D720008093F70580E090E0CF3211F481E090E043
:10D7300040E050E02430310511F441E050E0842312
:10D740009523892B29F08091FF058F5F8093FF053A
:10D7500080E090E0CF3411F481E090E040E050E0D0
:10D760002430310511F441E050E084239523892BC6
:10D7700029F08091FF0581508093FF05CF911F9183
:10D780000F9108950F931F93CF93C82F0E94A76006
:10D7900080E00E94C9728091DC0599279F938F9346
:10D7A0008091A10799279F938F938091DA059927FC
:10D7B0009F938F938091840799279F938F938FE5F1
:10D7C00098E09F938F930CEB12E71F930F93E091D8
:10D7D000DA03F091DB03099580E10E94C9722DB74D
:10D7E0003EB7245F3F4F2DBF8091FC0599279F9343
:10D7F0008F938091370399279F938F938091DB05B7
:10D8000099279F938F938091540799279F938F9384
:10D8100082E798E09F938F931F930F93E091DA0331
:10D82000F091DB03099580E090E02DB73EB7245FCF
:10D830003F4F2DBFCF3211F481E090E020E030E087
:10D8400040916B0150916C014130510509F49A01EE
:10D8500082239323892B29F08091DA058F5F8093AF
:10D86000DA0580E090E0CF3411F481E090E020E030
:10D8700030E04130510509F49A0182239323892B2A
:10D8800029F08091DA0581508093DA0580E090E0FC
:10D89000CF3211F481E090E020E030E042305105D9
:10D8A00011F421E030E082239323892B29F0809129
:10D8B000DB058F5F8093DB0580E090E0CF3411F4CF
:10D8C00081E090E020E030E04230510511F421E0A9
:10D8D00030E082239323892B29F08091DB0581504E
:10D8E0008093DB0520E030E0CF3211F421E030E01E
:10D8F00080E090E04330510511F481E090E0822314
:10D90000932360E070E02091DC052F3010F461E09B
:10D9100070E086239723892B19F02F5F2093DC0575
:10D9200020E030E0CF3411F421E030E080E090E0FE
:10D930004330510511F481E090E08223932360E0AD
:10D9400070E02091DC05222311F061E070E0862375
:10D950009723892B19F021502093DC0580E090E07B
:10D96000CF3211F481E090E020E030E04430510506
:10D9700011F421E030E082239323892B29F0809158
:10D98000FC058F5F8093FC0580E090E0CF3411F4BC
:10D9900081E090E020E030E04430510511F421E0D6
:10D9A00030E082239323892B29F08091FC0581505C
:10D9B0008093FC05CF911F910F9108950F931F93B2
:10D9C000CF93C82F0E94A76080E00E94C972809107
:10D9D000EA0599279F938F938091A10799279F9399
:10D9E0008F938091E60599279F938F938091840769
:10D9F00099279F938F9385E898E09F938F930CEBE3
:10DA000012E71F930F93E091DA03F091DB0309957E
:10DA100080E10E94C9722DB73EB7245F3F4F2DBFF2
:10DA20008091EB0599279F938F93809137039927D6
:10DA30009F938F938091E70599279F938F93809170
:10DA4000540799279F938F9388E998E09F938F932A
:10DA50001F930F93E091DA03F091DB03099580E0C7
:10DA600090E02DB73EB7245F3F4F2DBFCF3211F46A
:10DA700081E090E040E050E020916B0130916C013A
:10DA80002130310509F4A90184239523892B29F03C
:10DA90008091E6058F5F8093E60580E090E0CF34CB
:10DAA00011F481E090E040E050E02130310509F4CC
:10DAB000A90184239523892B29F08091E6058150C3
:10DAC0008093E60580E090E0CF3211F481E090E0B1
:10DAD00040E050E02230310511F441E050E0842371
:10DAE0009523892B29F08091E7058F5F8093E705C7
:10DAF00080E090E0CF3411F481E090E040E050E02D
:10DB00002230310511F441E050E084239523892B24
:10DB100029F08091E70581508093E70580E090E04F
:10DB2000CF3211F481E090E040E050E02330310545
:10DB300011F441E050E084239523892B29F0809152
:10DB4000EA058F5F8093EA0580E090E0CF3411F41E
:10DB500081E090E040E050E02330310511F441E0F5
:10DB600050E084239523892B29F08091EA05815088
:10DB70008093EA0580E090E0CF3211F481E090E0FC
:10DB800040E050E02430310511F441E050E08423BE
:10DB90009523892B29F08091EB058F5F8093EB050E
:10DBA00080E090E0CF3411F481E090E040E050E07C
:10DBB0002430310511F441E050E084239523892B72
:10DBC00029F08091EB0581508093EB05CF911F9157
:10DBD0000F9108950F931F93CF93C82F80EF8093D9
:10DBE000B40180E00E94C9728091BC07E82FFF2732
:10DBF00043E0EE0FFF1F4A95E1F7E058F94F8581AA
:10DC0000282F33278091B805482F55278091380356
:10DC100090913903BA010E94CA79261B370B3F93B2
:10DC20002F938BEA98E09F938F930CEB12E71F934F
:10DC30000F93E091DA03F091DB03099580E10E94F4
:10DC4000C9728DB79EB706968DBF8091BC07E82F2D
:10DC5000FF27E550FC4F808199279F938F938091F8
:10DC6000BC07992701969F938F938CEB98E09F9325
:10DC70008F931F930F93E091DA03F091DB030995E3
:10DC800020E030E08DB79EB708968DBFCF3211F4FB
:10DC900021E030E040E050E080915807843610F4F5
:10DCA00041E050E024233523232B19F08E5F80932D
:10DCB000580720E030E0CF3411F421E030E040E0BC
:10DCC00050E080915807882311F041E050E0242370
:10DCD0003523232B19F082508093580720E030E041
:10DCE000CF3A11F421E030E040E050E08091BC07F1
:10DCF0008F3010F441E050E024233523232B19F01A
:10DD00008F5F8093BC0720E030E0CF3C11F421E02E
:10DD100030E040E050E08091BC07882311F041E002
:10DD200050E024233523232B19F081508093BC0726
:10DD30008091BC07E82FFF27E550FC4F80915807E2
:10DD40008083CF911F910F9108951F93CF93DF93FD
:10DD5000182F80E00E94C9720E94D52199279F93B5
:10DD60008F938DEC98E09F938F93CCEBD2E7DF936A
:10DD7000CF93E091DA03F091DB03099580E10E94F3
:10DD8000C9728DB79EB706968DBF80916D01992798
:10DD90009F938F9389ED98E09F938F93DF93CF9319
:10DDA000E091DA03F091DB0309958DB79EB70696F3
:10DDB0008DBF1F3901F58091C1028823E1F4809164
:10DDC0006D010E940C210E94D52168E770E00E943D
:10DDD000262B8DE00E94C9728CEE98E09F938F9362
:10DDE000DF93CF93E091DA03F091DB0309950F9075
:10DDF0000F900F900F9020E030E01F3211F421E0DF
:10DE000030E040E050E080916D01853010F441E059
:10DE100050E024233523232B19F08F5F80936D016D
:10DE200020E030E01F3411F421E030E040E050E029
:10DE300080916D01823010F041E050E024233523C1
:10DE4000232B19F0815080936D01DF91CF911F91A9
:10DE50000895CF93C82F2091BD032093BE03992727
:10DE60008F32910589F1803391053CF48F30910513
:10DE700009F43CC04F97C1F065C08F34910561F142
:10DE80008F38910509F05EC080916B0190916C0113
:10DE90000197049708F456C086E0289FF0011124EA
:10DEA000EF52FB4F84911FC080916B0190916C01E8
:10DEB0000197049708F446C086E0289FF0011124DA
:10DEC000EE52FB4F84910FC086E0289FF001112491
:10DED000ED52FB4F849107C086E0289FF00111248A
:10DEE000EC52FB4F84918093BD032CC080916B0159
:10DEF00090916C01059779F486E0289FF001112438
:10DF0000EE52FB4F84918093BD0386E090E09093A6
:10DF10006C0180936B0180916B0190916C01892B56
:10DF200089F49091BD0386E0989FF0011124EF528F
:10DF3000FB4F84918093BD038FEF9FEF90936C0113
:10DF400080936B019091BD038091BE039813C0E054
:10DF50000E94CF729091BD0386E0989FF00111243A
:10DF6000EB52FB4F259134918C2FF901099580E0FC
:10DF700090E0CF91089510922D0810922C081092E5
:10DF800031081092300810922F0810922E0810922B
:10DF900032088AE090E00E940D149093C0038093B1
:10DFA000BF030895CF93DF938091BF039091C00387
:10DFB0000E941614882309F4AFC08091BF0390918A
:10DFC000C0030A969093C0038093BF03E0E0F0E0A3
:10DFD0009F0190E05FEFA0E8B6E04BE0ED018B81A0
:10DFE00087FF0BC09F5F8D81E80FF11D8981280F8E
:10DFF000311D8E81851708F4582F4150189647FF20
:10E00000EDCF50933208232B41F52091C30330917B
:10E01000C4034091C5035091C603BB27A52F942F7D
:10E02000832F9093390380933803AA27BB27281B9B
:10E03000390B4A0B5B0BCF01AA27BB27280F391FCF
:10E040004A1F5B1F2093C3033093C4034093C5034F
:10E050005093C603E5E0F0E013C0209138033091FF
:10E0600039032E173F0718F4E21BF30B02C0E0E060
:10E07000F0E0892F9927880F991FE80FF91F35962F
:10E08000F0932D08E0932C08EF3FF10578F4809190
:10E090001D0190911E018E9F90018F9F300D9E9FBC
:10E0A000300D1124C90164E670E013C0CF019695CC
:10E0B00087959695879520911D0130911E01289F87
:10E0C000A001299F500D389F500D1124CA0169E10C
:10E0D00070E00E94CA7970932F0860932E082091F7
:10E0E000C1033091C2032E0F3F1F3093C203209310
:10E0F000C1035EE02131350778F0809130089091BE
:10E1000031080196909331088093300820513E40A9
:10E110003093C2032093C103DF91CF91089500246F
:10E1200022273327442751E0BB27EE27FF27A0E112
:10E13000660F771F881F991F001C221F331F441F63
:10E14000660F771F881F991F001C221F331F441F53
:10E150002AF4050E2B1F3E1F4F1F04C0051A2B0B60
:10E160003E0B4F0B550FBB1FEE1F587F556047FDF1
:10E170005250AA95E9F6E695B7955795E695B79565
:10E180005795852F9B2F08952227332741E0552748
:10E1900068E0880F991F221F331F880F991F221FC5
:10E1A000331F1AF4240F351F02C0241B350B440FF4
:10E1B000551F487F456037FD42506A9551F7569587
:10E1C000479556954795842F0895AA2797FF04C031
:10E1D000809590958A1F9A1F77FF04C0609570956F
:10E1E0006A1F7A1F669F9001779FA001679F300D7D
:10E1F000411D5A1F300D411D5A1F889FF001999FE4
:10E200002E0F3F1F401D511D899F300D411D5A1F6C
:10E21000300D411D5A1FCA01B901112480CF4FB7DB
:10E2200020E430E0F8948091C9008F778093C90092
:10E230008091C9008F7B8093C9008091C9008F7D38
:10E240008093C9005A9A52985B9A539A832F9927C0
:10E250008093CD002093CC008091C8008260809391
:10E26000C80088E18093C9008091CA008F778093AD
:10E27000CA008091CA008F7B8093CA008091CA0037
:10E280008F7D8093CA008091CA008F7E8093CA00E0
:10E290008091CA00877F8093CA008091C9008B7FDC
:10E2A0008093C9008091CA0084608093CA008091E5
:10E2B000CA0082608093CA008091C80087FF03C0B3
:10E2C0008091CE00F9CF8091C90080688093C90009
:10E2D0004FBF08950F931F93CF93DF93482F4F5F46
:10E2E000893108F089C08091E006841710F44093CA
:10E2F000E006CB0183539B4268E170E00E94DE7927
:10E30000A42FBB27FD01EA0FFB1FEF51F94F8081BE
:10E3100091819B01281B390BC90137FF03C09095E0
:10E3200081959F4F069794F48091CA02883C30F4FF
:10E330008091CA02865F8093CA0208C088EC8093ED
:10E34000CA0280916F008F7D80936F00FD01EA0FFC
:10E35000FB1FEF51F94F808191819C01220F331FE8
:10E36000280F391F260F371F37FF02C02D5F3F4F81
:10E37000E901D595C795D595C795CB0101968C1721
:10E380009D0714F4219706C061507040C617D70747
:10E390000CF421968091CA02843BD8F08D010A0FBB
:10E3A0001B1FF801EF51F94F80819181FE01E81B9D
:10E3B000F90BCF0163E070E00E94DE79CB01880F9A
:10E3C000991F860F971F0B5E184FF801918380836A
:10E3D00007C0AA0FBB1FAB5EB84F11961C921E92CE
:10E3E000E42FFF27EE0FFF1FEF51F94FD183C083BA
:10E3F000443011F410924201DF91CF911F910F919F
:10E400000895CF93DF9320913308822F9927807F3F
:10E410009070409709F06CC02F3109F046C0809190
:10E4200034088093CB03209136082093CD0380914C
:10E4300037088093CC03822F99279093E20680932C
:10E44000E106222309F054C08091BA05282F332712
:10E45000220F331FF901EB5EF84F11821082809179
:10E46000BB05A82FBB27AA0FBB1FFD01EB5EF84F12
:10E47000118210828091BD05E82FFF27EE0FFF1F4C
:10E48000CF018B5E984FEC01198218822F51394FC2
:10E49000E90119821882AF51B94F11961C921E9250
:10E4A000EF51F94F1182108223C0C22FCF70CA30B2
:10E4B000F8F48091340880935D088091350880934A
:10E4C0005C088091360880935F08809137088093BC
:10E4D0005E0860915C0870915D088C2F0E946A71E3
:10E4E00060915E0870915F088C2F8F5F0E946A7147
:10E4F000DF91CF910895CF93C82F8F3F49F480913A
:10E50000CE038F3F29F41092D0031092CF0332C074
:10E510002091D003222339F4CF3111F485E001C0DA
:10E5200084E08093D1038091D1039091CF0382172F
:10E53000A0F4892F80958093CF038F3F19F48EEF3D
:10E540008093CF038091CF03C81711F40E9401720A
:10E550001092D0031092CF030BC0E22FFF27ED5C87
:10E56000F74FC0832F5F2093D0039C0F9093CF036E
:10E57000C093CE03CF9108959091CA03933240F493
:10E58000E92FFF27E75CF74F80839F5F9093CA03D3
:10E590000895833218F48D5F8093CA03089590E242
:10E5A000ECE3F8E08FE19193815087FFFCCF089571
:10E5B000CF93CFB723E031E0F8948091C9008F77F3
:10E5C0008093C9008091C9008F7B8093C90080919E
:10E5D000C9008F7D8093C9005A9A52985B9A539ACA
:10E5E000832F99278093CD002093CC008091C80081
:10E5F00082608093C80088E18093C9008091CA003E
:10E600008F778093CA008091CA008F7B8093CA0065
:10E610008091CA0080628093CA008091CA008061A4
:10E620008093CA008091CA0088608093CA0080915C
:10E63000C90084608093C9008091CA00846080937F
:10E64000CA008091CA0082608093CA008091C8008D
:10E6500087FF03C08091CE00F9CF8091C900806808
:10E660008093C9008091C90080648093C9000E9492
:10E67000CF72CFBFCF910895282F99278F709070B8
:10E68000892B31F420958091C903822B8093C90393
:10E6900008958091A101882309F441C080919602D8
:10E6A00085FF0AC082E98093390883E280933A08A3
:10E6B00085E580933B0802C0109239088091A20141
:10E6C0008F3071F48091C9030E94296F882341F033
:10E6D00081E98093390880933A0881E380933B086D
:10E6E0001092A1018091C80085FFFCCF8091C900E4
:10E6F0008F7E8093C9008091C9008E7F8093C9006E
:10E7000080913908882311F48EEF01C08EE7809341
:10E71000CE008091C9038093A2011092C90308958D
:10E720001F920F920FB60F9211248F939F93EF9326
:10E73000FF939091A101992309F040C08091D203E9
:10E74000882361F480913908882311F483E003C0A1
:10E75000813999F481E08093D2030FC0833099F41A
:10E7600080913908882349F0909339088091C90035
:10E770008E7F8093C9008EEF1EC08091C90081609A
:10E780008093C9000EC0833261F48091C9008E7FEE
:10E790008093C9008FEF8093CE0081E08093A10128
:10E7A00014C08091D203E82FFF27E75CF74F8F5FFB
:10E7B0008093D20380818093CE0007C01092D20351
:10E7C0008091C90080618093C900FF91EF919F9172
:10E7D0008F910F900FBE0F901F901895EF92FF92A0
:10E7E0000F931F93CF93DF937C018B01EA01452B9D
:10E7F00039F0F80181918F01F70109952197C9F747
:10E80000E6E0CDB7DEB70C94567AEF92FF920F9305
:10E810001F93CF93DF937C018B01EA01452B41F0DD
:10E82000F8010F5F1F4F8491F70109952197C1F7F8
:10E83000E6E0CDB7DEB70C94567A0F931F93CF93D3
:10E840008C01C62F161634F480E2F8010995C150E8
:10E850001C16D4F3CF911F910F9108950F931F931E
:10E86000CF938C01C62F161634F480E3F801099576
:10E87000C1501C16D4F3CF911F910F910895A5E3B9
:10E88000B0E0E5E4F4E70C942E7A2E96EEADFFAD01
:10E890002E978824992454018091C803882321F459
:10E8A0002C961FAE1EAE2C975EE4452E512C4C0EBE
:10E8B0005D1E6F01B60105C0153239F00894C11C08
:10E8C000D11CF60114911123B9F7A601461B570B71
:10E8D00031F02C968EAD9FAD2C970E9405741123BC
:10E8E00009F46AC20894C11CD11CFF24FDA6FCA631
:10E8F0004FEFE42EF9A6F6010894C11CD11C149127
:10E90000153721F0812F80628837B1F4F0FE0AC0FC
:10E91000F20124E030E0420E531E80809180A280FC
:10E92000B3800AC0F20142E050E0440E551E8081DF
:10E9300091814C01AA24BB24103221F489A588239B
:10E94000D1F61DC0133219F458E0F52AD4CF1A328B
:10E9500011F01D3291F41A3259F4F20182E090E084
:10E96000480E591EE081ECA7EE232CF6E195ECA7AA
:10E9700090E1F92AAFEDFA22BECF1B3211F419A7AC
:10E98000BACF1E32C1F5F6010894C11CD11C1491F6
:10E990001A3279F4F20122E030E0420E531E408137
:10E9A00051813FEF4F3F530714F44FEF5FEFE42ED9
:10E9B000A2CF40E050E0812F80538A30A0F4CA01FA
:10E9C00033E0880F991F3A95E1F7840F951F480FA0
:10E9D000591F410F511D40535040F6010894C11C6E
:10E9E000D11C1491E8CF8FEF4F3F580714F44FEF2D
:10E9F0005FEFE42E85CF103329F4F4FC7CCF90E256
:10EA0000F92A79CF812F81538930D8F440E050E042
:10EA1000CA0123E0880F991F2A95E1F7840F951FFB
:10EA2000480F591F410F511D40535040F6010894A3
:10EA3000C11CD11C1491812F80538A3048F34CA7FC
:10EA40005FCF183619F4A4E0FA2A55CF1C3619F412
:10EA5000B1E0FB2A50CF133661F43E010894611CEB
:10EA6000711CF20122E030E0420E531E8081898346
:10EA70003CC1143421F0143611F0193651F5143418
:10EA800011F431E0F32AF0FE0AC0F20144E050E054
:10EA9000440E551E80809180A280B3800CC0F2018C
:10EAA00082E090E0480E591E808191814C01AA2499
:10EAB00097FCA094BA2CB7FE0AC0B094A09490948E
:10EAC0008094811C911CA11CB11C8DE289A70AE0D5
:10EAD0006FC01F3411F01F3631F41F3411F491E070
:10EAE000F92A08E064C0103779F4F201A2E0B0E03E
:10EAF0004A0E5B1E808191814C01AA24BB2400E157
:10EB0000B0E4FB2A18E753C01337C1F5F20122E045
:10EB100030E0420E531E608071806114710489F4EC
:10EB20003E010894611C711C88E289838EE6F30122
:10EB3000818385E78B838CE68C838D8389E28E834A
:10EB40001F82E7FC13C08E2D992787FD9095AC019D
:10EB500060E070E0C3010E94DA78009729F0382E57
:10EB60003618E3140CF0C3C03E2CC1C0F301019071
:10EB70000020E9F731973E2E3618B9C0153511F04F
:10EB8000153731F4153511F4F1E0FF2A0AE00FC012
:10EB9000183519F0183709F0A0C000E1F3FE07C0DE
:10EBA00081149104A104B10411F020E4F22A19A601
:10EBB000EDA6E7FC02C03FEDF32289E2682E712C3E
:10EBC0006C0E7D1E81149104A104B10421F44DA5A5
:10EBD000442309F47BC0802F9927AA27BB278EA73F
:10EBE0009FA7A8ABB9AB202E332490E0891690E004
:10EBF000990691E0A90690E0B90648F0C501B40174
:10EC00002EA53FA548A959A90E94F17917C0AFEFD9
:10EC10008A169104A104B10449F040F0C401B10185
:10EC20000E94CA799B014427552708C0882D602F70
:10EC30000E94BE79282F3327442755272AAB3BABA8
:10EC40004CAB5DAB0A3059F48AA9880F880F880F46
:10EC50009AA9990F890F382D381B832F10C00031C6
:10EC600039F48AA98295807F482D481B842F07C0DC
:10EC70008AA9880F880F880F582D581B852F90E080
:10EC80002EA53FA548A959A982169306A406B50644
:10EC900008F091E08AA89BA8ACA8BDA88A3010F41F
:10ECA000805D04C0895A183509F48F7DD3018E9395
:10ECB0003D01992309F099CF083041F4F3FE06C0D5
:10ECC000803321F080E3FD0182933F01CE01019664
:10ECD000382E3618F8E23F0E0BC0112309F46CC031
:10ECE0003E010894611C711C1983B1E03B2E19A6EA
:10ECF000032D2DA4231827FC222489A5882311F095
:10ED00000F5F02C0F6FC0E5F020DEF2CFF24C7015F
:10ED100080739070892B49F48CA5801B682F2C96EA
:10ED20008EAD9FAD2C970E941D7489A5882331F06C
:10ED300041E050E0BE01675D7F4F0AC0E6FE0EC0B5
:10ED400080E38AA71BA742E050E0BE01665D7F4FCB
:10ED50002C968EAD9FAD2C970E94EE73C7018073E9
:10ED60009070809749F48CA5801B682F2C968EADEF
:10ED70009FAD2C970E942E74622D2C968EAD9FAD68
:10ED80002C970E942E74832D992787FD9095AC01B6
:10ED9000B3012C968EAD9FAD2C970E94EE73E4FECE
:10EDA00089CD2CA5201B2CA7622F2C968EAD9FAD54
:10EDB0002C970E941D747ECDE2E1CB5C0C944A7AC4
:10EDC0002FB740E0F894E0E0F0E081E28093570054
:10EDD0009491E2E0F0E0809357003491E4E0F0E0B9
:10EDE0008093570084912FBF9E3199F4363941F4B6
:10EDF000893011F441E00DC08A3059F442E009C075
:10EE0000373939F4863011F443E003C0853009F412
:10EE100044E0842F992708959FB7F8948091C90002
:10EE2000877F8093C9008091C9008F7E8093C9003D
:10EE30008091C9008F778093C9008091C9008F7B32
:10EE40008093C9008091C9008F7D8093C90052983A
:10EE50005A9A53985B9A9FBF08951F93CF93DF935D
:10EE6000182F8091C803882309F48DC08091A001D8
:10EE7000181709F488C08091C703882321F40E94E1
:10EE8000E0768093C7038CED99E09F938F93C9E858
:10EE9000D0E1DF93CF93E091DA03F091DB030995A2
:10EEA0000F900F900F900F90812F9927823091052E
:10EEB00001F1833091052CF4009761F0019769F01E
:10EEC00024C084309105D9F084309105ACF00597C9
:10EED000C9F01BC08CEC99E002C08AEB99E09F93CB
:10EEE0008F93DF93CF93E091DA03F091DB030995E1
:10EEF00018C081EA99E0F3CF8EE799E0F0CF80E780
:10EF000099E0EDCF88E699E0EACF89EE99E09F930A
:10EF10008F93DF93CF93E091DA03F091DB030995B0
:10EF200010E00F900F900F900F908091C7038430E6
:10EF300011F0823099F40E940C77812F8150833038
:10EF400018F40E94DA5B1DC0143019F40E94D872C4
:10EF500018C01530B1F40E940F7113C0112389F04D
:10EF60008FEF99E09F938F9389E890E19F938F9320
:10EF7000E091DA03F091DB0309950F900F900F9069
:10EF80000F901093A001DF91CF911F9108950F93DF
:10EF90001F9381E08093C80340919F01E8E1F9E06D
:10EFA00020E030E05FE4849199272F5F3F4F829FFC
:10EFB000B001839F700D929F700D11244627515010
:10EFC000319657FFF0CF40939F01E0EFF8E020E04B
:10EFD00030E057E2849199272F5F3F4F829FB00125
:10EFE000839F700D929F700D1124462751503196CA
:10EFF00057FFF0CF40939F018091C703882321F4EE
:10F000000E94E0768093C70380919F01833459F07A
:10F0100088E190E029E20FB6F894A895809360000B
:10F020000FBE209360008FE394E79093DB038093FF
:10F03000DA038AE19AE09F938F9309E810E11F9326
:10F040000F93E091DA03F091DB0309950F900F9095
:10F050000F900F9087E690E09F938F9380E590E06C
:10F060009F938F931F921F92809102016AE00E94EA
:10F07000BE79892F99279F938F93809102010E94D7
:10F08000BE7999279F938F9380E49AE09F938F9303
:10F090001F930F93E091DA03F091DB03099588E168
:10F0A00099E09F938F931F930F93E091DA03F09170
:10F0B000DB03099580EF98E09F938F931F930F9345
:10F0C000E091DA03F091DB0309958DB79EB7469680
:10F0D0008DBF84E79AE09F938F931F930F93E091E6
:10F0E000DA03F091DB03099583EC80938100809132
:10F0F0006F00806280936F000F900F900F900F90C1
:10F100001F910F9108958091C803882361F0809129
:10F11000A001843011F40E94497380919F018334CF
:10F1200011F01092C80308951F920F920FB60F921C
:10F1300011242F933F934F935F936F937F938F93FC
:10F140009F93AF93BF93EF93FF932091CE00909145
:10F15000A001892F8150833020F4822F0E94DB5B35
:10F160000BC0943021F4822F0E943C7305C095306F
:10F1700019F4822F0E947B72FF91EF91BF91AF91A2
:10F180009F918F917F916F915F914F913F912F91BF
:10F190000F900FBE0F901F901895FB01DC0140FFF0
:10F1A00005C002C005900D9205900D92425050404E
:10F1B000C8F70895FC014150504030F00190061608
:10F1C000D1F73197CF01089588279927089550588E
:10F1D000192E84D001D06AC0BA176207730784075A
:10F1E0009507B1F188F40EF410940B2EBA2FA02DD0
:10F1F000062E622F202D072E732F302D082E842FE0
:10F20000402D092E952F502DFF275523B9F0591B5E
:10F2100049F0573E98F0469537952795A795F040C9
:10F220005395C9F776F0BA0F621F731F841F30F42D
:10F23000879577956795B795F040939517FA0F2EB8
:10F240000895BF1BBB27BA0B620B730B840BF6CF61
:10F25000DEF670C097FB4ED09F3738F0FEE9F91B01
:10F26000982F872F762F6B2F05C061C096958795B5
:10F2700077956795F150D0F73EF49095809570950D
:10F2800061957F4F8F4F9F4F0895E89403C097FB80
:10F290000EF4F3DFB62F672F782F892F9EE9002415
:10F2A00005C09A95BB0F661F771F881F11249923ED
:10F2B000A1F08823B2F79F3F59F0BB0F48F421F427
:10F2C000002011F460FF04C06F5F7F4F8F4F9F4F8E
:10F2D000881F9795879597F9089529C0052E0926C7
:10F2E00007FA440F551F5F3F79F0AA27A51708F0CA
:10F2F00051E04795880F991F9F3F31F0BB27B91701
:10F3000008F091E0879508959F919F91112414C072
:10F3100097FB880F991F9F3F31F0BB27B91708F063
:10F3200091E0879508959F919F91112405C06627CC
:10F3300077278827992708959FEF80EC0895629F8B
:10F34000D001739FF001829FE00DF11D649FE00DDD
:10F35000F11D929FF00D839FF00D749FF00D659F3E
:10F36000F00D9927729FB00DE11DF91F639FB00D3D
:10F37000E11DF91FBD01CF0111240895991B79E00A
:10F3800004C0991F961708F0961B881F7A95C9F735
:10F3900080950895AA1BBB1B51E107C0AA1FBB1F84
:10F3A000A617B70710F0A61BB70B881F991F5A9511
:10F3B000A9F780959095BC01CD01089597FB092E82
:10F3C00007260AD077FD04D0E5DF06D000201AF426
:10F3D000709561957F4F0895F6F7909581959F4FB1
:10F3E0000895A1E21A2EAA1BBB1BFD010DC0AA1F86
:10F3F000BB1FEE1FFF1FA217B307E407F50720F09E
:10F40000A21BB30BE40BF50B661F771F881F991F18
:10F410001A9469F760957095809590959B01AC0161
:10F42000BD01CF01089597FB092E05260ED057FD8B
:10F4300004D0D7DF0AD0001C38F4509540953095A1
:10F4400021953F4F4F4F5F4F0895F6F79095809568
:10F45000709561957F4F8F4F9F4F08952F923F92E8
:10F460004F925F926F927F928F929F92AF92BF92D4
:10F47000CF92DF92EF92FF920F931F93CF93DF9380
:10F48000CDB7DEB7CA1BDB0B0FB6F894DEBF0FBEDD
:10F49000CDBF09942A88398848885F846E847D842A
:10F4A0008C849B84AA84B984C884DF80EE80FD802C
:10F4B0000C811B81AA81B981CE0FD11D0FB6F894A2
:10F4C000DEBF0FBECDBFED010895EE0FFF1F05900B
:10F4D000F491E02D0994F999FECFB2BDA1BDF89A3F
:10F4E000119600B40895F7DF01921A94E1F7089598
:10F4F000F2DFE02DF0DFF02D0895F999FECFB2BDD7
:10F50000A1BD00BC11960FB6F894FA9AF99A0FBEF5
:10F510000895F3DF012CF1DF112408950190EDDF50
:06F520001A94E1F70895C2
:10F526005E010A010164FF01FFFF01FC01FC01010C
:10F53600737373FF03007D0000C409C4096400539C
:10F54600706F727400004E6F726D616C00004265E0
:10F5560067696E6E6572000051756164726F0000B6
:10F56600640001200B050000ECFF6440415A46642C
:10F57600640A02969696960840403A10FB30380187
:10F5860090D0030090D00300F40105F9FF05780040
:10F59600FF036400020406070808080706040200C1
:10F5A600FEFCFAF9F8F8F8F9FAFCFE000204060780
:10F5B60008080B0A0D0B0C0E0B0F10FA2001017038
:04F5C600FF010F0032
:00000001FF
